:020000040000FA
:100000000C9419100C9438100C9438100C9438106F
:100010000C9410290C9438100C9438100C941B2A52
:100020000C9438100C9438100C9438100C94381030
:100030000C9438100C9438100C9438100C94381020
:100040000C9438100C9438100C9438100C94381010
:100050000C9438100C9438100C94CD2D0C9438104E
:100060000C9438100C9438100C9438100C943810F0
:100070000C9438100C9438100C9438100C94D42331
:100080000C9438100C9438100C9438100C943810D0
:100090000C9438100C9438100C9438100C943810C0
:1000A0000C9438105645523A32343038303300DE32
:1000B00013A9157615C315A812DE158C11681594B1
:1000C00011211244208E158C118C114D2109148C94
:1000D00011A9157615C315A812DE15FC1468154B69
:1000E00014211244208E15F6118C114D2109148C07
:1000F00011A9157615C315A812DE15C1126815973A
:1001000012211244208E15FC118C114D2109148CE2
:1001100011A9157615C315A812DE15231368159AB3
:1001200012211244208E1558158C114D210914B638
:1001300011A9157615C315A812DE158C1168159E28
:1001400012211244208E1505148C114D210914B66C
:1001500011A9157615C315A812DE15EA1168153711
:1001600014211244208E1511168C114D210914B63C
:1001700011A9157615C315A812DE15F01168157AA8
:1001800014211244208E1596118C114D210914B69C
:10019000118C118C118C11A8128C11F6158C11A7D1
:1001A00011211244208C118C118C114D218C118C39
:1001B00011A9157615C315A812DE158C116815AD99
:1001C00013211244208E15A8138C114D2109148C73
:1001D00011A9157615C315A812DE1557126815DF7B
:1001E00013211244208E1502128C114D2109148CFA
:1001F00011A9157615C315A812DE155F126815E34F
:1002000013211244208E158C118C114D2109148C50
:1002100011A9157615C315A812DE156412681545C7
:1002200010211244208E15CC148C114D2109148CF0
:1002300011A9157615C315A812DE158C1168153A8B
:1002400010211244208E15E7138C114D2109148CB6
:1002500011A9157615C315A812DE152C126815C143
:1002600014211244208E1533168C114D2109148C43
:1002700011A9157615C315A812DE153812681506D2
:1002800016211244208E153D158C114D2109148C18
:100290001129121E15B813A8127D12431289128D4E
:1002A00011211244208C1113128C114D218C119CA0
:1002B000ACCCB6F400C111214191A131B171F19CD6
:1002C000ACCCB6F4367491A1C111214131F1714425
:1002D0004547000055534552000052414400005329
:1002E0004849465400005052474D0000414C504888
:1002F000410000C0C1C2FFC4C5C618808182C3844A
:100300008586877071728374757677303132733475
:1003100035363710111213141516170304050A0881
:10032000060BFF0209070D010C00FF53554E004D4F
:100330004F4E00545545005745440054485500461B
:1003400052490053415400004A414E004645420084
:100350004D415200415052004D4159004A554E0006
:100360004A554C0041554700534550004F435400F7
:100370004E4F5600444543000000030205000305AC
:100380000104060204464B3A3A494A483A3A3A3A94
:100390003A4C4F3A3A3A3A3A3A3A3A3A3A3A3A3A96
:1003A0003A3A4D3A3A000000000000000000000018
:1003B000000000003FFF3C0000000000003FC000C4
:1003C0000000001540002A800017D7D42BEBE83F2F
:1003D000FFFC02828007F4D01F7DF40F3DF0020A7B
:1003E000803C0078001E8007A0142800281F47F4D6
:1003F0003C343C2F8AF80002080000001440002A18
:10040000000000000007FFD03E00BC2000080000F4
:100410000034001C2F55F802AA80000000024C6036
:10042000017F50006E40020820003C0003FFC00026
:100430003C000000000000000003D80000000000A5
:1004400000003C00003C00003C00002800000000D0
:100450000000F0000000000000000078001E80078F
:10046000A0002800001FFFF43C1E3C3DF57C0AAABA
:10047000A005003C3FFFFC00003C0000001F01FC09
:100480003C1FBC3DF83C0A80281F00F43C143C3D56
:100490007D7C0A82A0007F00078F003FFFFC000ADE
:1004A000003FF0F43CF03C3CF57C282AA01FFFF410
:1004B0003C3C3C3C3D7C280AA03C00003C1FFC3DF1
:1004C000F8002A80001FD7F43C3C3C3D7D7C0A822A
:1004D000A01FF4F43C3C3C3D7D7C0AAAA000000037
:1004E00001414002828000000000000001414402FE
:1004F00082A0000000001D0001E2D00E002C0000D0
:100500000001414003C3C003C3C000000004000455
:100510000B407800B7800008001F00003C1F3C3DE6
:1005200078000A800006AAA431AA4C24AA4C02AA88
:100530000007FFFC3E0F002F5F5402AAA83FFFFCFC
:100540003C3C3C3D7D7C0A82A01FFFF43E00BC3D4C
:10055000007C0A00A03FFFFC3C003C2F55F802AA9B
:10056000803FFFFC3C3C3C3C283C2800283FFFFCF3
:100570003C3C003C28002800001FFFF43C003C3CB1
:100580000F7C080AA03FFFFC003C00157D542AAAFE
:10059000A83C003C3FFFFC3C003C0000001400F481
:1005A0003C003C3FFFF82800003FFFFC003C0017E8
:1005B000C3D42800283FFFFC00003C00003C0000A2
:1005C000283FFFFC0B40001F55542AAAA82FFFFC10
:1005D00002D000157D542AAAA81FFFF43C003C3D20
:1005E000557C0AAAA03FFFFC3C3C003D7C000AA0D1
:1005F000001FFFF43C053C3D57FC0AAAA03FFFFC4E
:100600003C3D003D7EF40AA0281FF4343C3C3C3CB9
:100610003D7C080AA03C00003FFFFC3C00000000BD
:10062000003FFFF400003C15557C2AAAA03FFF4084
:100630000000B41555E02AAA003FFFF80007801516
:1006400057D02AAAA83D417C02BE8017EBD42800CF
:10065000283FD400003FFC3FE8000000003C01FCC4
:100660003C1E3C3DE03C2A00281555543EAABC3CAB
:10067000003C0000002D000002B400000AD0000081
:10068000281400143C003C3FFFFC00000001E00087
:100690001E00000B400000A00000003C00003C00D9
:1006A000003C0000282D000002D0000000000000E7
:1006B000000051F400F33C00F774002AA83FFFFC4F
:1006C00000F03C00F57C002AA0007FF400F03C0024
:1006D000F03C002020007FF400FC3C157D7C2AAA21
:1006E000A8007FF400F33C00F73C002A20057D546D
:1006F0003EBEA83D28000A0000007D1400F33C0027
:10070000F77C002AA03FFFFC00780000F554002A87
:10071000A80050003CFFFC0000000000000000F4B6
:1007200000503C3CFFF80000000FFFFC0007D00029
:10073000382C0000081400003FFFFC0000000000FF
:100740000000FFFC002D00007D5400AAA800BFFCA3
:1007500000F80000BD54002AA8007FF400F03C001F
:10076000F57C002AA000FFFC007AD000F5F0002AFA
:1007700080007FD000F0F0007FD400AAA800FFFC2A
:1007800000780000F400002800007D3C00F33C00ED
:10079000F37C00A0A015F5502AFABC00007C0000F4
:1007A000A000FFF400003C00557C00AAA000FF4020
:1007B0000000B40055E000AA0000FFFC0001E000CA
:1007C00055F400AAA800F47C002BA0007EF400A041
:1007D0002800FD14000F3C005F7C00AAA000F07C04
:1007E00000F3BC00FE3C00A02801C0001FFFFC0B72
:1007F000EAA8008000000000555555AAAAAA0000EA
:1008000000003C00557D55AABEAA003C0000FFC078
:1008100005FFD402FFE0002E000001F41557F82D6B
:1008200010000280003FFFFC30000C30000C300054
:100830000C3FFFFC31554C32AA8C30000C3FFFFCC2
:1008400031554C32AA8C33FFCC30000C30000C30C8
:10085000000C35555C31554C32AA8C30000C3555A6
:100860005C31554C32AA8C33FFCC35555C2AFFA83D
:10087000000000000000000000000000555400AA25
:10088000BC00003C00003C00557C00AAA800000011
:1008900000003C00003D55002AAA000000000000B6
:1008A000001555003EAA003C00003C00003C000042
:1008B0003C00003C00003C00557C00AABC00003C11
:1008C00000000000555555AABEAA003C00003C009F
:1008D000003D55003EAA003C00003C00557D55AA55
:1008E000AAAA000000005FFF07A0057807FEF03EFF
:1008F00000F03FFFBD2AAA0AF555FFD400502B4057
:10090000BFC2F007C0BCFF007CABC0A05F80001F6F
:10091000FFFFFFFFFFFF800FFF000FFF400FFFFFF4
:10092000FF2FFFFFFFFFFCFFFFFCF00000F00000C7
:10093000F00000FFFFFCFFFFFCFFFFFFFFFFFFFFDA
:10094000003FFF003FFF407FFFFFFF2FFFE0FFFF63
:10095000FCFFFFFCC003FCC003FCD007FCFFFFFC56
:10096000BFFFE01FFFFFFFFFFFFF8000FF0000FF52
:100970004000FFF0002FF000FFFFD0FFFFFC000B56
:10098000FC0003FC0007FC00FFFC00FFE0FFFFFF92
:10099000FFFFFFFF0000FF0000FF40003FFFFF0AD6
:1009A000FFFFFFFFFCFFFFFC0003FC0003FC000750
:1009B000FCFFFFF0FFFE80FFFFFFFFFFFFFF003F98
:1009C000FF003FFF003FFF0000FF0000FFFFFCFFB4
:1009D000FFFCC003FCC003FCC003FC0003FC0003DD
:1009E000FCFFFFFFFFFFFFFF003FFF003FFF002A6C
:1009F000FF0000FF0000FFFFFCFFFFFCC00000C085
:100A000000008000000000000000001FFFFFFFFF4B
:100A1000FFFF8000FF0000FF4000FFF0002FF0000C
:100A2000FFFFD0FFFFFC000BFC0003FCFF07FCFFF7
:100A3000FFFCFFFFE0FFFFFFFFFFFF00003F0000A4
:100A40003F00003FFFFFFFFFFFFFFFFFFCFFFFFC3A
:100A5000C00000C00000C00000FFFFFCFFFFFCFF63
:100A60000000FF0000FF5555FFFFFFFFAAAAFF008F
:100A700000FF00000003FC0003FC5557FCFFFFFCD7
:100A8000AAABFC0003FC0003FC000000000000FF18
:100A90000000FF0000FFFFFFFFFFFFFF000000FF5F
:100AA000D000FFFC000BFC0007FCFFFFFCFFFFE099
:100AB000000000FFFFFFFFFFFF00003F0001FF00FD
:100AC0001FF8FFFF80FFF800FFFFFCFFFFFCD000D6
:100AD00000FD0000BFD0000BFFFC00BFFCFFFFFFCC
:100AE000FFFFFF0000000000000000000000000009
:100AF0000000FFFFFCFFFFFC0003FC0003FC000301
:100B0000FC0003FC0003FCFFFFFFFFFFFF0AFF5098
:100B1000000FFF05FFA0FFFFFFFFFFFFFFFFFCFF30
:100B2000FFFC000000000000000000FFFFFCFFFFD2
:100B3000FCFFFFFFFFFFFF2BFF50002BFF00002BF0
:100B4000FFFFFFFFFFFFFFFFFCFFFFFC0000005067
:100B50000000FF5000FFFFFCFFFFFC1FFFFFFFFF37
:100B6000FFFF8000FF0000FF4000FFFFFF2FFFFF9F
:100B7000FFFFD0FFFFFC000BFC0003FC0007FCFFA5
:100B8000FFFCFFFFE0FFFFFFFFFFFFFF003FFF0055
:100B90003FFF407FFFFFFF2FFFFEFFFFFCFFFFFC3B
:100BA000C00000C00000C00000C00000000000172E
:100BB000FFFF7FFFFFFF8000FF0000FF4000BFFF3F
:100BC000FF2BFFFFFFFF50FFFFF0000BFC0FF6FCB9
:100BD0000AFF6CFDBFF4FFDBFCFFFFFFFFFFFFFF21
:100BE000003FFF003FFF407FFFFFFF2FFFFEFFFFA3
:100BF000FCFFFFFCFF0000FFD000EFFD00C2FFFC88
:100C0000002FFC17FFF57FFFFFFF80BFFF003FFFB6
:100C1000403FBFF02F2BF00A003F50403FF4C00B85
:100C2000FCC003FCD007FCFFFFF8FFFFA0FF0000A3
:100C3000FF0000FF5555FFFFFFFFAAAAFF0000FFBE
:100C40000000000000000000555554FFFFFCAAAA58
:100C5000A8000000000000FFFFFFFFFFFF000000F2
:100C6000000000000000FFFFFFFFFFFFFFFF50FF3D
:100C7000FFF4000BFC0003FC0007FCFFFFF8FFFF84
:100C8000A0FFFFFFFFFFFF000000000000000000CA
:100C9000FFFFFFFFFFFFFFD000FFFD0000BFD00000
:100CA0000FFC007FE0FFFE00FFE000FFFFFFFFFF03
:100CB000FF000000000000000000FFFFFFFFFFFF3B
:100CC000FFFFFCFFFFFC017FA03FF00002BF50FFD1
:100CD000FFFCFFFFFCFF5000FFFF5000AFFF0000D4
:100CE0003F005FFFFFFFA0FFA0000017FC17FFFC05
:100CF000FFE800F00000FFD4002BFFFC002BFCFFFE
:100D0000FFD0FFFFFD0000BF00000F00007FFFFFCE
:100D1000FEFFFFE0000000000000D55554FFFFFC7F
:100D2000EAAAA8000000000000FF0000FF0000FF8A
:100D30000007FF007FFF07FFFFFFFEFFFFE007FF49
:100D4000FC7FFFFCFFE3FCFE03FCE003FC0003FC74
:100D50000003FCFFFFFFFFFFFFFF0000FF0000FF9D
:100D60000000FF0000FF0000FFFFFCFFFFFC00038E
:100D7000FC0003FC0003FC0003FC0003FC14000067
:100D80003FD4002BFFD4002BFF00002B00000000FD
:100D90000000000000000000000000D40000FFD4AC
:100DA000002BFFC0002BC0FF0000FF0000FF000071
:100DB000FF0000FF0000FFFFFFFFFFFF0003FC003C
:100DC00003FC0003FC0003FC0003FCFFFFFCFFFF2F
:100DD000FC001F0001FF001FFFFFFFFFFF2FFFFFB1
:100DE00002FF00002F00000000000000FFFFFCFFDA
:100DF000FFFCFFFFFC0000000000000000000000FE
:100E000000000000000000000000000000000000E2
:100E10000003FC0003FC0003FC0003FC0003FC00D7
:100E200003FC0003FC0000000000000000000000C4
:100E300000000000000000000000000000000000B2
:100E400000000000000000000000000000000000A2
:100E50000000000000555555FFFFFFAAAAAA000098
:100E600000000000000000000000554154FFC3FCDA
:100E7000AA82A8000000000000555500FFFF00AA4C
:100E8000AA00000000000000FFFF00FFFF000000BC
:100E90000000000000000000000000000000000052
:100EA000000000000FF00FFFFF0FFFFF000FF00F1B
:100EB000FFFF0FFFFF000FF03FC000FFFFC0FFFF6D
:100EC000C03FC000FFFFC0FFFFC03FC0000055543F
:100ED00007FFFF0FE02FFFFFFFAFEAAF0FF40F0296
:100EE000FC0200540040FF40C02FC0FFFFFCEAAFEF
:100EF000E8F57FC0FFFE0001540003FC0002A801DA
:100F000000017F017FFE3FFE803E80000001400126
:100F10007FC07FFE80FE800080000003FC0003FC99
:100F20000000000101551F1FFFFF3E03FF3FDFE0F0
:100F30000AFA00000003FFFD40EAAFF04002FCF5B2
:100F400000FCBFF5F802FFD0FFFAB0000000FFFF81
:100F500000FFFF0000000000000000000000000093
:100F60000000000000000000000000000000000081
:100F700000000000000000000007FF01FFFF0FFA63
:100F8000007E0000A80000000000000000FF4000FC
:100F9000FFFD0002BFC00002F40000A80000000036
:100FA0000000F400003F40000BFD5500BFFF0002B1
:100FB000AF00000000000000007C0007F055FF803B
:100FC000FFF800EA0000000000003D0F000BDF000A
:100FD00015FF003FFF002AFF0007EF003E0FF07CE7
:100FE00000F7E000FF5400FFFC00FFA800FBD0006A
:100FF000F0BC0000000F00000F00155F003FFF0075
:101000002AAF00000F00000FF00000F00000F554C0
:1010100000FFFC00FAA800F00000F000000000074C
:1010200000000F00000F00005B0007CF01FA0F0067
:10103000000B400000C00000C00000940000CF4042
:1010400000C2BD0080000000000500000F00000F7E
:1010500000000F00000F00000F00000F500000F014
:101060000000F00000F00000F00000F00000F000D0
:101070000000000702F50F000BCF0000A700000FD3
:1010800000000F00000B400000C17E00CF80006810
:101090000000C00000C00000800000000000000050
:1010A0000000000100017F017FFE3FFE803E8000C6
:1010B000000140017FC07FFE80FE800080000000B4
:1010C000000000000017FFFF7FFFFFFF8001FF000F
:1010D0001FFF41FFBFFFFF2BFFFFFFFF50FFFFF48C
:1010E000FF8BFCF803FC8007FCFFFFF8FFFFA0006C
:1010F000000007FC007FFD55FFFFFFAAAAAA000021
:10110000000000000003FC0003FC5557FCFFFFFC3F
:10111000AAABFC0003FC0003FC1FF0007FF000FF03
:101120008000FF0001FF401FFFFFFF2FFFF8001F9F
:10113000FC01FFFC1FFBFCFF83FCF803FC8003FCAD
:101140000003FC1FF000FFF000FF8000FF003FFFE6
:10115000407FFFFFFF2FFFE0003FD0003FFC000B70
:10116000FCC003FCD007FCFFFFFCBFFFE000007FDA
:101170000007FF007FF807FF807FFD55FFFFFFAAF4
:10118000AAAAFF0000FF0000FF0000FF0000FF55BB
:1011900054FFFFFCFFAAA8FFFFFDFFFFFFFF00FFBA
:1011A000FF00FFFF00FFFF00FFFF002F003FD00008
:1011B0003FFC000BFC0003FC4007FCFFFFFCFFFFB3
:1011C000E01FFFFFFFFFFFFF807FFF00FFFF00FF2B
:1011D000FF00FFAA002FFFFFD0FFFFFC800BFC00E9
:1011E00003FC4007FCFFFFFCFFFFE0550000FF0091
:1011F00000FF0000FF0001FF001FFFFFFFFFFFF8DF
:10120000000000000000155554FFFFFCFAAAA8805A
:1012100000000000001FFFD0FFFFFFFF80BFFF00A6
:101220003FFF407FFFFFFF2FFFE27FFFD0FFFFFC6C
:10123000E00BFCC003FCD007FCFFFFFCFFFFE01F3E
:10124000FFF5FFFFFFFF80BFFF003FFF407FFFFF75
:10125000FF2FFFFF003FD0403FFCC00BFCC003FC52
:10126000C007FCFFFFFCFFFFE06FFFF9F4550FFC28
:101270000A8FFCFFF3FC054FFCAA0FE7FFF6BFFF48
:10128000E4C1547CCA80FC3FFCFCC540FCC2A8FC05
:101290007FFF6C00000700000F00000F00000B0034
:1012A0000000000000000000400000C01500C7E87A
:1012B000009E000000000000000000000000000789
:1012C00000007F0007F8007F8007F8003F800038AB
:1012D0000000400000F40000BF40000BF40000BF1D
:1012E00040000BF00000B0000FF0000FF0000FF016
:1012F000000FF0000FF0000FF0000FF00FF0000FE4
:10130000F0000FF0000FF0000FF0000FF0000FF0F2
:10131000003400003F40000BF40000BF40000BF41D
:101320000000BF00000B0000700007F0007F800786
:10133000F8007F8000F8000080000017FC007FFCB0
:1013400000FF8001FF001FFF41FFBFFFF82BFF8060
:10135000000000000000555154FFF3FCAAA2A800B1
:1013600000000000002FFFF902AA8F00000F00000C
:101370000B000000000000000000BFFFE0CAAA0050
:10138000C00000800000000000000000000000001D
:101390000000003FC0003FC0003FC0003FD0003F02
:1013A000FF000BFF1FFFD0FFFFFCFF8BFCFF03FCC8
:1013B000FF03F8FFFFFCFFFFFC0FFFFF0FFFFF0025
:1013C000001F00003F00003F00003F00000BFFFF38
:1013D000FCFFFFFCF80BFCC003FCD007FCFFFFFC8C
:1013E000FFFFE000007F0003FF0003FE0003FC009E
:1013F00003FD0003FF0000BFFFFFD0FFFFFC000B59
:10140000FC0003FC0007FC000FFC000FE0000001E3
:1014100000001F00003F00003F00002F0FFFFF0FE4
:10142000FFFFFFFFD0FFFFFCE00BFCC003FCD00779
:10143000FCFFFFFCFFFFFC00007F0003FF0003FE3A
:101440000003FC0003FD0003FF0000BFFFFFD0FF0F
:10145000FFFC3FCBFC3FC3FC3FC3FCFFC3FCFFC30F
:10146000FC400000F40000FC0000FC0000FC000058
:10147000FC0000E000000000000000000000000090
:101480000000000000000000000000400000F40028
:1014900000FC0000FDFFF4FCAAA0FC0000E000003E
:1014A000000000000000000000000000000000003C
:1014B0000000000000400000F40000FC0000FDFF00
:1014C000FDFCAAA8FC0000E00000000000001500E0
:1014D00007E800AA00000000000000000000004033
:1014E0000000F40000FC0000FDFFFDFCAAA8FC00C9
:1014F00000E0000000000000150007E800AA00005E
:10150000AF400002BD00000000400001F4000FFCED
:10151000000FFDFFF7FCAAA0FC0000E000000000A7
:1015200000C01500C7E8002A0000AF400002BD005F
:10153000000000400001F4000FFC000FFDFFF7FC6D
:10154000AAA7FC000FE0000B000000C01500C7E8D0
:10155000002A00006F4000C2BD008000000000159E
:1015600000003F00000000000500000F0000000028
:101570000000555550FFFEA000BF00555F00FFFF63
:1015800000001600000000000FF0000FF0000FF048
:10159000000FF5000FFF15FFF03FAFF00FF5FC0F48
:1015A000FFA85FF000FFF0000FF0000FF0000FF059
:1015B00000FD4000FFFD40FC2BFDFC002FFD000264
:1015C000FFC000FFC0000005FC05FFFCFFA0FCE021
:1015D00000FC0001FC000FFC000FFC0000000000FC
:1015E000000000000000070001FE007F800FE00007
:1015F0000001FC007FFC1FE0FCFF00FC0BD0FC00A6
:10160000BFFC0000FC00000100000F00003F0000D4
:101610003F00003F00003F00003EF001F0C17FF0BE
:10162000DFFA00E00550DFFFF0EA03F0000A0000F7
:10163000000500007F0003FF0003F80003FD000128
:10164000FF0003FAFFFF40FFFFF0A00FF0001FE0D4
:1016500057FF50FFFFF0AA03F017FFFF3FEAAAFE73
:101660000054FC00FCFF01FD3FFFFF0BFE8FFFFF5E
:10167000FFABFEAA00FF0000FF0001FF00FFFE001D
:10168000FFF80000000114001FFC007FFC00FCFDBF
:10169000403F3FFFFF0ABFFF5FF500FFFFF0800202
:1016A000FC0003F8517FE0FFFE00EA8000001FD439
:1016B00001FFFD07F82F0FF00F0FF00F0FF00A02D8
:1016C000FC001FFD00FFFFD0F00BF4E003FCC003A3
:1016D000FC8003FC000FF000001500003F07FFFF37
:1016E0003FFFFFFE003FFC002ABF00000003FC019B
:1016F0005FFCFFFFFCFEA3FC0003FC0003FC0003F7
:10170000FC0000FC005FFF0FFEFE3F80FCFE00FCC3
:10171000FD00FC3F4000FC0000FFD400FEFFC0FCC9
:101720000BF0FC02FCFC01FC0007E00000140001CF
:10173000F80013F007F3C0FE83F0A002FF00000AD8
:101740000155001FFFD07E02FCFC00FCFC07E0FFFF
:10175000FFFCAAAAA800001F0001FE0173F05FE3CE
:10176000F0F803F50000BF00000AFFFF40FEAFF4F1
:10177000FC02FCFC00FCFC01FCFC03F0A8000000E7
:1017800000500000F0007CF51FE0FF3E000000006C
:10179000000000000000FC0000FC5555FCFFFFFCB1
:1017A0000000FC0000FC00000000005F0001FE01E2
:1017B000F3F05FA3F0F802FF00002B000000FFFD34
:1017C00040AAAFF40002FC0001FC555FF8FFFE8068
:1017D0000000000003FF0010AA45F0003F80002831
:1017E00001FF0002AA000000FFFFD0AAABFC00002E
:1017F000FC0005F8FFFFFCAAAAA8000000000000FA
:1018000000000005FFFF3FFFFFFE00003C0000005E
:10181000000000001F00003FFFFFFFFFFFE8000087
:1018200000000000000000001FE0003FC0003FD0AB
:10183000000FF00003FC0003FC001FF07F8000FF9E
:101840000000FF00003FC0000FF0000FF0007F809D
:10185000000000FF07F0FF0F007E0BD3F007F3FD41
:101860000F80FF00002FFFFFFCFFFFFC00000000C7
:101870000000000000FFFFFCFFFFFC0017FF01FF5E
:10188000EA0FE8000FC0000FD40002FFD5002BFFC5
:10189000FF50FCAFFDFC000BFC0000000007FC5FEC
:1018A000FEFCFA80FC400000F40000FC0000FDFF9C
:1018B000F4FCAAA0FC0000E0000000000000000012
:1018C0000000000000000000000000000000000018
:1018D00000000003FC0003FC0003FC0003FD000308
:1018E000FF0000BF07FFD03FFFFC3F8BFC3F03FC26
:1018F0003F03F8FFFFFCFFFFFC0FFFFF0FFFFF00A0
:10190000001F00003F00003F00003F00000BFFFFF2
:10191000FCFFFFFCF80BFCC003FCD007FCFFFFFC46
:10192000FFFFE000000700003F00003F00003F0015
:10193000003F00003F00000BFFFFD0FFFFFCE00B6B
:10194000FCC003FCC003FCF00FFCF00FE000000142
:1019500000001F00003F00003F00002F0FFFFF0F9F
:10196000FFFFFFFFD0FFFFFCE00BFCC003FCD00338
:10197000FCFFFFFCFFFFFC00000100001F00003F18
:1019800000003F00003F00003F00000B555540FFA6
:10199000FFF4EFEFFC0FC3FC4FC3FCFFC3FCFFC31E
:1019A000FC000003007FFF03FFFF03FE0303FD03B2
:1019B00003FFC000BFC0FC0000FFFFFCFFFFFCFCFA
:1019C0000000FC000000000000000000007F000399
:1019D000FF0003FE0003FC0003FD0003FF0000BF47
:1019E000FD03F4FFC3FF2FC0BF0FC03F1FC07FFF29
:1019F000FFFFFFFFF803FFFF03FFFF0000070000EA
:101A00000F00000F00000F000002FFFFFCFFFFFCB3
:101A1000F80000F00000F40000FFFFFCFFFFFC00F6
:101A2000000000000000001500FF3F00FF3F000025
:101A300000000000000000000000400000FFFFFC6C
:101A4000FFFFFC000000000000000000000000009C
:101A5000000000000000001500FF3F00FF3F0003F2
:101A6000F40003FF0000BF00003F40007FFFFFFFC6
:101A7000FFFFF800FFFF00FFFF0000000000010073
:101A8000003F00003E000000FFFFFCFFFFFC1FF4D2
:101A900000FEBF40E00BFC0000BC000000000000A6
:101AA000000000000000003FFF003FFF00000000BA
:101AB0000000000000000000000000FFFFFCFFFF2E
:101AC000FC00000000000000000700003F00003F95
:101AD00000000F00003F00003F00000BFFFFFCFA7A
:101AE000AAA8D40000FFC000E80000F55554FFFF8D
:101AF000FC00003F00003F00001F00003F00003FCF
:101B000000003F00000BFFFFFCFFFFFCE00000C0F7
:101B10000000C00000FFFFFCFFFFFC00000700000A
:101B20003F00003F00003F00003F00003F00000B6F
:101B3000FFFFD0FFFFFCE00BFCC003FCD007FCFF65
:101B4000FFFCFFFFE0003FFF003FFF0007FE000F2C
:101B5000F0000FF4000FFF0002FFFFFFFCFFFFFC8F
:101B600002FD0000FF0001FF00FFFF00FFF8000082
:101B7000007F0007FF000FF8000FF0000BF4003F9C
:101B8000FF003FFFFFF400FFFF0002FF0000FF0027
:101B900001FE00FFFFFCFFFFFC00003F00003F00D4
:101BA000000700003F00003F00003F00000BFFFF68
:101BB000FCFFFFFCFE0000E00000D00000FC000085
:101BC000FC000000001F0000FF0000FE0000FC0001
:101BD00000FC0000FF0000BFFD0FD0FFCFFC2FC2B4
:101BE000FC0FC0FC0FD1FC0FFFFC02FFE000000364
:101BF00001555703FFFF02AAAB00000300000000DD
:101C00000000FC0000FD5540FFFFF4FEABFCFC01B2
:101C1000FC003FFC003FE000003F00003F000000F0
:101C200000000000000000003F00003FFFFFD0FF69
:101C3000FFFC000BFC0003FC0007FCFFFFFCFFFFA8
:101C4000E000003F00003F00000000000000000036
:101C500000003F00003FFFD000FFFD0002FFD0006A
:101C60003FFC01FFE0FFFE00FFE00000003F00003E
:101C70002A00000000000000000000001500003FE6
:101C8000FFFFD0AAAFFC0007FC03FFF0000BFC55E0
:101C90005FFCFFFFE000003F00002B0000000000A1
:101CA0000000000000001700003F4001FCF41FE8A6
:101CB000BFFE000FF0007FFD00F82FD48002FC0073
:101CC000003F00003F000000000000000015000081
:101CD0003F00003FFD03F4FFC3FC2FC0BC1FC03C0E
:101CE000FF807CFFFFFCFFFFF800003F00003F008B
:101CF000003F00003F00003F00003F00003FC001E8
:101D0000FCC01FFCC1FFFCDFFFFCFFE3FCFE03FC8B
:101D1000E003FC00000000000301400F7FFFFFFE16
:101D2000AAA8F00000A00000000000C00000F00120
:101D300040FFFFFD2AAABF00000F00000A000000BC
:101D4000000000555555FFFFFFAAAAAA0000000099
:101D50000000000000000000555554FFFFFCAAAA37
:101D6000A8000000000000000000F00000FC0000DF
:101D7000FFFFFD2BEAAF000003000002000000009F
:101D8000000F00001F1FFFFFFAABE8E0000080001B
:101D900000FD4000FFFD40FC2BFDFC002FFD00027C
:101DA000FFC000FFC0000005FC05FFFCFFA0FCE039
:101DB00000FC0001FC000FFC000FFC1FFFFFFFFFF9
:101DC000FFFF800FFF000FFF400FFFFFFF2FFFFF00
:101DD000FFFFD0FFFFFCC00BFCC003FCC007FCFFF3
:101DE000FFFCFFFFE000000000000000000000001A
:101DF00000000000000000000000000000000000E3
:101E00000001540003FC0002A80550000FF0000A76
:101E1000A000000550000FF0000AA0000000000024
:101E200000000000001547003FFE002AA00101014C
:101E3000FF02EB0202D76802D10102C0F607C128F7
:101E4000282828140005C20606060602CB0802B39D
:101E5000940BB4E56685FFFF5285FFFF5202B03F49
:101E600003B20005011101FF03C7A6E902362002F3
:101E70003A1102B809012001FF02B92301380129F2
:101E800000010101FF02EB0202D76802D10102C08A
:101E90008007C128282828140005C200000000027D
:101EA000CB1702B3940BB4A56601000040010000FB
:101EB0004002B03F03B20105011101FF03C7A6E9CB
:101EC000023620023A1102B8090120012902B9E3C1
:101ED00001FF02B923013900010101FF02EB0202F7
:101EE000D76802D10102C08007C128282828140021
:101EF00005C20000000002CB170BB4E577F1FFFF2D
:101F00004FF1FFFF4F02B064011101FF03C7A6E9C3
:101F1000023620023A1102B80902D01F012001291D
:101F200002B9E301FF02B9230272000139004255F0
:101F3000494C543A204175672020332032303234E6
:101F40002031333A32383A3233005645523A203053
:101F50002E393030004241543A004E414D45202048
:101F60002020506720426B0050582D3431435800D8
:101F7000426174742E20456D7074793A0044656234
:101F80006F756E636520542E3A004B6579202043AF
:101F900079636C65733A0044697370204379636CAC
:101FA00065733A0052756E20204379636C65733A0D
:101FB00000726573746F72696E672E2E2E002D206D
:101FC000202D00202D2D2D2D200053495A453A005B
:101FD0004D454E5520004449535020004245455040
:101FE0002000434F4D202000535045454400494EAA
:101FF000464F2000534C4545500056494557200058
:102000004D4F52452000524547532000464C414712
:1020100053004D4F44532000414456202000524F5E
:102020004D532000434F4E462000532E494D47004C
:10203000000011241FBECFEFCDBFDFE7DEBF10E4ED
:10204000A0E0B0E4EAE8F9E700E00BBF02C00790C7
:102050000D92A639B107D9F72EE6A6E9B0E401C082
:102060001D92A03FB207E1F70E94003A0C94C33CD6
:102070000C94000090913B6E81E0982790933B6E0A
:102080008093074080930640089510923B6E81E054
:10209000809307408093054080930640089581E037
:1020A0008093EF6E1092FC421092FD428093C85DC7
:1020B000E3EBF2E411921586138E11A617AA82E4BF
:1020C000E13CF807B9F710920843109209431092C7
:1020D0000A4310920C4310920D431092BE5D109271
:1020E000BF5D1092F9421092FA421092FB4280E1D9
:1020F00080930B431092EE5D1092C35D0895809122
:10210000FB42813019F089EF92E408958AEF92E45E
:1021100008958031910508F0C097E3EBF2E427E0E1
:10212000289FB001299F700D112490E080E0DC0110
:10213000A60FB71FA25FBC4B258D30E1239FA001E6
:102140001124248D242B2C930196329687309105EF
:1021500071F70895CF93DF93DC01EB013EE04991E5
:102160004D933A95E1F7DF91CF910895CF93DF93A7
:10217000342FDC01EB01231BA30FB11DC30FD11DB5
:1021800049914D932A95E2F7DF91CF910895242F3D
:10219000DC01261BA60FB11D1D922A95EAF70895B2
:1021A000CF93DF93342FDC01EB01231BA30FB11D71
:1021B000C30FD11D4C9158815D9349932A95D2F755
:1021C000DF91CF910895CF93DF93DC01022E000CB5
:1021D000330B51E0E42FF0E02E173F071CF4DF91A2
:1021E000CF91089580E06115710521F0EB01CE0FCC
:1021F000DF1F8881EA0FFB1F9081C091C85D9C0F93
:10220000980F908380910B43981730F0981B908320
:102210005093C85D4F5FDECF1092C85DFBCF0F9328
:10222000FC0131E0021714F40F91089590E061155C
:10223000710531F0DB01A20FB11D27FDBA959C910C
:1022400080E04115510531F0DA01A20FB11D27FDE3
:10225000BA958C91981B8091C85D981B97FF0FC011
:1022600080910B43980F3093C85D309731F0DF01B8
:10227000A20FB11D27FDBA959C932F5FD3CF10926B
:10228000C85DF3CFCF93DF93242FEC01C60FD11D90
:10229000261B498149932A95E2F71A92DF91CF9143
:1022A0000895CF93DF93DC011092C85D2417A4F04A
:1022B000E42F042E000CFF0B90E06115710521F056
:1022C000EB01CE0FDF1F9881EA0FFB1F808189177A
:1022D00031F081E08093C85DDF91CF9108954F5F29
:1022E000E5CFA0E0B3E48D919C911197E2E0F3E497
:1022F000208131812D933C93A4E0B3E42D913C9156
:10230000119720833183E6E0F3E4208131812D931E
:102310003C9310821182089508950E947111809358
:10232000FC429093FD4208950C9471110E9471112A
:10233000E3EBF2E4292F22952F7022A39F7091A343
:10234000982F92959F7090A38F70878F0895E3EBDD
:10235000F2E482A1829591A1892B90A19295278D7B
:10236000922BECEFF2E49083818308958295837041
:1023700090E09C01220F331F227095958795822B48
:102380009091FF42292F22952F7030E096E1929F85
:10239000F001939FF00D1124E355FF4B9589EDEA71
:1023A000F0E444E0840290011124458949130CC0F3
:1023B000DF01A20FB31F4D915D916D917C91452B73
:1023C000462B472B09F0848B769642E4ED30F407D8
:1023D00061F708956FEC72E48DED92E40C94AA100D
:1023E0006DED72E48FEC92E40C94AA106FEC72E441
:1023F0008BEE92E40C94AA106BEE72E48FEC92E4F4
:102400000C94AA10E3EBF2E4968D858D8295807F83
:10241000248D822B8093EC5D9093ED5D109226428B
:10242000109227420895E3EBF2E4858D20E1829F2C
:10243000C0011124248D822B809326429093274241
:10244000089582958F708093C05D85E08093EE5DE6
:10245000089510920C430895E3EBF2E4858D90E12A
:10246000899F90011124848D822B80930C430895C1
:10247000E3EBF2E480910C43982F9F70948F829548
:102480008F70858F0895E3EBF2E4ACE0B3E48C91B8
:10249000958D40E1949F90011124948D922B9C93F3
:1024A000982F9F70948F82958F70858F089580915B
:1024B0000C4380930A4380EA809307040895809137
:1024C0000A4380930C43089580910C4390910A43F2
:1024D00090930C4380930A4380EA80930704809191
:1024E0000240811109C088ED9DE1809303409093E3
:1024F000044081E08093024008950E947F10FC0117
:102500009081911103C08DE0808308959150908354
:1025100008950E947F10FC0190819F5F90830E942C
:102520007F10FC0120812E3008F010820895109257
:10253000FB42089581E08093FB4208959091F94217
:102540008091FA42981303C081E08093C85D08959A
:10255000CF93C82F0E947F10DC01EC91F0E0ED5486
:10256000FD4BC295CF70C48F0E947F10FC019081FB
:10257000911104C08DE08083CF9108959150908394
:10258000FBCFCF93DF930E947F10DC01EC91D091C1
:102590000943C0910843ED30B1F480919740982FE2
:1025A0009F7B953B11F0873F49F4C093DC42D09369
:1025B0000843C0930943DF91CF910895D093DC4243
:1025C000C093CF42F8CF809196408D3079F58091BD
:1025D0009740853F61F0982F9F70973039F582952D
:1025E0008F70982F977F973009F18B30F9F0D09347
:1025F0000843C09309430E947F10DC01EC91F0E096
:10260000ED54FD4BC58F0E947F10DC01EC91F0E092
:10261000ED54FD4BD48F0E947F10DC01EC91F0E073
:10262000ED54FD4B858D8093CF42C5CFF0E0ED5446
:10263000FD4BD58F0E947F10DC01EC91F0E0ED5452
:10264000FD4BC48FB8CFCF93DF930E947F10DC0186
:102650008C91C09108438D3001F590919740809105
:10266000DC42292F2F7B253B11F0973F49F48093C3
:10267000094380930843C093DC42DF91CF910895D2
:10268000909109432091CF422093084380930943BE
:102690009093DC42C093CF42F0CF20919640D091EE
:1026A000094390E02D3099F520919740253F61F046
:1026B000322F3F70373059F522952F70322F377FE8
:1026C000373029F12B3019F18D549D4BFC01858D4C
:1026D000809309430E947F10DC01EC91F0E0ED54FF
:1026E000FD4B848D809308430E947F10FC019091E4
:1026F000CF42E081F0E0ED54FD4B958F0E947F10BA
:10270000DC01EC91F0E0ED54FD4BD48FC3CF8D5440
:102710009D4BFC01858D809309430E947F10DC0155
:10272000EC91F0E0ED54FD4B848D809308430E94C2
:102730007F10DC01EC91F0E0ED54FD4BD58F0E9451
:102740007F10DC01EC91F0E0ED54FD4BC48F95CF90
:102750008091B2428093FC4208958091B242E3EBB3
:10276000F2E4982F92959F7090A38F70878F0895B1
:1027700080913C6E90913D6E892B91F080913C6EE2
:1027800090913D6E019780933C6E90933D6E81E0F9
:1027900090912542911101C080E08093C85D089519
:1027A0008091C35D823099F71092C35D10922542EB
:1027B0001092B2428091A74290E0E5CF089580E167
:1027C00080930B4308958AE080930B430895E3EBD5
:1027D000F2E482A1829591A1892B90A19295278DF7
:1027E000922B9093AB408093AC4082E08093EE5D5F
:1027F0000895E3EBF2E4968F982F92959F70958F52
:102800008F70848F1092EE5D089583E08093EE5D6B
:102810000895CF93DF93CDB7DEB72E97CDBFDEBF40
:1028200082958F70E82FF0E0E55EFC4FE491DE01C9
:1028300011969E01215F3F4FBD0181E08E0F0E2E4C
:10284000000CFF0BED54FD4B948D9D93E0E08E301A
:102850000CF4E82FA217B30781F78FEC92E40E94E3
:10286000AA102E96CDBFDEBFDF91CF910895809143
:10287000A9422AE0829FC001112420914B6E309121
:102880004C6E8217930720F081E08093C85D089515
:102890001092C85D089584E08093EE5D0895F894E9
:1028A0008091015E8823B9F0E091FF5DF0E0E15195
:1028B000F24A80819091FF5D9F5F9093FF5D9091C0
:1028C000FF5D9F709093FF5D9091015E915090939A
:1028D000015E7894089580E0FCCF9091240895FFE4
:1028E000FCCF8093220808952EE0FC0111922A95D6
:1028F000E9F7089583EB92E40E94741481EC92E46A
:102900000E9474148FEC92E40C947414EEE0F3E4DF
:1029100080EB9AE1DF019C011D9221503040E1F7EC
:102920000895CF93DF93DC01FC013B966B3061F49B
:102930001B968C911B9792919183EA17FB07D9F70D
:102940008083DF91CF9108958C91ED0199819993C6
:10295000CE17DF07D9F71B968C93F3CF9C014097D6
:10296000C09768F0211582E0380749F0C901805FFF
:102970009240419720F081E0203F334008F080E012
:1029800008958091B142882331F00E9471118093A3
:10299000FC429093FD420895CF93DF9380912642AD
:1029A00090912742009731F08D3F910589F0DF919A
:1029B000CF910895C091EC5DD091ED5DCE010E9464
:1029C000AE148823A1F3CE01DF91CF910C9489102E
:1029D0002091D1428091D04230E1839FC0011124E7
:1029E000922B2091CF42822B8093376E9093386E3A
:1029F00081E080930640DBCF0E947F10DC01EC91E8
:102A0000ED30A1F4909197408091DC42292F2F7BEB
:102A1000253B11F0973F39F4909109439093084377
:102A20008093094308959091CF42F8CFF0E0ED54A0
:102A3000FD4B848D80930843858DF2CF80913C6E51
:102A400090913D6E892B51F080913C6E90913D6E3E
:102A5000019780933C6E90933D6E08958091C35D85
:102A60008130D9F7809135428111F7CF82E0809390
:102A7000C35D8091A74290E0ECCF8EE0815078F466
:102A80008091B142882351F08091C15D8D3031F445
:102A90008091CF428093DC428093C0420895E82F1A
:102AA000F0E0ED54FD4B948D20819223948FE6CF7E
:102AB000CF93DF93AFECB2E4CBEED2E43EE04C91A7
:102AC00058815D9349933A95D1F7DF91CF9108955D
:102AD000CF9382958F70E82FF0E0E55EFC4FC491B4
:102AE0000E947F10FC01C083CF91089582958F7062
:102AF000E82FF0E0E55EFC4FE491ACE0B3E421E0C8
:102B000030E002C0220F331FEA95E2F78D919C91CD
:102B10001197822B932B8D939C9308952091BE5DEA
:102B20003091BF5D82958F70E82FF0E0E55EFC4F3D
:102B3000E49181E090E002C0880F991FEA95E2F7E6
:102B40008223932321E0892B09F420E02093C85DA0
:102B5000089582958F70E82FF0E0E55EFC4FE491D8
:102B6000ACE0B3E481E090E002C0880F991FEA95E1
:102B7000E2F7809590952D913C91119782239323B4
:102B80008D939C93089582958F70E82FF0E0E55E19
:102B9000FC4FE49181E090E002C0880F991FEA9514
:102BA000E2F720910C4330910D438223932321E0DF
:102BB000892B09F420E02093C85D0895CF93C82F96
:102BC0000E947F10C295CF70EC2FF0E0E55EFC4FC5
:102BD000E491DC018C910E2E000CFF0B8E171F066A
:102BE00019F481E08093C85DCF910895CF93DF936E
:102BF000AFECB2E4CDEDD2E43EE04C9158815D9370
:102C000049933A95D1F7DF91CF9108958091B142E0
:102C1000811106C00E9471118093FC429093FD4285
:102C20000895E3EBF2E482A1829591A1892B90A112
:102C30009295278D922BE4E0F3E42081318120935B
:102C4000064330930743A2E0B3E42D913C911197E2
:102C500020833183E0E0F3E4208131812D933C93A4
:102C60009083818308958EE0815078F48091B14201
:102C7000882351F08091C15D8D3031F48091CF4235
:102C80008093DC428093C0420895E82FF0E0ED5439
:102C9000FD4B948D2081922B948FE6CFE0E4F4E0FD
:102CA00081818D608183E0E0F4E0818180648183B3
:102CB000E0E6F9E084E0818381E3808308958093F6
:102CC00064098091630987FFFCCF08951F93CF9318
:102CD000DF93C0E0D4E010E41E830E945F161D83E2
:102CE000DF91CF911F91089527E731E0829FF00196
:102CF000839FF00D1124EE5FF14A20E081819281E3
:102D00009695969530E4839FA0011124942B92838D
:102D100090818695869530E4939FA0011124842BA1
:102D200081839695969590832F5F33962D3731F753
:102D3000089527E731E0829FF001839FF00D112471
:102D4000EE5FF14A2DE781819081990F990F382F1D
:102D50003295369536953370932B90839281880FF8
:102D6000880F392F3295369536953370832B8183B2
:102D7000990F990F9283215033962111E4CF089532
:102D8000E2E0FEE58DE190E1DF019C011D92215022
:102D90003040E1F70895E2E0FEE59191DF011197FF
:102DA00098279C939EE6EF31F907B9F70895E2E082
:102DB000FEE59191DF01119798239C939EE6EF31F8
:102DC000F907B9F7089527E731E0829FF001839F63
:102DD000F00D1124EE5FF14A9F0129583E4F819179
:102DE000DF01119786238C93E217F307C1F708954B
:102DF00027E731E0829FF001839FF00D1124EE5F01
:102E0000F14A629FD001639FB00D1124AE5FB14AB9
:102E1000CF0189589E4F21912D93E817F907D9F7D3
:102E2000089570E027E731E0482F429FC001439F9B
:102E3000900D112447E751E08E5F914A0C94BC3C01
:102E40000F931F93CF93DF93182F8AE20E94661689
:102E5000C9E1C10F8C2F0E945F168C2F0E945F1654
:102E60008BE20E94661680E00E945F168CE70E944B
:102E70005F168CE20E94661687E791E0189FE001DA
:102E8000199FD00D1124CE5FD14A8E0109581E4FD3
:102E900089910E945F16C017D107D1F7DF91CF91BA
:102EA0001F910F910895CF93DF938AE20E946616D7
:102EB00089E10E945F1683E20E945F168BE20E9406
:102EC000661680E00E945F168CE70E945F168CE217
:102ED0000E946616C2E0DEE589910E945F168EE6CA
:102EE000CF31D807C9F7DF91CF910895CF93DF9302
:102EF000A82FA052BB0B3CE03A9FC0013B9F900D16
:102F000011248B559C4FC62FC695E7E7F1E04E9FE5
:102F1000D0014F9FB00D1124AE5FB14A33E0C39F83
:102F2000E00111248A1B9B0B60FF30C0AE014D5F96
:102F30005F4FCA0FDB1FA40FB51F3CE0841B950B2E
:102F4000FC01EA0FFB1F2636F1F0E491E2274881ED
:102F50004A7A48834C9145754C93F0E0AF01559502
:102F60004795542F55754881452B4993EE0FFF1F08
:102F7000EA7A4C91E42BED93315011F788E0860FFB
:102F8000DF91CF910895E491E676E1CFAC0FBD1FBC
:102F90003CE08C1B9D0BFC01EA0FFB1F263641F029
:102FA000E491E227EC93315011963111F4CFE6CF42
:102FB000E491E676F7CFFF920F931F93CF93DF93C1
:102FC0008C01D42FF22EC0E0F801EC0FF11D8081AE
:102FD000811107C0862FDF91CF911F910F91FF9034
:102FE00008952F2D4D2F0E947617682FCF5FECCFBD
:102FF000FF920F931F93CF93DF938C01D42FF22E68
:10300000C0E0F801EC0FF11D8491811107C0862FFB
:10301000DF91CF911F910F91FF9008952F2D4D2F8C
:103020000E947617682FCF5FECCF5F926F927F92EE
:103030008F929F92AF92BF92CF92DF92EF92FF92C8
:103040000F931F93CF93DF93CDB7DEB72597CDBFF7
:10305000DEBF89836A834B832C830D831092C45D0A
:103060001092C55D1092C65D41E35BE68091C45D40
:103070009091C55DA091C65DFA0180839183A28382
:103080009A01285B3F4FF90180839183A283455BBE
:103090005F4FFCE6483A5F0749F76AE089E00E9423
:1030A000F816CE0101967C0110E000E096E0692E52
:1030B00022E3C22ED12C80E098E7A1E0BB27F701E4
:1030C00081907F01869C40011124092C000CAA08E4
:1030D000BB08880E991EAA1EBB1EABBEF4017790DA
:1030E000B601F8E07F9E60197109112477FF02C0D4
:1030F0006F5F7F4F75956795600F711F512C8FEF34
:10310000881A980AA80AB80A57101AC00E5C1F4FEE
:103110000A3F110581F689E02596CDBFDEBFDF911C
:10312000CF911F910F91FF90EF90DF90CF90BF90C4
:10313000AF909F908F907F906F905F900C947416DB
:10314000ABBEF40187912FEF49E00E947617682FFC
:103150005394D5CF99E1899F802D112461E0282FC8
:10316000260F30E0A901440F551F240F351F2E5F95
:10317000314AF901E15DF24F9081492F440F440F2C
:10318000D901A05DB24F9C919295969596959370BA
:10319000942B90839C91492F440F440F3296908139
:1031A0009295969596959370942B9C93408194E07C
:1031B000499FA0011124436040832A55314FF901F2
:1031C00010826F5F683159F608952F923F924F92A7
:1031D0005F926F927F928F929F92AF92BF92CF92A7
:1031E000DF92EF92FF920F931F93CF93DF9380E0D4
:1031F00090E8A1E0BB276C017D0128E7D20EE11C1D
:10320000F11C0E94C01630E020E087E7882E992448
:103210009394A1E0B0E05524539450E040E0289D01
:103220003001299D700C389D700C112426C0EBBE16
:10323000F60117918FEFC81AD80AE80AF80A90E049
:10324000EBBEF6018791EFEFCE1ADE0AEE0AFE0A18
:10325000980F092F0095C92FC81B811111C0152582
:103260009A3F70F3625071096E3F8FEF7807F9F65D
:103270004F5F5F4F4330510539F166E070E0D7CFC3
:10328000113001F5C695D0E0FE01EE0FFF1FEC0FE7
:10329000FD1FE60DF71DEE5FF14AE40FF51FC02F8D
:1032A000C80FC0FBAA24A0F8B12CE501C60FD71F98
:1032B0001D0102C0220C331CCA95E2F7E101D08146
:1032C000CD2BC0838150C7CF2F5F3F4F2B303105AF
:1032D00009F0A3CFDF91CF911F910F91FF90EF9055
:1032E000DF90CF90BF90AF909F908F907F906F9026
:1032F0005F904F903F902F900C945317BF92CF92B6
:10330000DF92EF92FF920F931F93CF93DF93362FAD
:103310009AE2899F800111240B51174F83E0689F27
:1033200070011124B0E0A0E085E1B82E50E097E7ED
:10333000C92EDD24D3948A2FAA32B10561F487E027
:10334000830FDF91CF911F910F91FF90EF90DF904E
:10335000CF90BF900895FD01E00FF11FE4916B2D18
:103360000E946E3BBA01680F711D6C9DE0016D9D5E
:10337000D00D7C9DD00D1124CE0DDF1DC90FD11DA8
:10338000CE5FD14AE227E8831196D5CFCF92DF9264
:10339000EF92FF920F931F93CF93DF93D62E92E17C
:1033A000899FE0011124CB51D24E83E0689F8001B8
:1033B000112430E020E089E0C82E50E097E7E92EA4
:1033C000FF24F394822F2231310559F483E08D0DCF
:1033D000DF91CF911F910F91FF90EF90DF90CF90F1
:1033E0000895F901EC0FFD1FE4916C2D0E947A3BCA
:1033F000BA01680F711D6E9DD0016F9DB00D7E9D4D
:10340000B00D1124A00FB11FA90FB11DAE5FB14ABD
:10341000EC932F5F3F4FD6CFCF93DF938AE20E948A
:10342000661689E10E945F1683E20E945F168BE2B6
:103430000E94661680E00E945F168CE70E945F166D
:103440008CE20E946616CDE1D0E180E00E945F161A
:103450002197D9F7DF91CF91089580E10C946616FA
:1034600081E10C946616262F2150330BF901E758A1
:10347000FC4FE49191E0633008F090E0891B282F25
:1034800026952695280F3327331F64E60E946E3B4E
:10349000B901681B7109CB018E0F911D840F911D1D
:1034A00067E070E00E949C3B8F5F0895823021F4BA
:1034B000637081F48DE108958150990B67E070E0AD
:1034C0000E949C3B62E070E00E949C3B9FE1981B45
:1034D000892F08958CE108958D3010F08C50089557
:1034E000811101C08CE00895CF93DF93DC01362F6A
:1034F0004423C1F06A30B0F4E0E0222311F02C93B1
:10350000E1E0ED01CE0FD11D832F6AE00E946E3BFA
:10351000905D9883EF5FEA0FFB2FF11D1082DF9122
:10352000CF910895832F6AE00E946E3B805D8C935B
:10353000E7CFFF920F931F93CF93DF93CDB7DEB703
:103540002597CDBFDEBF0CE912E4D8015096EC916F
:10355000B4E0EB02F00111242FEF40E0682FCF011F
:10356000895D9C4F0E94F8172FEF40E0682F8DE295
:103570000E947617D8011796EC91B4E0EB02F001A7
:1035800011242FEF40E0682FCF018C5B9C4F0E94ED
:10359000F8172FEF40E0682F8DE20E947617F82E83
:1035A000F801608520E041E0CE0101960E94741A86
:1035B0002FEF40E06F2DCE0101960E94DB1725967C
:1035C000CDBFDEBFDF91CF911F910F91FF90089586
:1035D0001F93CF93DF93CDB7DEB72597CDBFDEBF67
:1035E000182F80919E42813009F040C06091AB421B
:1035F00020E241E0CE0101960E94741A2FEF40E0D4
:10360000612FCE0101960E94DB172FEF40E0682F5B
:103610008AE30E947617182F6091A04220E040E0D4
:10362000CE0101960E94741A2FEF40E0612FCE0167
:1036300001960E94DB17682F80919E42813079F4B9
:1036400080919F422FEF40E08C30ACF080E50E94EB
:1036500076172FEF40E0682F8DE40E9476172596AD
:10366000CDBFDEBFDF91CF911F91089560919F4242
:1036700020E240E0BFCF81E4EACFCF93DF93109206
:103680003B6E85E080939B42EFE9F0E4CFE3DEE61A
:10369000AEEDBDE5119219921D9280E4EB3AF80768
:1036A000C9F71092376E1092386EDF91CF9108955E
:1036B00060E089E00E9411178091376E80FF07C09B
:1036C00020E049E060ED8CEE92E00E94F8178091D6
:1036D000376E81FF07C020E049E06AEA86EE92E09B
:1036E0000E94F8178091376E82FF06C020E049E003
:1036F0006CE984E30E9476178091376E83FF06C0E1
:1037000020E049E064E983E30E9476178091376EF8
:1037100084FF06C020E049E06CE882E30E9476174F
:103720008091376E85FF06C020E049E064E881E3C0
:103730000E9476178091376E86FF06C020E049E030
:103740006CE780E30E9476178091376E87FF07C091
:1037500020E049E06EE48FED92E00E94F81780913E
:10376000376E9091386E90FF07C020E049E060E32B
:103770008AED92E00E94F8178091376E9091386E32
:1037800091FF06C020E049E068E287E40E947617D6
:103790008091376E9091386E92FF07C020E049E02B
:1037A00062E084ED92E00E94F8178091376E90916C
:1037B000386E88279370892B39F420E049E060E364
:1037C0008FEC92E00E94F81789E00E94741689E05D
:1037D0000C9420170F931F93CF93DF9380913B6E30
:1037E000882331F10AEE1DE52FE33EE6CFE9D0E470
:1037F000EDE0F2E46EED7DE5D9011B969C91D801D8
:103800008E918D01B4E08B9FA0011124892F8370CC
:10381000842B8295807F4B85840F868B9695969519
:10382000978B21503109219732976017710721F743
:10383000DF91CF911F910F910895CF93DF9388E18E
:10384000EDE0F2E4AFE1BEE601900D928A95E1F77A
:1038500060E087E00E94111760E088E00E94111785
:10386000CDE0D2E485E020E047E0682F8E890E9419
:103870007E1947E0682F8F890E94C619229791E42C
:10388000C53FD90781F78091376E9091386E83706C
:103890009927892B31F420E048E061E088E50E9417
:1038A000761787E00E94201788E0DF91CF910C9473
:1038B0002017EDE0F2E4AFE1BEE691918D9198130F
:1038C00006C082E4E432F807C1F781E0089580E0A1
:1038D0000895DC011596FB0135963E912291321335
:1038E00005C0A817B907C9F781E0089580E00895D9
:1038F000FC01108211821282138214820895DC016D
:103900001596FB0135963E912291231728F0321728
:1039100028F0A817B907B9F781E0089580E0089565
:103920006F927F928F929F92AF92BF92CF92DF92CF
:10393000EF92FF920F931F93CF93DF938B01DB01E5
:103940001D921D921D921C921397EC0122963C0130
:10395000BEE06B0E711CC12CD12C7601C394A991D1
:10396000B0E0A70196010E94E23BF80180809180BF
:10397000A280B380DC01CB01880D991DAA1DBB1D5F
:1039800080839183A283B383AAE0B0E00E94E23BEC
:103990006B017C016C167D0611F7DF91CF911F91B1
:1039A0000F91FF90EF90DF90CF90BF90AF909F90DE
:1039B0008F907F906F900895AC0190E070E0292F78
:1039C000092E000C330B261737070CF00895240F2F
:1039D000351FF90110829F5FF2CF4F925F926F9275
:1039E0007F928F929F92AF92BF92CF92DF92EF928F
:1039F000FF92CF93DF9300D000D0CDB7DEB7F8941D
:103A0000BE016F5F7F4F87E492E40E94901C789420
:103A1000C980DA80EB80FC808CE3882E912CA12C6D
:103A2000B12CC701B601A50194010E94B03B60937F
:103A3000A142CA01B901A50194010E94B03B609363
:103A4000A042C701B60120E13EE040E050E00E9404
:103A5000B03BCA01B90128E130E040E050E00E94EB
:103A6000B03B60939F4280919F420E946C1A80936A
:103A7000AB42C701B60120E831E541E050E00E94C9
:103A8000B03B69017A01C982DA82EB82FC82CA0109
:103A9000B9016C557C498F4F9F4F22E0660F771F0D
:103AA000881F991F2A95D1F721EB3AE342E050E0B5
:103AB0000E94B03B215F3F4F4F4F5F4F82EAC80EDD
:103AC0008FEDD81E84E2E81EF11CC20ED31EE41E48
:103AD000F51E62E056954795379527956A95D1F77B
:103AE000C21AD30AE40AF50AA4E1B0E0A7019601DC
:103AF0000E94E23B2B013C012AE8421A29E0520ACB
:103B000061087108C301B20129E83CE140E050E0DE
:103B10000E94B03B49015A01ADE6B1E00E94E23B90
:103B2000C61AD70AE80AF90AC301B20124E232E749
:103B300040E050E00E94B03BC21AD30AE40AF50A02
:103B4000A8EEB3E0A70196010E94E23B29E837E71F
:103B500040E050E00E94B03B29013A018EE1289FED
:103B6000C0181124A9E5B2E00E94E23B28EE33E040
:103B700040E050E00E94B03BC21AC092A4422EE046
:103B8000421651046104710480F58CE6881A82E1C2
:103B9000980AA108B10821E0421A51086108710889
:103BA00080E3880E8092A2424092A3424091A442B8
:103BB0006091A3428091A2420E94331A8093AC424A
:103BC00081E080939B402496CDBFDEBFDF91CF91F3
:103BD000FF90EF90DF90CF90BF90AF909F908F902D
:103BE0007F906F905F904F9008958BE6881A82E1E6
:103BF000980AA108B1082DE0421A5108610871081D
:103C0000CFCF2F923F924F925F926F927F928F927F
:103C10009F92AF92BF92CF92DF92EF92FF920F935B
:103C20001F93CF93DF93CDB7DEB72997CDBFDEBF0C
:103C3000C090A2420C2C000CDD0820E3C21A28EF31
:103C4000D20A0D2C000CEE08FF083091A342232E5F
:103C5000022C000C330829823A829101233031056D
:103C600048F4245F3F4F29833A8331E0C31AD108D7
:103C7000E108F1081091A442ADE6B1E0A701960178
:103C80000E94E23B4601570122E0B694A794979424
:103C900087942A95D1F7860E971EA81EB91EC701D4
:103CA000B60120E931E040E050E00E94B03B820ED6
:103CB000931EA41EB51EC701B60124E630E040E005
:103CC00050E00E94B03B821A930AA40AB50A2981E7
:103CD0003A812F5F3F4FC901880F991F820F931FB1
:103CE00065E070E00E94883B2EE129803A80229DA9
:103CF000C001239D900D1124810F911D17FD9A95F0
:103D0000FB01E80FF91F9F0150E040E060E070E028
:103D1000CB01E9833A834B835C836D837E838F83FE
:103D200098879401A50160E070E080E090E0A980B0
:103D3000BA80C12CD12CE12CF12C00E010E00E94C3
:103D4000A43C2A5E36494A4051096109710981093A
:103D50009109E0E8AE2EF1E5BF2ECC24C3940E9479
:103D6000ED3B59016A017B018C01A0919F4240917A
:103D7000A0424090A1420A2E000CBB0B20E13EE085
:103D80000E94DB3B042C000C550866087708DC0118
:103D9000CB01840D951DA61DB71D3CE34302A00178
:103DA0001124840F951FA11DB11D1C012D01612C33
:103DB000712C43013A82AB835C826D827E828F825A
:103DC00098869C01AD0160E070E080E090E00E9488
:103DD000A43C29014A01698779831C01F894109257
:103DE000C75DA9E46A2EA2E47A2E8AE0A82EB12C3F
:103DF000C12CD12CE12CF12C00E010E09201A401A7
:103E000069857981C1010E94453CF30121933F01FD
:103E10009201A40169857981C1010E94473C290171
:103E20004A01698779831C0125E532E426153705A7
:103E3000E1F667E472E48FE792E40E94AA107894B6
:103E40002996CDBFDEBFDF91CF911F910F91FF90DB
:103E5000EF90DF90CF90BF90AF909F908F907F902A
:103E60006F905F904F903F902F900895FC0195E0E8
:103E700020E08191980FDF0111979A3060F49C93B4
:103E800090E0211101C09E5F2F5F2E3011F0911143
:103E9000F0CF892F08959A509C9391E0F2CFCF9361
:103EA000803108F06FC0E82FF0E0E75AF04E0C9434
:103EB000D23B691F761F8E1F991FD21FDD1FC21FA5
:103EC000F31FF91F0C201D2025202D2035203D201B
:103ED0004120809146422EE0829FC00111246FEC68
:103EE00072E4895B9D4BCF910C94AA10809146425D
:103EF000CEE08C9FC00111246FEC72E4895B9D4B76
:103F00000E94AA10E0914642CE9FF0011124EA5C83
:103F1000FD4B118A128ACF910C94ED1C8091464280
:103F20002EE0829FC00111246FEC72E48D599D4BED
:103F3000DACF80914642811127C09091364220917C
:103F4000D04280E1289F900111248091CF42806C63
:103F5000822B892380933642809136428F7391F46D
:103F60008091BE5D9091BF5D9F7D8093BE5D90937B
:103F7000BF5D8091BE5D9091BF5D9F7E8093BE5D71
:103F80009093BF5DCF91089523E040E060ED72E42F
:103F900088E392E40E94B61080913B428170809346
:103FA0003B42F0CF809146422EE0829FC001112417
:103FB0006FEC72E481589D4B96CF24E040E06FECAB
:103FC00072E481E492E40E94B6108CE392E40E94D1
:103FD000781C8091364290913742946080933642AB
:103FE00090933742CFCF80913642909137429B7F5A
:103FF000F5CF409136425091374220914642255F9D
:1040000081E090E002C0880F991F2A95E2F7809521
:10401000909584239523E2CF4091364250913742C8
:1040200020914642255F81E090E002C0880F991FF1
:104030002A95E2F7842B952BD1CF409136425091AF
:10404000374220914642285FDBCF40913642509163
:10405000374220914642285FE6CF40913642509148
:104060003742209146422A5FCBCF40913642509151
:104070003742209146422A5FD6CF81E08093464264
:1040800081CF109246427ECF7F928F929F92AF92C5
:10409000BF92CF92DF92EF92FF920F931F93CF9335
:1040A000DF93082F02950F70C02FD0E0E090EC5DF9
:1040B000F090ED5D20EFE22223E0F222E02AFD2ADB
:1040C000E092EC5DF092ED5DC7010E94AE14182FF6
:1040D000882381F0C701DF91CF911F910F91FF904D
:1040E000EF90DF90CF90BF90AF909F908F907F9098
:1040F0000C94891080912642909127428B3F910524
:1041000009F469C08D3F910541F5C154DD4FFE01B1
:10411000C49180E0C7FD8BE0FC2FFF709F2E00E074
:104120002C2F2071822EDBE0D81B90E0FC01E156A1
:10413000FF4B7F01FC2FF0727F2E9C01215C3149E7
:104140006901C074FC01E252F24A5F01901213C08F
:1041500081E08093074080930540DF91CF911F91CC
:104160000F91FF90EF90DF90CF90BF90AF909F9016
:104170008F907F900895882069F06D2F8FE990E4EB
:104180000E949114E12FF0E0ED54FD4B848DF70176
:1041900080831F5F772069F06D2F8FE39EE60E947A
:1041A0009114E12FF0E0ED54FD4B848DF6018083F6
:1041B0001F5FCC2371F06D2F8EED9DE50E94911451
:1041C000E12FF0E0ED54FD4B848D8170F50180838B
:1041D0001F5F0F5FBBCF802FDF91CF911F910F919A
:1041E000FF90EF90DF90CF90BF90AF909F908F9017
:1041F0007F900C944F1F8230A1F038F08430E9F1A9
:10420000C8F0853009F442C00895609146428EE0BE
:10421000689FB0011124695B7D4B8FEC92E40C9494
:10422000AA10609146428EE0689FB00111246D593A
:104230007D4BF3CF80914642811117C08091364269
:104240008F708093CF428091364282958F70809399
:10425000D042809137428F708093D1428091374213
:10426000829581708093D242089523E040E068E314
:1042700072E480ED92E40C94B610609146428EE0B8
:10428000689FB001112461587D4BC7CF24E040E006
:1042900061E472E48FEC92E4EECF6F927F928F92A2
:1042A0009F92AF92BF92CF92DF92EF92FF920F93C5
:1042B0001F93CF93DF93182F12951F708FEC92E40A
:1042C0000E94741480912642909127428B3F910561
:1042D00009F4B9C08D3F910509F440C0892B79F5E7
:1042E000112359F08091EC5D9091ED5D807F93708A
:1042F000812B8093EC5D9093ED5D0091EC5D1091CE
:10430000ED5DC8010E94AE148823C9F0003111058B
:1043100010F00053110987E0809FE001819FD00DCC
:104320001124C25FDC4BAFECB2E467E04991542F3B
:1043300052955F704F704D935D936A95B9F7DF9119
:10434000CF911F910F91FF90EF90DF90CF90BF9092
:10435000AF909F908F907F906F900895153001F5EA
:104360008091376E9091386E9093D1429C0194E089
:10437000369527959A95E1F72F702093D0428F704C
:104380008093CF4280913B6E8823C9F21330B8F2FC
:104390001530A9F281E08093074080930540CFCF8C
:1043A000E12FF0E0E155FD4FC4910BE0C7FF00E0C5
:1043B0002C2F2F70822ED0E0912C3C2F3071732E39
:1043C000802F90E0DC01A156BF4B7D01BC2FB07265
:1043D0006B2E9C01215C31496901C074DC01A25241
:1043E000B24A5D01891471F2772069F0ED2FF0E097
:1043F000ED54FD4BD7018C91848FDF5F602F8FE9E7
:1044000090E40E949114662069F0ED2FF0E0ED54E5
:10441000FD4BD6018C91848FDF5F602F8FE39EE68A
:104420000E949114CC2369F0ED2FF0E0ED54FD4B88
:10443000D5018C91848FDF5F602F8EED9DE50E940A
:1044400091149394CFCF812FDF91CF911F910F9132
:10445000FF90EF90DF90CF90BF90AF909F908F90A4
:104460007F906F900C94FB206EE087E492E40E94B2
:10447000DC1C6EE083E692E40E94DC1C6EE08FE7B9
:1044800092E40E94DC1C6EE085E592E40E94DC1C54
:104490006EE081E792E40E94DC1C6EE08DE892E41D
:1044A0000E94DC1C64E088E392E40E94DC1C8CE344
:1044B00092E40E94781CE6E3F2E4108A8081918104
:1044C00080648083918380819181916080839183D6
:1044D0004AE050E069E070E084E792E40E94BC3C6E
:1044E00080E280938E420C94011E8F929F92AF9235
:1044F000BF92CF92DF92EF92FF920F931F93CF93D1
:10450000DF93EDEAF0E480E691E0DF019C011D928B
:1045100021503040E1F7EDE4FEE682EADF011D9232
:104520008A95E9F7C0E0D8EFDF0140E096E1992EE7
:1045300056E0A12C24E1B22E88248394FE0104913C
:1045400031962491319684913196E49111960C9391
:10455000119716962C93169717968C931797189673
:10456000EC931897003108F04DC010E030E0909EB9
:10457000F001919EF00D1124BF0163557F4B7B012B
:10458000620F731FFB01408BF701858B842F652F12
:104590000E946E3B9A9D60019B9DD00C11240D2CB6
:1045A000000CEE08FF08813009F43FC0823009F4A6
:1045B00041C060E070E880E09927C60ED71EE81E73
:1045C000F91E1296CD92DD92ED92FC92159746302F
:1045D000C8F48C92F901EE0FFF1FEE0FFF1F909EA3
:1045E0009001919E300D1124E20FF31FE355FF4B14
:1045F00012960D911D912D913C9115970083118379
:10460000228333834F5F24961996423109F096CF67
:10461000DF91CF911F910F91FF90EF90DF90CF909E
:10462000BF90AF909F908F90089560E070E081E020
:104630009927C3CF60E070E881E09927BECFE62FCD
:10464000E69527E0AC01249FC001259F900D112421
:104650008D549D4BE80FF92FF11DE55AFF4F8081D6
:1046600060FD82958F700895CF92DF92EF92FF9256
:104670009C01892F992782958F7066E1689FA00120
:10468000699F500D1124FA01E355FF4B948984E092
:10469000989FF0011124E40FF51FE355FF4BC080F4
:1046A000D180E280F38080E090E0C114D104E10485
:1046B000F10449F1C9019F70B701A601480F591FC4
:1046C000611D711D6BBFFA01A791AC01569547950D
:1046D0005695479570E060E0505F6F4F7F4F4C0DEF
:1046E0005D1D6E1D7F1D6BBFFA01479150E0880F65
:1046F000991F8670992702C0559547958A95E2F7CC
:104700008A2F942F9370FF90EF90DF90CF900895B1
:104710008091015E8823E1F30E944F1490ED980F81
:104720009A3030F09FE9980F963020F499EA980F6C
:10473000892F08959FEB980F963010F499ECF7CFDE
:10474000803231F390E0F4CF8A3310F0875508952A
:1047500080530895F894EFEEFDE5108A118A128ACD
:1047600078940895F8949091015E9031B1F0E091C1
:10477000005EF0E0E151F24A80838091005E8F5F3D
:104780008093005E8091005E803110F01092005E98
:104790008091015E8F5F8093015E7894089580918F
:1047A000240886FFFCCF08951F920F920FB60F9238
:1047B00011240BB60F928F93EF93FF93E091005E5D
:1047C000F0E080912008E151F24A80838091005E00
:1047D0008F5F8093005E8091005E8F708093005E9B
:1047E0008091015E8F3028F48091015E8F5F80930D
:1047F000015EFF91EF918F910F900BBE0F900FBE56
:104800000F901F9018950F931F93CF93DF93EC0198
:104810008C01FE0101900020E9F73197EC1BFD0BA4
:10482000C8018C1B9D0B8E179F0728F0DF91CF913D
:104830001F910F910895F80181918F010E946D14CD
:10484000E8CF813408F0875F8F70089547E0489F74
:104850009001499F300D11242D543D4BBC016C5FDC
:104860007F4F8617970710F080E0089550E040E0F2
:10487000FA01E55AFF4FE20FF31FE081E11109C091
:104880004F5F5F4F4730510599F70196295F3F4FC2
:10489000E8CF81E0089597E0899FB001112430E0CE
:1048A00020E0A901460F571FFA01E753F24A425F81
:1048B0005C4BDA019C9190832F5F3F4F273031058D
:1048C00081F7089527E0829FC001112430E020E0A5
:1048D000A901480F591FFA01E753F24A425F5C4BA6
:1048E0006081FA014081641307C02F5F3F4F27307A
:1048F000310571F781E0089580E00895FB016AE0D9
:104900000E946E3B905D9283811107C080E281839B
:1049100080E28083838314820895805DF8CF382FEE
:10492000FB016AE00E946E3B282F905D92838A30E3
:1049300070F0832F64E60E946E3B805D8083822F3F
:104940006AE00E946E3B905D9183138208954083DC
:104950008111F5CF4183F9CFCF93DF93EC01FB01B8
:104960006AE070E00E94883B9B01805D83836A302F
:10497000710570F0CE0164E670E00E94883B605DD6
:104980006083C9016AE070E00E94883B805D04C0DA
:1049900080E38083672BA9F782838EE2818386E59B
:1049A00084831582DF91CF91089581E08093000682
:1049B00024E090E080E031E030930A0640910D065B
:1049C00040FFFCCF4091100650911106840F951FB7
:1049D000215091F796958795969587956AE070E0B6
:1049E0000E94883B059710F06F5F7F4F1092000682
:1049F000CB010895262F30E0082E000C990BB90149
:104A00000E949C3B820F931FB9010E949C3B08951A
:104A1000E62FE69527E0829FC00111248D549D4B1F
:104A2000E80FF92FF11DE55AFF4F808160FD829557
:104A30008F70089527E0289FD001299FB00D112481
:104A400030E020E0F901EA0FFB1FE25FFC4B9081B0
:104A5000492F4F70FB01408392959F7091832F5F88
:104A60003F4F6E5F7F4F2730310561F708958F927A
:104A70009F92BF92CF92DF92EF92FF920F931F937C
:104A8000CF93DF93CDB7DEB76897CDBFDEBFD42E0F
:104A90008E010F5F1F4FAE01435F5F4F780120E231
:104AA000D7012D937D011B961C921B974A175B071C
:104AB000B9F7382F4C0120E072E0CC24C39483E096
:104AC000B82E882D831B8617D8F4D401ED914D01A3
:104AD000822F90E0E7FD54C0E03618F4E03488F10E
:104AE000E054800F911FDC01EC93F4018081982F3A
:104AF0009D7F9C3219F08A3309F040C02C3008F3B6
:104B000085E020E04D2D682FD8018D918D010E9408
:104B10007E194D2D682FF80183850E94C6190E1548
:104B20001F0579F76896CDBFDEBFDF91CF911F914A
:104B30000F91FF90EF90DF90CF90BF909F908F905C
:104B40000895E03238F0EA3349F4840F951FDC0110
:104B50007C9314C0F0E0EB57FC4FE491EE3251F03F
:104B6000EA3B99F3EC3209F0BCCF840F951FFC01AE
:104B7000B08204C0840F951FFC01C0822F5FBECF9E
:104B8000EAE3AFCF6F927F928F929F92AF92BF92E4
:104B9000CF92DF92EF92FF920F931F93CF93DF9309
:104BA000CDB7DEB7A697CDBFDEBF982E0E944B24AF
:104BB000CE0101967C015E019DE0A90EB11C67014A
:104BC00080E2F60181936F011386AE16BF06C9F726
:104BD000892D90E047E0489FF001499FF00D112496
:104BE000EC5EFC4B2081203109F050C0949EA00166
:104BF000112425E030E0622FFA01E20FF31FE25F9B
:104C0000FC4B7081711104C021503109A0F76FEF86
:104C10006F5F20E0A62FB0E037E0389FA001399FFA
:104C2000500D11244D545D4B822F022E000C990B18
:104C30008A179B07CCF0492D440F4F5FCE01499650
:104C40000E943725A696CDBFDEBFDF91CF911F9181
:104C50000F91FF90EF90DF90CF90BF90AF909F901B
:104C60008F907F906F90089509E110E00C0F1D1F49
:104C7000080F191FFD01E81BF90BE40FF51FE65A99
:104C8000FF4F8081F80180832F5FCECF8E01075EBA
:104C90001F4FB8010E941A2580907343A1E0B3E032
:104CA00083FC02C0A3E0B1E09091714392959C70A7
:104CB000309172433F70532F898D2A8D482FFAE02F
:104CC0002F9F400D1124242F4B8D4423F9F044E6EF
:104CD000421B242F41E09830D9F4E22F022E000C21
:104CE000FF0B632F70E06F5F7F4F6E177F070CF431
:104CF00057C041E0E617F70721F49DA141E0953048
:104D000018F098E02A3024F090E002C09830C9F3FF
:104D10006EA1662311F06DE26983943009F4CEC070
:104D2000983009F43FC091111BC1442311F08DE26A
:104D30008A87822F6AE00E947A3B90E3980F9B87D4
:104D400090E3920FF6EF8F9F900D11249C87AE8712
:104D5000383008F0B0C0F801E31BF10991E0838519
:104D6000853008F490E031E0350F6DE070E0E32F1E
:104D7000032E000CFF0BDB01AE1BBF0BA00FB11FFE
:104D80008C91890F90E08A3010F080E091E0EE0D78
:104D9000FF1D805D8083315051F72111E7C038C07D
:104DA00041E0B2CF413009F048C03F5F832F821B02
:104DB000F801E81BF10987FDF39591E084858530C2
:104DC00008F490E0422F220F550B6DE070E03701A0
:104DD000640E751E032F032E000C110B5801A41A2C
:104DE000B50AB7FC0CC05B01A01AB10AA60CB71C2F
:104DF000F501808D890F90E08A3010F091E080E01D
:104E00000E0D1F1D805DF8018083315019F7AE87AC
:104E1000990C939485E020E0492D682FF70181914A
:104E20007F010E947E19492D682FF70183850E941A
:104E3000C619CE14DF0479F705CF8F5F380F3A30EB
:104E400034F551E0F801E31BF10937FDF395848552
:104E5000853008F450E0832F330F990B081B190B92
:104E6000035F1F4F1816B4F0E1E0E20FEA0DFB2DCF
:104E7000F11DA083225082FECBCF12164CF6F50115
:104E8000E20FF11D27FDFA95B0832350F6CF542F82
:104E90003AE0E1CFF80131918F01350F542F3A30CC
:104EA00010F0342F51E0B701680F791F305DFB011E
:104EB00030830197D7CF90E057E055CF383008F0D6
:104EC00046C0F801E31BF109B1E08385853008F4A1
:104ED000B0E088248394850E6DE070E0882D082C66
:104EE000000C990BFB01E81BF90BE00FF11F30815F
:104EF0003B0FB0E03A3010F0B1E030E08E0D9F1D76
:104F0000305DFC0130838A948110E8CF442309F19D
:104F1000121614F48DE28A872E5F33E0822F632FFE
:104F20000E947A3B391B291BA30EB11CF501A083FB
:104F3000822F6AE00E947A3B90E3980F9B8790E370
:104F4000920FF6EF8F9F900D11249C8726CF57E08C
:104F5000BFCF822F63E00E947A3B31E0390FE3CF6D
:104F6000222309F455CF983009F452CF8A81803337
:104F700009F04ECF2336A9F441E0252F550F330B0E
:104F80002F5F3F4F59E305C08E0D9F1DFC015083DD
:104F90004F5F842F042E000C990B28173907A4F7B4
:104FA00037CF81E38A83442379F02150822F6AE04E
:104FB0000E947A3B90E3980F9B87205DF6EF8F9FCE
:104FC000200D11242C8724CF2F5FF0CFF894E8E236
:104FD000F2E411861086128613861486158678945C
:104FE00008958F708A3010F0895A0895805D089571
:104FF000CF93C82F82958F700E94F1270E946D1465
:105000008C2F8F700E94F127CF910C946D141F93F9
:10501000CF93DF9327E0289FE001299FD00D112433
:10502000CB5EDC4B16E08A9182958F700E94F1274F
:105030000E946D1488818F700E94F1270E946D1468
:10504000115088F7DF91CF911F9108950F931F930F
:10505000CF93DF938C01EC012E968A918F700E9482
:10506000F1270E946D140C171D07B9F7DF91CF913E
:105070001F910F9108950F931F93CF93DF938C018E
:10508000EC0125968A918F700E94F1270E946D1481
:105090000C171D07B9F7DF91CF911F910F9108955C
:1050A000CF93C82F892F0E94F127803311F00E94DF
:1050B0006D148C2F82958F700E94F1270E946D14C1
:1050C0008C2F0E94F127CF910C946D141F93CF93D6
:1050D000DF93D82F162FC42F82958F700E94F1274F
:1050E00020E04C2F612F0E947617182F8D2F0E94E1
:1050F000F12720E04C2F612FDF91CF911F910C946D
:105100007617EF92FF920F931F93CF93DF93E82EC2
:10511000C62FD42F0E94662868E06C0F20E04D2F28
:105120008AE30E947617C45F87E0E89E700111242D
:1051300010E000E0F701E01BF10BEC5EFC4B4D2FA3
:105140006C2F80810E9466280F5F1F4FC85F073059
:10515000110581F7DF91CF911F910F91FF90EF9093
:105160000895909132429730BCF4E0913042F0E0E3
:10517000E85DFD4B8083809130428F5F80933042A9
:1051800080913042877080933042809132428F5FAD
:105190008093324281E0089580E00895F8948091F0
:1051A00032421816BCF4E0913142F0E0E85DFD4B6C
:1051B0008081909131429F5F909331429091314232
:1051C0009770909331429091324291509093324235
:1051D000789408958FEFFCCF8091EF6E811104C019
:1051E00080913B6E8823D9F08091C35D811117C0F7
:1051F0000E94CE288F3F99F0E82FF0E0ED50FD4F50
:10520000E491E093B24281E0809325428093C35DB4
:105210008091A74290E080933C6E90933D6E0895FC
:105220001F920F920FB60F9211240BB60F922F936D
:105230003F934F935F936F937F938F939F93AF931E
:10524000BF93CF93DF93EF93FF938091C75D8F5F01
:105250008093C75D8091C75D83708093C75D8091A7
:1052600036429091374286FF0FC087E492E40E9455
:10527000361F882349F080913642909137428260F0
:1052800080933642909337428091364290913742D4
:1052900087FF0FC085E592E40E94361F882349F0FE
:1052A0008091364290913742886080933642909345
:1052B0003742809136429091374292FF19C08CE379
:1052C00092E40E94361F61E472E48CE392E40E944F
:1052D0007F1C882369F08CE392E40E94781C809103
:1052E00036429091374280618093364290933742A4
:1052F000809136428F73D9F08091BE5D9091BF5DF1
:1053000090628093BE5D9093BF5D8091BE5D9091F1
:10531000BF5D90618093BE5D9093BF5D81E080939F
:10532000EF6E80919940813011F4109299408091F4
:10533000C75D811168C080919940823049F08091A9
:105340003E6E882329F080913E6E815080933E6EA0
:105350008091A1428F5F8093A1428091A1428C33C2
:105360000CF451C0C1E0C0939B401092A1428091C7
:10537000A0428F5F8093A0428091A0428C330CF4B6
:1053800042C01092A04280919F428F5F80939F42C3
:1053900080919F4288318CF110929F428091A4426B
:1053A0008F5F8093A442D091A4426091A2428091E9
:1053B000A3420E94561A2D2FDD0F330B82171306BE
:1053C00094F4C093A4428091A3428F5F8093A34240
:1053D0008091A3428D303CF0C093A3428091A242C1
:1053E0008F5F8093A2424091A4426091A34280913A
:1053F000A2420E94331A8093AC4280919F420E9445
:105400006C1A8093AB4281E080935301FF91EF913E
:10541000DF91CF91BF91AF919F918F917F916F91CC
:105420005F914F913F912F910F900BBE0F900FBE48
:105430000F901F9018951F920F920FB60F92112484
:105440002F933F934F938F939F9381E080939A4044
:1054500080913542813089F5809108408150809358
:10546000084080910840811128C08091A842809313
:1054700008404EB18091396E90913A6E880F991F15
:1054800021E030E04F3F11F430E020E0822B932BFD
:105490008093396E90933A6E8091396E90913A6E06
:1054A000892B59F410923542109202408FEF8FB938
:1054B0009DE090936B0480936C0481E080930B0AD1
:1054C0009F918F914F913F912F910F900FBE0F9011
:1054D0001F901895CF93DF9300D000D0CDB7DEB7E3
:1054E00080919B408130D9F50E94D52480934B6EEA
:1054F00090934C6E2091A9424CE251E0BA01EAE04F
:105500002E9F6019710911249B01369527953695B8
:105510002795BA01621B730B6817790730F582E88B
:10552000898385E88A8386E88B831C826FEF80E01D
:105530000E9411172FEF40E062EECE0101960E940B
:10554000DB1781E00E94991A80E60E94E81A80E049
:105550000E94991680E00E94201710929B4024968A
:10556000CDBFDEBFDF91CF910895B901660F771FE0
:10557000FA01E61BF70BE817F90720F482E88983A4
:1055800084E8D0CF620F731FFA01E61BF70BE81710
:10559000F90720F482E8898383E8C4CF220F331F00
:1055A000220F331F421B530B4817590710F481E891
:1055B000F2CF80E8F0CF0895CF92DF92EF92FF9282
:1055C0000F931F93CF93DF938091994081118CC0EB
:1055D000D12CC2E0CC2ED4E7ED2ED4E0FD2E11E08C
:1055E0008091EE5D8230F1F58091AB409091AC40BE
:1055F0008093FE429093FF42D09297400E947F108A
:10560000FC018081809396408091FE429091FF4200
:105610002091024021110AC08C3FF1E19F0739F52A
:10562000E0920340F0920440109302400E94342321
:105630009C013695279536952795D22E7091C85D99
:105640007093B1421092C85D4091EE5D423009F412
:10565000FEC1A0F4442331F1413009F49EC11092FF
:10566000EE5D3EC08091FC429091FD42C1CF883CEE
:1056700020E19207D9F6C0920240D8CF443009F415
:10568000F6C108F4E7C1453051F72091FC42309152
:10569000FD422F5F3F4F2093FC423093FD4280FD3F
:1056A000DECF9ECF4091FC425091FD42FA013196EF
:1056B000E093FC42F093FD42682F6370623031F159
:1056C000633009F459C16130C1F0F901FF27EE0FD1
:1056D000FF1FE155FF4F45915491822FFA01099523
:1056E0008091EE5D81117CCFDF91CF911F910F9161
:1056F000FF90EF90DF90CF9008956093EE5D8093E0
:10570000EA5D9093EB5D70939E40EACFD22FD695E1
:10571000D695D695C22FC770EFEFEC0FE73078F42F
:10572000F0E0EB56F44D0C94D23BE62BCF2B9C2BA8
:10573000D42BDD2BE02BE32B2DE060E005C00E9495
:105740007F10FC016081262F2093C15DD150DF3195
:1057500008F03EC0ED2FF0E0E055F44D0C94D23B44
:10576000EE2BF22BF62BFE2B062C0A2C102C162CD3
:105770001C2C242C282C2E2C382C4D2C522C572C05
:105780005D2C632C6B2C762C742C7D2C852C8B2C17
:10579000942C992C9F2CA32CA92CAD2CB12C0E94BD
:1057A0007F10FC012081C9CF6091F9422091FA421B
:1057B00026170CF0C9CF2DE0C7CF22E062E0C4CF9E
:1057C0002CE063E0C1CF2DE06DE0BECF22E0B5CF8D
:1057D000422F83EB92E40E94C71082CF422F81ECCC
:1057E00092E4F9CF422F8FEC92E4F5CF462F61EC93
:1057F00072E483EB92E40E94D01072CF462F63EBE9
:1058000072E481EC92E40E94B6106ACF462F6FECEE
:1058100072E4EFCF462F61EC72E48FEC92E4F3CFA9
:10582000462F6FEC72E481EC92E4E5CF462F6FECEB
:1058300072E483EB92E4E7CF462F61EC72E483EBF2
:1058400092E40E94E3104CCF462F6FEC72E4F7CF46
:105850001093C85D462F70E060E0F1CF022F262F35
:1058600041EC52E463EB72E4CB010E940F1138CF9C
:105870001093C85DC73061F480910B438A3041F4C6
:105880008091C0428B3020F089508093C04228CF55
:10589000022F262F50E040E0E5CF022F262F4FECBD
:1058A00052E4E0CF462F6FEC72E4CB01CACF462F13
:1058B00063EB72E48FEC92E4C4CF1093C85D462F83
:1058C00070E060E0F7CF022F262F4FEC52E463EB3D
:1058D00072E4CA01CACF1093C85D022F262F50E090
:1058E00040E06FEC72E4C0CF1093C85D022F262F0A
:1058F0004FEC52E470E060E0ECCF462F70E060E0E7
:1059000081EC92E40E945111EBCE462F70E060E0F2
:105910008FEC92E4F7CF022F262F4FEC52E463EB8B
:1059200072E490E080E0A1CF022F262F41EC52E4F8
:10593000F6CF462F70E060E083EB92E4E3CF462F92
:105940006FEC72E4F9CF422F83EB92E40E94421194
:10595000C7CE422F81EC92E4F9CF422F8FEC92E434
:10596000F5CFC3EBD2E4C20FD11D261B4A91498368
:105970002A95E1F71882B4CE822F86958F7327FD82
:10598000805421702713B0CE480F511D87FD5A95C2
:105990004093FC425093FD42A3CE4091FC42509173
:1059A000FD424F5F5F4F4093FC425093FD42109287
:1059B000EE5D60919E409C012170332762171306B3
:1059C00009F092CE2091EA5D3091EB5D36952795F6
:1059D00036952795BC01E6E0660F771FEA95E1F75B
:1059E0006627262B372B81FF05C02093FC4230937E
:1059F000FD4276CE80910443909105438093064307
:105A00009093074380910243909103438093044312
:105A1000909305438091004390910143809302430A
:105A20009093034340930043509301432093FC42DF
:105A30003093FD42C9010E943423892B09F050CED6
:105A40000E9471118093FC429093FD4249CE0E94C6
:105A5000F91346CE2091FC423091FD422F5F3F4F1B
:105A60002093FC423093FD420E94F91339CE8823E3
:105A700051F08091FC429091FD4201968093FC424E
:105A80009093FD42ECCD1092FC421092FD42809129
:105A90003B6E882319F010939940E1CD1092EF6E80
:105AA0001093C85DC0929940DACD2091AD42022E8C
:105AB000000C330B2F5F3F4FAC01249FC001259F8B
:105AC000900D349F900D1124019708F40895EFEC88
:105AD000F7E03197F1F700C00000F6CF1F93CF93A6
:105AE000DF9383E090E00E94552DC0E4D4E018E0FD
:105AF0001E8383E090E00E94552D1D8381E090E09D
:105B0000DF91CF911F910C94552DEF92FF921F932F
:105B1000CF93DF930E946E2DC8EDDEE1FE0114915C
:105B20001123F1F03196849122968F3F29F484E677
:105B300090E00E94552DF2CF84910E9466167E015E
:105B4000F7018FEFE81AF80A8E2D8C1B811720F0D1
:105B50001150C10FD11DE2CF84910E945F16F0CF8A
:105B6000DF91CF911F91FF90EF9008952091AD426A
:105B7000022E000C330B2F5F3F4FAC01249FC0015E
:105B8000259F900D349F900D1124019708F40895DE
:105B900052E05A95F1F700C0F8CF1F920F920FB65E
:105BA0000F9211240BB60F92BF92CF92DF92EF9219
:105BB000FF920F931F932F933F934F935F936F9396
:105BC0007F938F939F93AF93BF93CF93DF93EF9385
:105BD000FF9388E080936B048FEF80936C04DFB1B8
:105BE0008FB9DD2309F487C0ED2EF12CC701019791
:105BF0008D239F21892B09F07EC0809199408230AE
:105C0000B9F110E000E08FE1B82ECC24C394D12C80
:105C1000C02FB0920204C601002E01C0880F0A9462
:105C2000EAF78093010485E090E00E94B62D8EB1E2
:105C300090E0809590958E219F21892B31F40F5F04
:105C40001F4F0530110521F7C5E080E0D69571F4AE
:105C5000CC0FCC0FCC0FC80FC83258F08FEF8FB9D4
:105C60009DE090936B0480936C0420C08F5FEECF17
:105C7000C7E0D6E910EA80919D4281111093070494
:105C80008EE591E00E94B62DD150A9F78C2F0E948D
:105C9000B128882359F081E08093354224E632E32D
:105CA0002093034030930440809302408FE180931F
:105CB00001041092994080919C4280933E6EFF9126
:105CC000EF91DF91CF91BF91AF919F918F917F9194
:105CD0006F915F914F913F912F911F910F91FF9085
:105CE000EF90DF90CF90BF900F900BBE0F900FBE44
:105CF0000F901F9018958FEF8FB99DE090936B04D4
:105D000080936C04DCCFCF92DF92EF92FF92CF931F
:105D1000DF93ADE4BEE626E036E1D7964C91D79707
:105D20004F3F61F150E0DC968C91DC9790E0D69685
:105D30006C91D697613069F5DD966C91DD97EC0139
:105D4000CC0FDD1FCC0FDD1F349FF001359FF00D10
:105D50001124CE0FDF1FC355DF4BD896CD90DD90B9
:105D6000ED90FC90DB97C882D982EA82FB82E355F2
:105D7000FF4B8E0F9F1FEC01288B658B2F5F1996B1
:105D8000223159F6DF91CF91FF90EF90DF90CF90C5
:105D90000895349FB001359F700D1124EB01C35558
:105DA000DF4BC80FD91F48894213E8CFFC01EE0F23
:105DB000FF1FEE0FFF1FE60FF71FE355FF4B10828B
:105DC000118212821382DACF1F93CF93DF93CDB764
:105DD000DEB76C97CDBFDEBF11E060E0812F0E947F
:105DE00011171F5F1730C9F78091AE428230A9F1B9
:105DF000833051F0813019F520E046E061E089E51B
:105E00000E94761782E019C020E042E061E084E55C
:105E10000E94761720E044E061E08AE50E94761750
:105E200020E046E061E089E50E94761782E00E946A
:105E3000C22581E00E94C22580E00E94C22511E0B7
:105E4000812F0E9420171F5F1730D1F76C96CDBFAE
:105E5000DEBFDF91CF911F91089520E046E061E021
:105E600081E40E947617E9E4F3E467E1829181110D
:105E700002C06150D8F76F5F89F520E045E065E02A
:105E800082E00E947E1963E0680F20E045E08CE02C
:105E90000E947E1963E0680F20E045E081E00E94E7
:105EA0007E1963E0680F20E045E08EE00E947E19D5
:105EB00063E0680F20E045E08BE00E947E1966E613
:105EC00085E00E94E31666E686E00E94E31620E085
:105ED00046E061E081E40E947617B1CFE62FF0E062
:105EE000EF5CFC4BCE010196DC0122912D932A2F11
:105EF000281B2617D4F345E00E943725E8CF2F92C0
:105F00003F924F925F926F927F928F929F92AF9249
:105F1000BF92CF92DF92EF92FF920F931F93CF9396
:105F2000DF93CDB7DEB7A397CDBFDEBF6C017A019B
:105F3000062F10E0CA0140960817190708F054C050
:105F4000041B150B6E2C40E3BE016F5F7F4F8E2D3F
:105F50000E948F248DE28C831D822FEF40E06EEB38
:105F6000CE0101960E94DB178FEF8E0D40E3BE013C
:105F70006F5F7F4F800F0E948F242FEF40E06EED08
:105F8000CE0101960E94DB17EC0CFD1CD12C4E01BA
:105F90002AE0820E911C8AE0B82E9DE2A92E24E60A
:105FA000522E30E2432E41E4742E5CE4352E60E53F
:105FB000262E8D2D90E080179107C8F0A396CDBFB7
:105FC000DEBFDF91CF911F910F91FF90EF90DF9097
:105FD000CF90BF90AF909F908F907F906F905F9089
:105FE0004F903F902F90089500E110E0ABCF8E0DC1
:105FF0009F1D27E0289FF001299FF00D1124EC5EE2
:10600000FC4B2081203169F579823A822B8288E429
:106010008C837D821E82CD2CC694C394D0FC54C048
:1060200040E2BE01615E7F4F862D8D0D0E948F2460
:106030008AE38AA31BA220E04C2D61E0CE014F969B
:106040000E94DB1720E04C2D62E2CE0101960E94F7
:10605000DB1720E04C2D6AE88CE70E947617D3947A
:10606000A8CFBE016F5E7F4F0E941A258E8D8823B8
:1060700031F1A9828D8D805D8A838EE28B83FE0152
:106080007196DE0114968385805D8D9331978E160F
:106090009F06C9F79A8989899B9D800D11249B8948
:1060A000992379F0AB86952D981B892F6B2D0E9433
:1060B0006E3B805D8C87905D9D871E86ACCF49824C
:1060C000D9CF2BE22B87F2CF20E04C2D62E9CE0115
:1060D00001960E94DB17C3CF8130A9F028F08230EF
:1060E000F9F0833031F1089588ED94E184BF909305
:1060F00068008AE990E08093260A9093270A8AE054
:1061000080930206089588ED9CE184BF9093680017
:1061100085E391E08093260A9093270A8CE0F0CFE4
:1061200088ED25E230E084BF2093680080ED91E0A7
:10613000F1CF88ED2DE230E084BF209368008BE63C
:1061400092E08093260A9093270A8DE0D9CF84EFBE
:1061500091E00E94552D81E3809360098091AD42CA
:106160000C946C3083E00E946C30E0E2F8E087E54C
:1061700094E08087918783E087838681806C868323
:1061800080E8858384E690E00C94552DCF93DF93CF
:10619000109260090E94B2308CE00E946D1489E078
:1061A00090E40E940324C2E0DEE5899182958F701D
:1061B0000E94F1270E946D14FE01319780818F703B
:1061C0000E94F1270E946D148EE6CF31D80769F73F
:1061D0008AE00E946D148FE090E40E94032484E022
:1061E0000E946D14DF91CF910C94A7300F931F93F1
:1061F000CF93DF93109260090E94B2308CE00E942E
:106200006D148AE00E946D1480E50E946D1488E58B
:106210000E946D1484E30E946D1481E30E946D144A
:106220008AE00E946D14D0E0C0E0CE010E942624D6
:106230008823E1F0CE01C031D10508F0C0960E945C
:10624000502880E20E946D1410E000E0C8018C0F1D
:106250009D1F0E94072880E20E946D140F5F1F4F50
:106260000430110599F78AE00E946D142496C03D10
:1062700043E0D407D1F681E40E946D148AE30E94C2
:106280006D1480E20E946D1483EB92E40E94262834
:1062900080E20E946D1480E20E946D1482E40E94EC
:1062A0006D148AE30E946D1480E20E946D1481ECEB
:1062B00092E40E94262880E20E946D1480E20E94EF
:1062C0006D1483E40E946D148AE30E946D1480E2D1
:1062D0000E946D148FEC92E40E9426288AE00E94AE
:1062E0006D1483E50E946D148AE30E946D1480E2B0
:1062F0000E946D14CDE0D0E001E010E020910C434D
:1063000030910D43C8010C2E02C0880F991F0A94CA
:10631000E2F782239323892B09F055C080E30E9482
:106320006D14219758F78AE00E946D148DE40E9445
:106330006D148AE30E946D1480E20E946D148DED4D
:1063400092E40E94262880E20E946D1480E20E945E
:106350006D148EE40E946D148AE30E946D1480E235
:106360000E946D148BEE92E40E94262880E20E9427
:106370006D1480E20E946D1487E40E946D148AE31C
:106380000E946D1480E20E946D14809109438F7009
:106390000E94F1270E946D14809108438F700E9423
:1063A000F1270E946D148AE00E946D148FE090E442
:1063B0000E94032484E00E946D14DF91CF911F910D
:1063C0000F910C94A73081E3AACF109260090E942C
:1063D000B2308AE00E946D148AE00E946D1484E15C
:1063E00090E40E9403248091FD420E94F82780914E
:1063F000FC420E94F8278AE00E946D1485E190E437
:106400000E9403248FEC92E40E9426288AE00E94D6
:106410006D1488E190E40E9403248091BE5D909108
:10642000BF5D892F0E94F8278091BE5D9091BF5D6E
:106430000E94F82780914642811166C08DE190E468
:106440000E9403248AE00E946D148FE290E40E946F
:10645000032487E492E40E94262886E390E40E94C5
:10646000032483E692E40E9426288EE390E40E94AF
:1064700003248FE792E40E9426288AE00E946D148C
:1064800086E490E40E94032485E592E40E94262895
:106490008DE490E40E94032481E792E40E94262880
:1064A00085E590E40E9403248DE892E40E9426286A
:1064B0008AE00E946D148DE590E40E94032481E43B
:1064C00092E40E943B2885E690E40E9403248CE33A
:1064D00092E40E943B288FE690E40E94032480917E
:1064E00037420E94F827809136420E94F8278AE0BE
:1064F0000E946D140E94CF2384EF91E00E94B62D7C
:1065000081E380936009089586E290E499CF8F92A9
:106510009F92AF92BF92CF92DF92EF92FF92CF9372
:10652000DF93C2E0812C912C540180E090E8A0E040
:10653000BB278A539748AF4FBF4F6C017D01C80CF2
:10654000D91CEA1CFB1CDFE161E0EBBEF601879180
:10655000882369F020E04C2F0E947617682FD150D5
:106560008FEFC81AD80AE80AF80AD111EECF80E2F4
:10657000880E911CA11CB11CCF5FC630B1F6DF9113
:10658000CF91FF90EF90DF90CF90BF90AF909F9012
:106590008F900895CF9388E790E00E94552DC0E03A
:1065A00080913542813019F08C2FCF91089582E38C
:1065B00090E00E94552D7299F3CF8FEF0E94CB1679
:1065C0000E9453170E94C6308FEF0E94CB160E9484
:1065D0005317C1E0E5CF2F923F924F925F926F9297
:1065E0007F928F929F92AF92BF92CF92DF92EF9263
:1065F000FF920F931F93CF93DF93CDB7DEB76C97C6
:10660000CDBFDEBF80916B4320E1829FC00111248A
:1066100020916A4322952F70822B20E032E04901BD
:10662000881A990AAC01405351094B8F5C8FD12CC9
:10663000C12CF12C2FEF31E0F901E81BF90BE98FA8
:10664000FA8F59EB452E5EE6552E0E94C0166FEF6D
:1066500080E00E9411176FEF89E00E9411176FEF21
:106660008AE00E941117F6E0FF9EC00111242FEF6F
:1066700040E061E08053904E0E94F8172FE02F1504
:10668000E8F0EF2DF0E0E95BFC4C0C94D23B573383
:106690009A33AA336B3471347B345434C0338E3321
:1066A0000434C6330135A63470359433B63309E06B
:1066B00026E042E065E080E00E9415180E94531732
:1066C00080915000897F84608093500080915000B9
:1066D0008160809350008895809150008E7F8093D8
:1066E000500080913E6E8111B7C287E00E94B128B0
:1066F0006C96CDBFDEBFDF91CF911F910F91FF90C0
:10670000EF90DF90CF90BF90AF909F908F907F9051
:106710006F905F904F903F902F90089508E026E291
:1067200044E06EE18BE2C8CF08E02CE243E067E092
:1067300081E0C2CF08E026E147E168E189E10E94FB
:1067400015188091AE420E94AA180E941D1C0E943A
:10675000E42EB4CF08E026E246E26CE08DE00E9431
:10676000151880919D420E94AA18A8CF08E026E241
:1067700046E26DE28EE20E9415188091AA42F3CFA4
:1067800008E026E246E26BE18AE196CF08E026E2E5
:1067900046E266E286E20E94151846E7642E43E46C
:1067A000742E1E8A01E02E88312C37E0A32EB12CE6
:1067B000BE016F5F7F4F822D0E947E24F301808196
:1067C00090E00A2C02C0959587950A94E2F720E0A4
:1067D00080FF26E6402F632DCE0101960E94DB1735
:1067E0002394F1E0AF1AB10820E2320E3FEFA31676
:1067F000B306F1F60F5F4E89485F4E8B51E0651A84
:106800007108083081F65ACF8114910409F447C009
:1068100081E090E1C916D1040CF480E09601215F7B
:106820003F4FE98DFA8D2E173F0708F4826008E08C
:1068300026E246E2823071F1833079F166E28130FE
:1068400051F58DE10E9415182FEF40E06CE58AECC0
:106850009FE10E94F81740E2BE016F5F7F4F882DD5
:106860000E948F242FEF40E064E8CE0101960E9441
:10687000DB178114910431F0A601682D8B8D9C8D5E
:106880000E947F2F01E0802F0E9420170F5F0930A8
:10689000D1F714CF6CE186E2D5CF6CE1D2CF08E01E
:1068A00026E246E266E2F7CF08E025E144E163E153
:1068B00082E10E94151880919C42883751F0803FF8
:1068C00021F08C3321F480E04ECF82E04CCF83E086
:1068D0004ACF81E048CF08E026E246E26BE08AE05A
:1068E000EBCE08E021E140E16FE08EE00E94151858
:1068F0008091AD4238CF2FEF40E061E688E69FE11E
:106900000E94F8170E9487320E94D524BE016F5F53
:106910007F4F0E94AC242FEF40E062EDCE01019644
:106920000E94DB1720E047E061E08AE49FE10E94DB
:10693000F81720E048E061E08EE29FE10E94F8173E
:1069400008E026E246E266E281E2B6CE20E042E0DE
:10695000410F61E08EE70E94761720E042E069E097
:1069600084EA9FE10E94F81720E043E069E087E9AC
:106970009FE10E94F81720E044E069E08AE89FE187
:106980000E94F81720E045E069E08DE79FE10E9452
:10699000F81720E046E069E080E79FE10E94F817E1
:1069A00099E0A92EB12C00E02AE0722E0430F1F417
:1069B0008091A942BE016F5F7F4F879DC001112466
:1069C0000E94AC2442E0400F20E06CE6CE0101962C
:1069D0000E94DB170F5FFFEFAF1ABF0A053031F7D8
:1069E00008E025E244E263E282E266CEF501E45685
:1069F000FD4B808140E3BE016F5F7F4F0E948F247B
:106A0000E1CF08E026E246E268E280E2E1108FE1B1
:106A10000E94151848E0E49E9001112446E1429F2F
:106A2000C001439F900D1124FC01E355FF4B5F0112
:106A300000E02E2C220C220C220C2A940F5F822DB7
:106A4000800F0E94F12720E0402F62E00E9476171D
:106A5000AE8ABF8A8CE0382E712C612C20E0402F4A
:106A6000632D8CE70E947617EE89FF8981919191C1
:106A7000A191B191EE8BFF8B892B8A2B8B2B49F146
:106A8000F501E60DF71D808929E0289FF00111240A
:106A9000E35BF149908126E6911120E037E0839F86
:106AA000C0011124402F6AE0630D885B97400E946B
:106AB000F8174FEF641A740A5CE3350E84E0681629
:106AC000710461F696E1A90EB11C083009F0B6CF49
:106AD000F5CD26E6402F6CE0630D83EC9FE1E7CF18
:106AE000812F012E000C990B069629E0289FF001BA
:106AF000299FF00D1124E35BF149818108E026E232
:106B00008F3F39F0808108E026E24BE0882311F0C6
:106B10002AE246E263E282E20E94151820E041E0A8
:106B20006AE08AE59FE10E94F81720E041E06AE808
:106B30008AE59FE10E94F8170FE181E020E042E042
:106B4000682F8BE80E9476170150C1F720E042E0E1
:106B500068E78DE70E94761720E041E068E78CE760
:106B60000E947617812F66E00E947A3B9D5F9E8B84
:106B70008795882787958F5F888FADE4AA2EAEE62C
:106B8000BA2EB2E76B2EB8EF7B2E312CF50186A919
:106B900000E0813009F006E6F5E0F31510F1F3E0CE
:106BA0002F2E230C202F422D6AE0C3010E94F817DC
:106BB000F50187A9202F422D6AE48F3F41F10E9401
:106BC000F127202F422D6AE40E947617F50184AD4B
:106BD0008F5F0E94F127202F422D62E60E947617D8
:106BE0001AC0EDEF2E2E230C20E0422D68E78CE733
:106BF0000E947617202F422D6AE8C3010E94F817E1
:106C0000F50187A98F3FC1F4202F422D6CEC8EEB4C
:106C10009FE10E94F81720E04E89688D8EE70E9460
:106C200076173394F9E0AF0EB11C27E0620E711CA9
:106C30003CE03312ABCF42CD0E94F127202F422DF2
:106C40006CEC0E947617F50184AD8F5F0E94F127EE
:106C5000202F422D64EEC2CF80913542882309F463
:106C60002FCD0E94CE28082F0E94CA32813009F40D
:106C70000FEF0E94E6274FE04F15F8F0EF2DF0E000
:106C8000EC5BF94C0C94D23B543679369036F9369D
:106C900052386F38D236AA362C38B636BA36B238B1
:106CA0007838BF383B389F36003109F4EBC2D0F456
:106CB000002341F0083009F45CC2033019F00730BA
:106CC00009F0C3CC0E94C0160E94531781E0809344
:106CD0009B400E946A2A0E94EA1B0E941D1C0E947F
:106CE000E42E06CD083109F4CAC2003231F701E0C2
:106CF00086C0003199F048F4002309F480C083E095
:106D00000830D9F68093AE42A0CC083129F0003289
:106D1000A1F61092AE4299CC81E0F4CF82E0F2CF9E
:106D2000083149F0003221F00111C7CF0EE067C0F1
:106D300010929D428ACC81E080939D4286CC08319E
:106D400029F0003289F71092AA427FCC81E080932B
:106D5000AA427BCC083139F0003209F49CC20111FF
:106D6000ACCFF12C72CC7AE0F72E6FCC083171F0F9
:106D7000003221F00111A1CF07E041C050E1C51A56
:106D8000D108D7FE62CCD12CC12C5FCCC6010F96A6
:106D9000E98DFA8D8E179F0708F057CCF0E1CF0EE2
:106DA000D11C53CC0031C9F048F40023F9F008306D
:106DB000B1F080919C4280933E6E7FCF083159F0B4
:106DC0008CE30032B1F780939C4280917143877FBE
:106DD00080937143EECF88E7F6CF80EFF4CF8FEF4B
:106DE00080939C42809171438860F2CF6EE0F62ED2
:106DF000E0CF083149F0003221F001115ECFF02ED2
:106E000024CC0E94F63021CC20E044E062E081EB0B
:106E10009FE10E94F81784E00E94201785E0E0E9D6
:106E2000F0E4DE01519601900D928A95E1F71092FF
:106E300060090E94B2300E9486148AE00E946D149C
:106E400087E790E40E9403240E94AA231092C25D67
:106E5000F12CE12C7724739494E0992E6E0121E1BA
:106E6000C20ED11C25E0622E30E3832E42E0442E78
:106E700053E0552E8091C25D823089F040F4882322
:106E8000D9F1813009F463C09092C25D93C0833020
:106E900009F4DBC08530C1F70E948614DAC037E000
:106EA0003E9D80013F9D100D11240D541D4B84E02B
:106EB000382EA5E0AA2EB12C0E948823282E2294D9
:106EC000B0EF2B220E948823F501E45AFF4FE00F18
:106ED000F11F8229808341E0A41AB1085EEFA51654
:106EE0005FEFB50649F73A94095F1F4F3110E1CFC4
:106EF00084E0E80EF11CA2C010E08091015E8823BE
:106F000059F00E944F14F601E10FF11D908189178D
:106F100011F01230B8F41F5F0E94CE288F3FA1F00D
:106F20006092C25D8091C25D853009F443C00E94C9
:106F30004F148A3021F00E94CE288F3FC1F3709207
:106F4000C25D38C010E0E8CF1430B9F6EBCF898AC3
:106F50008A8A8B8A10E000E08091015E882361F0CC
:106F60000E944F14182F80ED810F8A30B8F5F6017A
:106F7000E00FF11D10830F5F0E94CE288F3F09F4B0
:106F800042C06092C25D8091C25D833099F00C0D69
:106F90001D2D111DB12CA12CF12CE12C0C151D0562
:106FA000B1F520E1E216F10418F030E3E31AF1083C
:106FB0004092C25D8091C25D843009F05BCF8CE865
:106FC00090E40E9403240E94A7300E94C0160E94F1
:106FD000531781E080939B4083E088CB8FE9810F3A
:106FE000863028F28FEB810F863038F4F601E00FFF
:106FF000F11D80E2810F8083BECF1A3309F0BCCF30
:107000005092C25DB9CF103209F0A6CFBCCFF801C3
:1070100082918F010E94A42390E00A2C02C0880F65
:10702000991F0A94E2F7E82AF92AF4E0AF0EB11C9E
:10703000B5CF0E94CE288F3F09F081CF0E944F1418
:107040008A30B9F77CCF0E944F148091015E811184
:10705000FACF0E944F1018CF003109F416C108F47E
:107060007ECE083121F0003209F460CE26CEE12C2C
:10707000FBE0FF2EEACA003109F40AC148F40023FC
:1070800009F477C0083009F018CE7FE0F72EDDCA8A
:10709000083129F0003209F010CE02E0B0CEE6E06F
:1070A000FE2ED3CA0031B1F050F40023A9F083E0E2
:1070B000083069F08091AD420E946C30FECD0831FD
:1070C00029F00032B9F71092AD42F4CF81E08093FD
:1070D000AD42F0CF82E0FBCF6EE0F62EEBCF002387
:1070E00009F447C0003209F0E8CD10E00CE087CE8B
:1070F000003141F1B8F4002309F4D1C0083009F09F
:10710000DCCDE12F012E000CFF0BEB55FD4B8081F8
:10711000815080838091A9428F3108F496CA8EE114
:10712000808393CA083141F0003209F0C6CD115076
:1071300017FF8BCA14E089CA1F5F15300CF485CA8B
:1071400010E083CAE12F012E000CFF0BEB55FD4B25
:1071500080818F5F80838091A9428F3108F475CA46
:10716000108273CA083109F49CC0003229F0011161
:10717000A4CD88E0F82E69CA81E0E82666CA00310D
:10718000B9F138F5002309F48FC0083009F095CD26
:10719000812F012E000C990B069629E0289FF00103
:1071A000299FF00D1124E35BF1492085EDE4FEE613
:1071B00036AD321301C016AA39964E165F06C1F7D6
:1071C00039E0389FF001399FF00D1124E35BF1495C
:1071D000C7CF083141F0003209F06FCD115017FFD1
:1071E00034CA1BE032CA1F5F1C300CF0A9CF2DCA75
:1071F000812F012E000C990B069629E0289FF001A3
:10720000299FF00D1124E35BF14940855DE4A52E33
:107210005EE6B52ED501DE968C91DE9784131DC0F7
:107220008DE49EE6FC0156AD451791F0D7963C9152
:10723000D79727A932130CC02DE43EE6F90166ADBD
:10724000561301C016AA275F3F4F42165306B1F7E7
:107250000996FEE6893B9F0729F719962EE6A93B7A
:10726000B207C9F681E0F50196AD491301C086ABBE
:10727000F9E0AF0EB11C4A145B04A9F7E6C947E078
:10728000F42EE3C933E0F32EE0C925E0F22EDDC988
:1072900094E0F92EDAC9D12CC12C09E0B0CD05E07B
:1072A000AECD10E00DE0ABCDE12C10E00BE0A7CDB2
:1072B000CF93DF9381E08093AD428091AD420E94F5
:1072C0006C3080917C008E7F98ED94BF80937C0021
:1072D0008091630083FDFCCF80917C0098ED8B7FD3
:1072E00094BF80937C0080917C00816094BF8093E8
:1072F0007C00809141018111FCCF82E080934701A5
:10730000C1E0C093520181E680935001C0930A0A04
:107310001092010A8091090A8E7F8093090A86E003
:107320008093000A8091000A81608093000ADFEF59
:10733000D0930104D093060480E8809305040E9452
:107340004E16D09362048DE080936B04D0936C044E
:10735000DFB91092A000D5E0D093A40080E4809320
:10736000850689E480930806109200060E94E627AD
:1073700087E38093A1428BE38093A04210929F42C7
:107380008CE08093AB42D093A44283E08093A342ED
:1073900085E18093A2424091A4426091A3428091F2
:1073A000A2420E94331A8093AC42C0939B40C09388
:1073B000AE421092C75DC0939E4210929D4288E7F4
:1073C00080939C4284E68093A5428CE18093A64200
:1073D0008CE38093A742D093A84288E18093A9428E
:1073E000C093AA420E94D52480934B6E90934C6E1A
:1073F00080919C4280933E6E7894DF91CF91089566
:107400000E94583984E690E00E94552D0E94852DF7
:107410000E94E51880ED97E00E94552D0E94C0164D
:107420008AE00E9420170E946A2A0E94E42E0E948D
:1074300034220E94E6270E9486140E944F100E9468
:10744000752211E0C1E00EEF88E0F82EDFEF9DE03D
:10745000E92E20E8D22E80919940813009F4FCC0B9
:1074600008F46AC08230B9F78091AA42813031F4C1
:107470000E94E51888EE93E00E94552D109202407C
:107480000E94E6270E940C1A0E942D1A10930004F5
:10749000009304048AE090E00E94B62DF0926B0401
:1074A000D0936C04E0927704DFB980915000897F1B
:1074B00084608093500080915000816080935000E0
:1074C0008895809150008E7F8093500080919940E4
:1074D000823059F3D09300040E94301AD0930604EE
:1074E000D09205040E94832E82E390E00E94552DE5
:1074F000739906C00E9486140E944F100E94752244
:1075000080913542813009F4A2C0C093EF6E109291
:10751000FC421092FD421092EE5DC093C85D109245
:10752000C35DC0933B6E0E94EA1B0E94581B0E94E1
:10753000E42EC0939B4085C08091A54290E080934B
:107540009C4090939D4080919A40813021F08091A1
:10755000024081114AC08091C35D811116C00E9412
:10756000CE288F3F91F0E82FF0E0ED50FD4FE491F1
:10757000E093B242C0932542C093C35D8091A7427D
:1075800090E080933C6E90933D6E0E94DC2A809147
:107590000240813061F48091034090910440009753
:1075A00009F452C001978093034090930440809166
:1075B0000540813079F48091A64220919C40309121
:1075C0009D40820F932F911D80939C4090939D40EE
:1075D0001092054080919C4090919D40019780932E
:1075E0009C4090939D4010929A4080919C40909135
:1075F0009D40892B09F0A7CF809106408823B9F0E0
:107600002091376E3091386E80910040909101400A
:107610002817390751F00E94581B8091376E9091BE
:10762000386E809300409093014010920640809104
:107630000740882331F00E94EA1B0E941D1C109213
:1076400007400E946A2A07CF10920240B0CF82E31F
:1076500090E00E94552D54CF109202400E94E42EDB
:107660000E94EA1B0E941D1C80915000897F84604B
:1076700080935000809150008160809350008895E5
:10768000809150008E7F809350000E946A2A8091E2
:107690003E6E811109C08091714383FD05C087E072
:1076A0000E94B1281092994080913542813071F446
:1076B000109299400E94CE28833069F40E94CA3209
:1076C000811102C00E94EB320E94581B80919940A8
:1076D000813051F2C0CE0E94B128F6CF991B79E0DB
:1076E00004C0991F961708F0961B881F7A95C9F752
:1076F0008095089587FB082E062687FD819567FDF6
:1077000061950E946E3B0EF4919507FC819508955A
:10771000AA1BBB1B51E107C0AA1FBB1FA617B707B7
:1077200010F0A61BB70B881F991F5A95A9F78095D3
:107730009095BC01CD01089597FB072E16F4009497
:1077400007D077FD09D00E94883B07FC05D03EF4A6
:10775000909581959F4F0895709561957F4F0895FD
:10776000A1E21A2EAA1BBB1BFD010DC0AA1FBB1F45
:10777000EE1FFF1FA217B307E407F50720F0A21BB7
:10778000B30BE40BF50B661F771F881F991F1A9424
:1077900069F760957095809590959B01AC01BD014E
:1077A000CF010895EE0FFF1F0024001C0BBE0790B1
:1077B000F691E02D09940E94AD3CB7FF0895821B1D
:1077C000930B08950E94AD3CA59F900DB49F900D22
:1077D000A49F800D911D11240895DF93CF931F93D3
:1077E0000F939A9DF02D219FF00D8B9DF00D8A9D9A
:1077F000E02DF10D039FF00D029FE00DF11D4E9D58
:10780000E00DF11D5E9DF00D4F9DF00D7F936F9388
:10781000BF92AF925F934F93D5010E94AD3C8B0115
:10782000AC01D7010E94AD3CEB01E80FF91FD60176
:107830000E943C3C2F913F91D6010E94AD3CC60F67
:10784000D71FE81FF91FAF91BF910E943C3C2F91B9
:107850003F910E94AD3CC60FD71FE81FF91FD6010C
:107860000E94AD3CE60FF71F9801BE01CF010F91BA
:107870001F91CF91DF9108950E94AD3C460F571F95
:10788000C81FD91F08F431960895689401C0E89480
:107890008F929F92CF93DF930E94533CDF91CF91C1
:1078A0009F908F90089588249924F401E401B0E416
:1078B0009F93AA279A158B049C04ED05FE05CF051E
:1078C000D007A10798F4AD2FDC2FCF2FFE2FE92D85
:1078D000982C892E982F872F762F652F542F432F82
:1078E000322F2227B85031F7BF9127C01B2EBF91EE
:1078F000BB27220F331F441F551F661F771F881F8A
:10790000991F881C991CEE1FFF1FCC1FDD1FAA1F8B
:10791000BB1F8A149B04EC05FD05CE05DF05A007FF
:10792000B10748F08A189B08EC09FD09CE09DF0968
:10793000A00BB10B21601A94E1F62EF49401AF0173
:10794000BE01CD01000C08952A0D3B1D4C1D5D1D8F
:107950006E1D7F1D801F911F0895A29FB001B39FD0
:10796000C001A39F700D811D1124911DB29F700D48
:10797000811D1124911D0895DC0101C06D934150BA
:107980005040E0F70895F894FFCFFF0001C80001D0
:10799000010105444953500A00454F460A0050432F
:1079A0003D002046493D002054696D65723D41000F
:1079B0002054696D65723D4200434C4B5F413A0073
:1079C00020414C4D5F413A00205343525F413A0001
:1079D000434C4B5F423A0020414C4D5F423A0020FD
:1079E0005343525F423A00494E545F54563D002083
:1079F000494E545F434E543D0020544D525F533D19
:107A00000057616974696E6720666F7220646174E3
:107A1000612E2E2E0A004F4B0A00505834310000C0
:108000000106B5064E70F858985684D84C5B8C4BD8
:108010004C3B1C427070384BAE783C0670B958CE61
:108020008CA08D08849B76761908AE58FC58F3997D
:108030009E990AB5960D9E1596BD966262C6CA5067
:108040001C231908AE58FC58E21BE2371100EE5C05
:10805000981C45028CA08411008D08580CA0B5A274
:108060007B9BCBC313E3DB4B43CB3B434B535BBD0E
:10807000B25100E30E1C5016B523110CAE0E93C482
:108080008370FA70A033F0B80E6150F86550C4F0F8
:108090007C30147C3050BCE0C8CCF73008C8CC66CB
:1080A000EBE0D5884FA550F0D44FA550D43FA8F0B1
:1080B000EECBA550AEB87C58AE8CA74C3344983C60
:1080C000A883B5BC84634C6100431300A550EED473
:1080D000D3B87C588C33A3B070E0A550EED433B83D
:1080E0007C588CC378A84E703868F828EEE8B5BC88
:1080F0008860A04E70B85860434C3748ED04711C3E
:10810000EC1F0C1B919CCC9BCCA3203C560630183A
:108110006621463087662F110C1D02C8CC5C5AD0F0
:108120007038CC9704624728707C3014FCE090666D
:10813000281C70381B2E28BC30EB33B898A8E00000
:10814000A383634323387C8338FC6B383C53387CEF
:108150003B387C2338083C8C1BADBC300670FCE0FF
:1081600048711C8C7F0C238914538C2B0441B02341
:10817000F8992C4C3F305166FB610044ED040CC76C
:108180000100D50CCC0F3008999C0CCFB83C580C92
:10819000D91C6000711CEB5924305006CC4F300CB8
:1081A000B19CA6CB091E201CE2153221460100E03D
:1081B000D50CCC3F300A999C0CBBB8F10C7CD80490
:1081C000884484D83C467CA8C46100CC4B30C306AC
:1081D000203C1C6ADB78EE30BF0E66267BA606705C
:1081E00038EE4B3EB75EF0FC56468B300770999CDC
:1081F00051844E7020B8BC588CC50284983CA8E0CD
:108200006D5820091EC8CC6046F070306906787C35
:10821000660FBC6670380EBAF038BA6EB7F04670AA
:10822000B858CCA03846BC30E660C4783C1C420A42
:10823000BD8E60A0587058585870707070E0DCA007
:10824000C44484C44404B1702DD91C610030FF0EB5
:108250004EF0E020F0AE70AEF0A6DB309C3C30A7D4
:108260003C309B685A2E28704E9C103020E84E708F
:108270009C90105C1010A8883006999C3069067894
:108280007CA63C68D5060ECC1F4CA038CC432E28CB
:10829000BC30B606E00C6B90662870387C1C0A1C5B
:1082A0004E70E06228E01908AE581C58F6BDBE4476
:1082B000F64348F62BF6603D02568C33841100B12C
:1082C0000EAE8E301EC63F4CC3301AC6A36E3008A9
:1082D000EE4E702E3C86F313EE66F3EEB8AE3D0222
:1082E000D588387E7E8953065E04467056607CA62B
:1082F0004708FCA627FCA64B3CED08E606E6E6464A
:1083000046FC06E01C8ECECC474C37784C1758E024
:10831000CC8338BC3AEEE2DFCE308E1A3C7E1E4E65
:108320001CAE3A30AEAA3CBECB133CEAF358AE6E5C
:108330001C53CE3A303C46FC6E1A3A3CEA38CA2806
:10834000E044E23349A459A41B49A4E5A43C1E4ED1
:10835000BE4F58E5A4D898D83CBB2550581CDD8C9E
:108360006EB858E065BC8C1BCCA0044841B0336D9E
:10837000BCCE992CF90C8C2F3C580C6765204670AC
:10838000B85888D3C4B83C5804987C58042B492466
:10839000B8587CD804D8FCD88404D87C8498A8E049
:1083A00085BC390C048CBBB85804ED04C4E0B01A89
:1083B00030E61B1C50BCAEC1B0AE4D14DDAC492440
:1083C00065205DBC651C4C752EB85888987C580893
:1083D000983CA81D02B85884987C5804A341B0F971
:1083E0000C3330A7C8CCF91E66DB2DAA8D08F681A8
:1083F0000B1C98B10A30FD70F0B8150A46A809BAEE
:108400008BA3ABDBB3ABA39B93FBA3F3032B23C9DE
:108410001230CFA663B51230903B1D140912309173
:108420000286061D146684E37330D04330CE0663A3
:1084300065169C021D1411B41DB4D884D81B30A835
:108440000629BF30AE06AF19B4D8D91C8C2330E052
:108450001B30D02D149388309C0613841D1411B446
:1084600006D91CA6D88C7384D884E6BD1C090E04DA
:10847000DD14661BD806163066066B1E7E8C177ED2
:10848000A1140CDDAC5D1E307006C7668B307466BF
:10849000D3069B3071463C301A7E3766EB305C4623
:1084A000E80B3065DB307A4636BB30689B301D0602
:1084B000CB3B301A06CF6667B8D8485CA2E2178873
:1084C000D8E88B266637DD1430053B302D23A61CFB
:1084D000D0E51411B46E5606D91C301D1C621F065F
:1084E000970C2B301FE5140912E6161D1411B46EFB
:1084F000060404CC13081C02A65A56BC1AD91CB890
:108500003007E8BAEF6E49241C0C2DB50CE5A46EBB
:1085100006D91CA675B0E9145B6E3DA41DB48E0689
:10852000D91C1C627330CF2D1449246E3DA46EAE4D
:10853000C512AA625830C02D14CCEF8CDBE0B8B85D
:108540003044E86914061ED91CA1143020E8F89CB8
:10855000E213A83060A820045330C848C8CCA066F5
:10856000E34404048449242DA806864C2BAD7043B3
:1085700093C1B01EA114C66FCC4F6914061ED91C3E
:10858000A11409123020E84924B80E41A41DB41CDE
:10859000EAE38E56063C3040FCE0BD1C2012050785
:1085A000204924785A0E43660E7038EE477A30C060
:1085B000661BAEA3AE3CE03020E80C57302006F836
:1085C000A85666A00879B2D91CA6063C30147C30A7
:1085D0001C50BC087A3056D84C1B36448C1B048483
:1085E000D8E80C8F3020E8E09E4EA0A60E3C266610
:1085F000EEEEEEEEE6A63C266606BEEEEEEEEE06ED
:10860000AEFC2E6E0E60DE77DC101E7CFE7FFCBEA4
:10861000FE5FFCBE437E9EBE1F3CEB7E3C1A9EFC72
:108620009CBE603003FCE8D34670CEED28041413E2
:1086300008AE58FECD7DE05CE0D460D0DC6202D7AD
:10864000629362E97CE0C2E223302C1B302ED4A07E
:10865000D57C33E97CE0D414030CA01C98E217D439
:10866000A03045D57C98F6CD7D7B1C38BC44137A70
:108670003076EF76DF7617483C0AE0CC1BAA7339D8
:1086800088E60952D5883ED74DA6251CD91C302036
:10869000E81538004C73B0E22F302DE813B8957C04
:1086A000D91C7B30C30E203C0A2365202B4E203C76
:1086B000D026E806303404661708B0C606C61CD0BB
:1086C0000C1BE21722E866F13A0E30410660304B8F
:1086D00006F3302506FCE61C0A301E6A23666A375C
:1086E000FC0E66813A30CD6A2F3C3E3EA366E030F8
:1086F000610660306606A0301ADBB03C0E660401ED
:10870000AC0C0F1CE22F0E16913E70012053AED818
:108710000C27B0B13E088BC1B0B1BC492444B0A114
:108720001CF93E589DBC981C1D88FC1EBEBEDDA4D5
:108730004E70E5A4D8B0D83CBEC32550704670B08A
:1087400068301E7CA11C0441EEB83CD844D8FCA87B
:10875000D91C78D884D8F04926410CA83080A6E6E8
:108760004EF070B858CC1F0C1B66664C17168C1355
:108770006E3C588C233080464C2F8C23767676BC0A
:10878000588C2B76767676BC56EE3C56EEEE4E3016
:10879000107030FDF0AEF046F070B858E07CD80CA8
:1087A000DD2F580C2B30844D320CDF890C4C3304F8
:1087B000B170434BF8E61F26E865144C19387DBCB0
:1087C000651CC8F84666E8B858F6F62B9DBC410C07
:1087D00004B898A859248C47C1B0302EA84924C1A8
:1087E000024E28E8A89868E0FC5C0AB8AAA8E0B0A5
:1087F00030E83AF6E3E030107030FDF0E0000000C1
:108800005AEEEEFCC6E6E6C63C06BC5CEA5A505C94
:1088100030662B22E399C63AC60E3006C3A6E67A26
:108820005ABC1A30F6F63C58FC0E3C3A301C0A3C56
:108830005AB03AE07AF30438BC585C98FE9526FCAE
:1088400010D0900EEE7E93EE0C31237EDBEE7EA3F5
:10885000FE13081C78221BDCEB1465238C27787E22
:108860006881228CAF88DB780EDC901E6F080CC705
:108870004E6E56DC5050087B0C5F0C1F0CE30C1F37
:1088800008330423780E561C561750DB7E63EE7EA9
:108890004B9C78221BDCEB9443E030D066FB20E05D
:1088A000D400980278A26838BC983C28E01CAE58E6
:1088B0000813044E6E56DC90688DB8B8580C2BC95E
:1088C0008C89B68CB551884EE80CDDB641A48A4936
:1088D00024DD20792419B46A1C0A301D623F0A2B5A
:1088E000AE9C58636E1DA4DD8CC1026E601CCB383B
:1088F000BC58780ED91CE9501C622B62BEDCDBA28E
:108900000C471437D4A250DCDC8C5BBE1FDCEB8C34
:108910001BD013D0DC4C9BD47F1EBE2F5467DCDBF6
:108920008C1BD013D0DC9BBE131EBE5EDC0C135020
:10893000BEE0DCA0760C831C6247A29C622FA222C0
:10894000230AA2501CE0169CE0D2D268AED2D228F4
:108950004EA846F070E0D91C78D808D8F0AB781C47
:10896000221BDCEB6206569C622BC6DC14DBA05695
:1089700013860EDC50BEDE774277FABEE3A6426F66
:108980007E07A6FAD31EBBBE2766EBE31E0C13BE02
:10899000AE0C83A550E854670CAD2355BC410C1DAB
:1089A000024EE860E078E05CA01E0C1B9C131C22C9
:1089B0002B62BEDCDB0C83144742F21F0404D00B95
:1089C0007676130456DBD45F8C2F543F3E63BE5340
:1089D0008483B8580C2B410CFD8A4EE8203077E098
:1089E000689D2244781CEA31B60EB8AAAE3C68F8FD
:1089F000AAAE3CA838AAAE3CE8387C4AFC2878FEEF
:108A00003B09B8B8D84C578C47D8DE3EFE31B8F396
:108A10004484D8063020665746F07038566637D9F9
:108A20001CA6E853D91C230841B0CE6DB81902B872
:108A30003C5806F804A0965C1427D4B6E30EF62B37
:108A40008C63DC541F66E333D4144FA6E32E8A3ABA
:108A50005B0E0A061C2A4F0E7E8E9C0ABA60E0AEA0
:108A600056E346A38C431B66239A3A370C1F4E737A
:108A700084762B0C4B069CA206BF1BEE608DB8CEF5
:108A800008D528EEE9502E0EA0B8BCEE7EE6C6FE54
:108A90001BDC508C752A5CF65B752C552CD4DABE29
:108AA00026E37B661FD4EB46BE3F752C552CD414B1
:108AB00047BEE3D4141FA2E39CE04C437E9EBE4716
:108AC000DCD4E3DCA07E83A28C1BD013D0DCA26BB1
:108AD000552C4C752DF3BEB6AE60EE5D1E5C4C930E
:108AE000063003562FC6FB462746FBC68606A6372A
:108AF000D4BEE31ED3752CD4143FBEE3A2D414EB32
:108B0000D61B1C501CA63033A6E00D2AC6A6C6A64E
:108B1000F306F6C70BE0DC201FD4EBA0E0A28C1B11
:108B2000D013D0DCA2E0A01E7E7E43ED28D91CEE3F
:108B30002526DC10FEE0DCD0D07C70D91CB07C7027
:108B4000061C4AD36A2775B0AB3020DE7E2320494D
:108B500026E8D309CA008CB3F12E461AAEBCFA1A25
:108B60003A30E63A303CC61C3CA2BC02F6F6DE6B5C
:108B7000F6277CD90E7CAE0819BCF90EF6CF75CA63
:108B8000AE5851000E389C0A983CBEAE2838FC26E0
:108B900084E6C67C287E7E677E01CBCDC63000EEA3
:108BA000CC4371CC66250E22C8EE66A30B000000F4
:108BB00000000000E55CBB6100A3E55C8838FC6652
:108BC000E6876B1CC4E666664B095010841CEE01F8
:108BD0003041A478901C8C476A550E4DA43DA49D4D
:108BE000A48C1F7CAAB18CC1B0041D1425FEA55015
:108BF000EED44B4670B87C588CED02B070EEF0E0CD
:108C00004EE8286AB3B83C58A020BC30C1FC1CE038
:108C100000105B504B903BF3D023BD8E103C064CB4
:108C200023308006708C83AE1CE2EEEEEEFC5C50CE
:108C3000303CE6E60E9CF83C5842A65844D91C301D
:108C40002006861CB86AF3AA6A37C6E8A8B8D3F823
:108C50007E60BEB03AE006B8588C233055737C581D
:108C60004C3305BCEEE91BB8580CDFB05A3C06305B
:108C7000667E679CD0FE431CD03EFE53FE470658DE
:108C80000ECD90EE87B00EB85830505E7C067C302A
:108C900076B1B5BCEEB85CCA46A80C2BE21B1C2210
:108CA0009C5858CEBC30147C301C50BC5870305985
:108CB000E2B858E0D8A686251CC1B030E02D1404D7
:108CC0001D1030E09C58BC0E66483D3A44251C1DE2
:108CD0003C984D14987A30F6453AF6F6167A3016E6
:108CE0003C5804D89CA298A2580C9321382B4C5184
:108CF000370C33BD386520A30CB5374CC9370CB7DA
:108D00008CCD378C8F5E7B3091AEFC9C425D1CAE6F
:108D10004D32C1B0711C9DBC110C1D028C1B0CB3DB
:108D20001538838C6B4CF53B0CF53B4CC9376520F3
:108D3000838C653BD32D38DB4C41370C3381346554
:108D400020A3203C0A30836A7F3031E82D383B0C69
:108D500081356520C3B8FB0C3B8C678C1B4924060E
:108D6000A6A6B8A6A803B8F8E806A6F13B4924B819
:108D70003C0E8CA730CD8C2FD91CD532AAAEBCA806
:108D80009858889858653A4C5330AEAAAEBCA80C97
:108D9000571B301E0C0B668CF39C98D844D8581C7B
:108DA0003001AAAEBCA8C1B030D02D14A83060E804
:108DB000D53649249C98D848D858D91CBD1C090ED2
:108DC000042021386B4C778C5F0C1BBD3865209BD1
:108DD0003030E81B30305E172EE83CBEFCE8953A98
:108DE000BEFCD056E82138430C1BBD386520BBB80B
:108DF000E04936BD1C1314201538BB3020A8A8A8A4
:108E00006D7CDC100E304C66CF21B0DDAC49249C6B
:108E10009858B81CD04C1B1CD0AE7CA2813A65205F
:108E20009B3057BE5E2B2666DF03305466E3834ECD
:108E3000BEFC1CD0E81538630C276520CB4EBEFC69
:108E4000D0E81BB8E0301F43301F23301FE8E8E8AC
:108E5000DDAC4924F81C98E8B83C58880898FC6DAB
:108E60001C61001106DCD01C0EB87E584CE706F8D9
:108E7000425646BE47A6E606E6E646A39C98584CF0
:108E80002330804686DDAC4924B80E8CA76686E682
:108E900083DDAC4924B80E30C8E0C8CC3B66E32083
:108EA0001938436D00C1B020492495BC110C9C9821
:108EB000D84C3B4C1FAEBCD1A6D84E5CD070AEBCDB
:108EC000FE6D076645023040E6C8CC6D0266DB04E5
:108ED000B1703C30E866FB59364924A5BCB8D88847
:108EE000D8A84E68D91C1538734CD13E957CB35D1B
:108EF0001C8498A84936492478EEAB7C4A68251C26
:108F0000D91CB81B0CCB6520E36D7C06251CB6BBB9
:108F10001C307F6A93303A6A73302E6A53302C6A61
:108F20003378EA1FAA0A3C68EED91C21B0B30000CE
:108F30000000000049248C931C78EE4B255068B843
:108F40005884986D1CB83C06300F6A291A86D91CC3
:108F5000DDAC492478E0DCA01CF2251866301E1C2C
:108F60006ACF78581598EE8FB858F83C9C580C5F2B
:108F7000B80E95BC110C810A4C37587C7048840C93
:108F80002B88B0A11C44B8D80C23584898589C583A
:108F90004C4B1D3C4924980E1DBCB80E86813A8C62
:108FA000537C560EB858AE444D32587CA11CB8586C
:108FB0001C98BC580C5B30E61BD03B3A30E617E0FF
:108FC0009010589C583532F8E6C1B04CA066664CFB
:108FD00013061EA1143020E8E060B0303360B030DA
:108FE0003A70EEEEDADADAEEEE7CE041A4584DA407
:108FF000EDA4D8E05CF84A0EBEBE175031020E8CCC
:109000002248E30130028C043EAEC242880480BE96
:10901000202C51C0202ECC0DA241A9AA84F902C453
:1090200050020D3384537FBC3F00000004DC78778E
:1090300077A50400DC4E0DC0AD804070097E441061
:10904000226323144F8CCCC30DC912942379D33FD0
:109050000030004100E45C480640200180840B3071
:109060003417E33B03614413D323C1903331FAF443
:10907000E4D2CA44F24DD4908823743880DFCFB351
:10908000F3BC6C759792E288CFD3CE4060C1562175
:109090001E168C74E8237655D4B87088323931D5D1
:1090A000D193F0E04D472E1FB82F2C89617420C258
:1090B00040844410A0363513834E847F64D84E55C7
:1090C000E88080D274124C1BE360A307800F28CC89
:1090D0001B31841C91DC3E01FC279EC001316D8256
:1090E0000FEEFF13DFCFFBFC27D90F9E1BC43013FD
:1090F00072813CF7F73CF743182F2EE388A4033C1A
:10910000000010D544483012D070C5713003B0173C
:10911000470C3C12C470CC030D8BCF8002470C4D22
:10912000F348CCC44C7888871F871EC715335F84EB
:109130008F2341C0084013CF4688CC00253840CD4E
:109140007512080A0D21334073C4044383C700F825
:10915000B1C44CFC72FC85BFDB87C4040C232031F6
:1091600023715CC00E193400C6848914C3703CD1CD
:10917000F3CF90E150CE6192DFF120A955A34A15BB
:10918000A82A166262403C8777F8480491C33833B6
:10919000C3400431F3B0F7C9C4E4C88DBBCB34700D
:1091A00038E013130741C43C7324232378D1C43D12
:1091B000215E141F13CAC53884C4AC737C7CC8B547
:1091C0001012024080D844C84417612520B33D20C6
:1091D000C623FCECD36EC8C1EC0B5420F944001537
:1091E0004F1534551823FBF73284FC4C018B8773E1
:1091F000E1F81727FF0113C760D19278AF17C603B4
:1092000094D754508F8FF450E4E5A41F659A3D8A9B
:109210006BDFCB3C02CA23A3CA8DC94D8842132001
:10922000668633F3ACFC18FE43A28D0B11A2CA83F1
:109230004813144140001733CC0C0CB26D33847DBD
:1092400003C74F3CC48314F3303D14CA20CED191E0
:1092500010CC3F3CC03EFD2EF2C6F1EE98127337A3
:10926000D673F4480C30CDC980CB3483D88F2072AC
:10927000CA2033DEF32003C48A6D1458608219A813
:10928000C5878C047931ACCCF07340CC1EC97667AD
:10929000F2355B43440B1D38CF7ED0C162733F0A69
:1092A00001630E80B8B3007C8E3C05B0F4D203108D
:1092B000BB0030CD0058885CC574351A37C3D2ED79
:1092C000E2D03010A2633C03F10C4D0CE1E8CF304A
:1092D000FD1107723C7012948ECB9025A18C23094E
:1092E0001C480F8A036AC214130FE30300A3388BD0
:1092F0002AA04C03C431CF0C0CC02C0200DE0AE2C1
:1093000038FC494000C0001D841057195F3DC44E11
:10931000C47FC3FF5DD64BD524CE0358C8CA19629B
:1093200081D117FB420808B2338443F5FC414CCC91
:10933000125328C634B952B9CE0350C400C846F2FD
:10934000CE7FE00932713233F100402233870C8C3A
:109350002CC5C40123EF0B0725F653843401339049
:10936000CC4C04E415AFCECC013931C710733303B4
:10937000188101C831313E1E080700F2C38071FC1C
:1093800063C5C8C4AC85332246E31F3B380720833E
:10939000DC0741FC13C33F6F88F8DDCC5050D57318
:1093A000444C18C04C58F8F883CC7132C3C10C0738
:1093B0000692BD78413BC4BD8F1304B3F810FA1870
:1093C000F3274ED1C7C7C7C7EBA48C080081ABE316
:1093D0007B48B13013223AC467233F437632168864
:1093E000C0F0303F32516308408F12F357B0804BCA
:1093F000F0CC0CD3C0C4DBD8567F5D34F2430503F8
:1094000041460000020103044247000027242120B6
:109410004348000028252200444900002926230053
:109420004540000F800000981E19B0456C63AB13D7
:109430000D08B0C964F0B8C9640EB01D6088C96475
:10944000CBAD130D08B0BEF053ABB063840F0DB0BD
:1094500071643BADB0BE001D606902AAB03560D337
:10946000A5A6A6B035603102B21E18B00EBBAFB0D3
:1094700061603B930201B05EE0930F030151848869
:1094800008080176008435928C031201595A860827
:109490001301215E8E0913015184338E1301A99E9D
:1094A0008F141301715E8E0114015184AB9705096D
:1094B0001601910E008883900505023007455A94E5
:1094C000130200418A940103012E8603355A810C50
:1094D000034E68A8E828E08F141398F0E0840C038A
:1094E000410C511E900C03318A87120C0308CD5E8B
:1094F000CE0C03C15294130C034E2868A82B980C71
:10950000034EE8090299100F039586922D04B005C9
:1095100066870504715E84011207995E84011289D1
:109520005E8C0504A18A0000BD8A8513047D5684E3
:109530000E05870E0548015A9E1205140E05B550FA
:10954000B8E81102981E05B0296A96040175BCE0BE
:1095500094030106B0B162BF0306AEAEAE2BB12DCF
:10956000181E0548B0296A833F030635586B9809D1
:109570000688015A940E098823831206B0ED66BF4F
:109580001306155A833F13063558C30065A68F147A
:10959000079208B0C966930D0888CB8713098481A8
:1095A000568C020C8E0CB0156E870F0C88CB96056E
:1095B000041341743B8E01050DF9709502902D1234
:1095C00051842574BB86060FE03009999C1508610B
:1095D000004106982F31B02D62922D105184080859
:1095E000D578CB8B0301100182880325BEBEBEB0A7
:1095F0001D606666B869603102851310CC2308EDE2
:1096000004B10E94100D0F1210810E842D12B03182
:1096100066900F1413A50E0000751E982B310E0CCA
:10962000B0CD6E981413010C38EE238C03128CB558
:10963000514E70EEE8B902930803B0FA1BBEE8B3CE
:109640008910A06964EE3A460BBE3C1898F01B8E58
:109650000412F552840E12BD2A8E14120D9E9E1213
:109660009552890313015A8613295AAB4E2172ADC4
:109670004E88DB8705124E655A930F0351846B8E1B
:1096800001145184438E091351848808E17A851AA4
:109690000913555E94121113B0F9629413130081EB
:1096A0008A8E0F4552AA14134950356043AB1413E8
:1096B00049501D60B92EAD141398A0BE589BAF142D
:1096C00013495061607B981E3031E16E850E0F1496
:1096D000795A97050916BD0EBF304D18455ABF1966
:1096E0004D18A55ABF303C18E956BF303D3C1825EF
:1096F0005ABF193D3C18055A993E3C18F8AEB8E8D7
:10970000AEA8B902BF193C18BD56BF303D18195A52
:10971000BF193D18515ABF303E18C556BF193E18E3
:10972000E156001D92910518830504482394030F08
:10973000B0E57E8E070913D13E8E0F0188ED0471CE
:109740001E86060F0184BB00009D7CAB0000201C20
:10975000E2E2E283B87CD84C1F481344D83C98A876
:109760004451064DBCE27F410C8C3B8498A8448553
:1097700006880CCB53410C04840C1F08830498A862
:1097800009B8634EE6BCAEB90C004A545C6FD6CA49
:10979000767D4D453C8C92989EA4AAB2BBC2C8CCA3
:1097A0003AD1E0E7EDF3F901097C0E2B14242D32B8
:1097B000353E4763545A6B717C82881A91993245C1
:1097C00093779E28A4A620ACB94F30C8A3DCE761EC
:1097D000EC4209FC600EC01F2E52575CB265696DE9
:1097E0007177883792989EB0B9A8C1DA1582D0D621
:1097F0000EDCE8EF1A14E208F6204CFC286B2A0075
:10980000C88C2409E71892C29EA3E7274DE0489E22
:10981000ECB83C5808987CA8E04E70F8E085B5E0BC
:10982000FFA0B0BE001D6070E0FA174EA05CF6A06D
:109830006636761B26E0F61B4E2B4A6A56D4D4E0D9
:109840004A545C6F0820F66D7132454F61ECDCC004
:10985000A66B982A3A47ACCA63887C82987DAA2B6B
:10986000D67654DC1A20E80E777C0E0E999357308A
:10987000F3FC42F96052280114E237EFB9B2B2E0CA
:10988000141F1A3E155CBBD192FCED453CC8094D36
:109890002EDAB0B9A8C19E2DD677A48C716535D0CB
:1098A000E7FDBCEEC10295BE69CC886B825A23F0FD
:1098B0009D585C0EAEF0AE6E70D494CBE0A55043D4
:1098C00032EC4E70783C0602E01CEA603CEB4CA4A3
:1098D00091EE6E98AE6150AEA0FEA03E337EE000E9
:1098E0002800D58818B550B902B550B5504E70381B
:1098F000AE7828B868F8A8AEE8E0A04E6E60EEE05A
:1099000047710E834140424348700E0078464567D8
:109910006075E00017141110534C0F00A8869C725C
:109920005259911C1815121A515CCF96A94E9D766A
:10993000565A901B19161305575DD085AC4F9E984B
:10994000505B08000C0C0C00555E07770C0C0C00EB
:1099500041460E4E5155593A617E0E5E2D2B2A2FEF
:1099600042474B0052565A2062257F00373431302F
:1099700043484C4F53573D2C631D9A0D3835322EBA
:1099800044494D5054583F05643C9B243936337E3E
:10999000454A08000C0C0C00653E07870C0C0C882F
:1099A000EE61501BDA26F6EF1D64989417D44AFA3C
:1099B000EE58AE0EF09C4A5CEA271C505C0E0A4A38
:1099C000EEEEEE5C262666421FFA06E247FC4626CD
:1099D000E21FFC468C13BE70981D60580E38A60618
:1099E000DA661FFAE7461AB160F08898AE8C5385A4
:1099F00050A0B0EED33E1BBB85508C97A0B03E7BF1
:109A0000CB8550EEAB630EB07BF8615070B0EE5377
:109A1000630EB0CBB8AEF86EB7CC6F4E70B8D84C02
:109A20003FD88C27AD7062C102B8AEF86E6760CCCB
:109A30004341A4E5A8BD8C834E70B8D84CA7D88C00
:109A40003FAD70641BCEB0EE8F2BEE702BCEAE0010
:109A5000B0A8AE58711C98AEE0B0A558B0AE4E702C
:109A600078BC46063C68E078BCAE300560061972EA
:109A7000EE38A02E6EFE433E2F385E3E537EF61B20
:109A800056765CE2174E60EE0EF0386E334C810B6A
:109A9000C90ACEF0AEE0CE7EFEBBA118CC60B858AD
:109AA0004C608CA00841B0B83C58084898FCA8E02D
:109AB00046705CA0D4D4542FCE58E09CD251B5A3AC
:109AC000983C98FC58B83CD88C132E0C1B2E2EBCFE
:109AD000F375583005755830087558300758B8BCBC
:109AE000D80CA0C4D8584E30FFD8BC0E7CA0BE60A5
:109AF000F1585B657387A1C90B3F8F15B01A30A66B
:109B00007E677E777E8F1ED8BEFBA6DBE0D8A6F3ED
:109B1000E0D800A6EBE0D80000A6E3E0A95C98BC82
:109B20006D1EA95C88CBA95C08ABB83C588404E0E6
:109B3000044E70783C5A70AE38EEAE0EF0386E605F
:109B4000EE0C134EF06EAE7BD55C542B1C52F0E045
:109B50004EF0D460AE7038DCDCDCDC93D55C544B6A
:109B60003CDC5010F070F03BD4C7AE7038DCAADC9F
:109B7000DC7C94E36B300870AEE0DCA05C38521CF7
:109B8000AEEE6FAE0E7038D494BB5CF260DCE09C3D
:109B9000D4D4F2EBE048A670851458C15C4E708EA8
:109BA000783CC6B0C67F08CEAE584E3CE6BCEE78D8
:109BB0005A7AAEC39806374C098348E07806BCEE63
:109BC0005A3AAE5878E62BBC1AEEF0EEAE0C3306DD
:109BD00033AE2E6366E3AE70FABC1A3CE638EE3C58
:109BE00070662FEEF098EE41A4CC17266E78063CF6
:109BF000063C063C686E4435BEB8584898A8E0005C
:109C00004E1B4EBE5C501B2E7AD898463E5ED81C2A
:109C1000D4763654E3EEEE6BD86EEE4B2687D86ED4
:109C200026DFAED80E23D8AE2BD8AED86E9E5E5BA4
:109C30008E1E263BD8FCD86EA66E264B66CEBE1E68
:109C4000D4D4C34EAE98EE2E76767600CB2E7AD84C
:109C500098463E5ED8065E139E0ED8DCDC8E132E30
:109C600062F354CB98AED898FE1B66CEAE5C4ABF6A
:109C7000EEAE5C0EE66B3A5BC62622DE6EFA604EF6
:109C80001EE0C6C36E63424F66EAE32EFAAE4ED8BC
:109C90004E5C50EEAED8AE332E7AD898463EFA23BC
:109CA000D8465E139ED85EAE6E2E2BD8EE66D85C7C
:109CB0004E13228EF32EEED4D4D3AE98C1622EFA78
:109CC000AE5E1BB5A23ECE6EEEEE0EEE5A0EEEE688
:109CD00013BA4E9C4217AE8E4E6EDC50CE5322CE3F
:109CE000F34EEE94C963D4CABBA63BC3FEB7F6A736
:109CF0000E8E1CEE8A5C4A9766061B36E04E22CE1C
:109D00003EEEC21BAA260EC223EE2EFBDE338A6E67
:109D1000262EFB6A626B7E5BEE865A5E2A4EBAE0A6
:109D20004E709ECE68B8A606A8E07E78EE68B8A60B
:109D30007EBB4E7078FED8B8DED8E01D648CB5626C
:109D400098941FD44AC9622EFAAEDCCED86ECEF6F5
:109D50006026E63B66EE1ED44ECF66E076FA3B36D2
:109D60007E13484623B6AE932EF0BEF01E06FA8E42
:109D7000FB2EEE66DB8EB0B5604CA0FAA00EF81D8F
:109D8000620E6964EEB03D60556469620E556435DB
:109D900060696475624E5C2650E04ED88564EECEF4
:109DA000E05C4ED01050D050105090D0D050D050D9
:109DB0005CE0FAA00E8E2626065C4647D4941BCEA5
:109DC000E066D34EDA8C93DCD4239D642BDC9D6457
:109DD000D4D49D640ECE95620E9564DCD417DC95C8
:109DE00064EE4EEE93CA0A0ACAEAEA4A8C330E06B9
:109DF0000E46E04ACAEAEFE0BE6E8ED8988E4E2735
:109E0000980EE026CB5C626EA5622EFAAE045E135D
:109E1000081E1A6ECEE673CE5E7FDCD494856B2668
:109E2000DBF568A3B9685C336E66AE333A8EF32E09
:109E3000EE66539CE22B62E24F225C23AEFAAEE266
:109E40006B4E5C6A0E1C500C13A66E0E4C1B096008
:109E50008C1BBE1E1162228EF32E543FEE66D4EE92
:109E60000BEE4C2B2968AE6EDC909CFA9BDCE23347
:109E7000628ED89883268E7E9BCECECE626E0E0CDE
:109E8000396153AE7EF32E7E982BD8988EEEEEEE8F
:109E90000E6ECEEE2798AEE066CB8ED82695626E1B
:109EA0005A5E0E0C1BE1644C1F0160416AEE5C902F
:109EB000D010905010501050905050100B4E54979E
:109EC0007A103AD4E7543F148F94CF54FF9CD05C5F
:109ED0006B9050D05010D050101050905CEEE000BD
:109EE000D0501050D050101010D0D09C8B1CD0D01F
:109EF000101050D0509010DC2B5CD0D0D01010D06F
:109F0000505CDB5CD0D0D0D0501C9B1CD0D0D09CFF
:109F10006B2EFAAE8964B861500EF85EBB06BAF6D5
:109F2000330D62E6EB66EE5ADFE64FBE1EFEFE1E06
:109F3000FE1388B85E2EFAAE08DA77D164FA1B9861
:109F4000FE072E11622EFAAE3E5EBFDAABA606E623
:109F500083461BA6080E5E5A5C8A62228ED8988BB6
:109F60005CCE62AE4E4D6E422766EEE3D8A5608BA6
:109F70000160B32EFA0EAE0E26E6B35E57AEE56470
:109F80005C4EA60E6E3B08CB54F7D43E26DB738E98
:109F90007EF3982EBE333E6EEED4940BAE8EEAEA7C
:109FA000EAAE9CD086C6E35C8EEEF568A56CFAE35B
:109FB000D4BB2E9C822E8EB5680C376E8E6E2E6EA4
:109FC0001CA56CFA3B8EDBEEDB8E235EEF665E0C2F
:109FD0001BBE00B5600CCBD164496098FE356AA603
:109FE000EEDB8E29686E5C1B2E62F34226DCE08C71
:109FF000A04ED8B968EE75620EB968B03D60EB004E
:10A00000000000B0094648167616810B70C15A014F
:10A010000C10080120040114010401140120051290
:10A02000120F120D050D0F1219200C0F13140E0F25
:10A030000E0518091314050E140E150C0C10120938
:10A04000160114050F1514200F062012010E070526
:10A050001001030B090E0714121920010701090E44
:10A060001905130E0F12010D120F0D08B060303AD2
:10A0700070BC5C50100EC1B0AE307A0656A856D3F4
:10A0800049240CA08DBCF10E2170B8F0B00E4C2309
:10A09000BD701BB57069708D70B00E356069704C05
:10A0A00023B9701BB17081704670F84C1F48EB0EDD
:10A0B000B835606970AD7081700E626970A9708D7D
:10A0C00070F04E70F8280D729D585CEE615060EE95
:10A0D0006670EE38D494B34E70138CA0BEBEBEE052
:10A0E00025601B1D60A550F05CE0D4D4D4D4D460AE
:10A0F0004E7078BC26DCD4EB667038A05CE0217032
:10A10000B5701D74F0BD700EA970EE4E70EE6162F8
:10A11000842170B1700EA970356081648C27B57090
:10A120001BBD700E3560BEBEC9643160A970696028
:10A130008164A9702EFA0E0960C9644D60FE89031E
:10A1400005608C60F088B9706BB0FA33FE238888A4
:10A150005EF00E35608964B80E3560D164316005FB
:10A1600060F00EB8AE6160FADF0ECB8C1F88E08421
:10A17000E0AE88FE13485EF0B0FAA00EEBAD74E3DB
:10A180002E0E7AFE4B480C338C238488445CA60642
:10A19000E6B177468FCECE235C62EE570C0785641E
:10A1A0000EA6AE3D7A0C0D633960AD746ECE5C5A6E
:10A1B0005E26E6433ED454D3EE3D7AD84E3ECE6B77
:10A1C000AED8221ED8AEAEBEEB1E2EAE8ECE93D82B
:10A1D0003ED86EEED454B3EEBD606ED8469CEEE130
:10A1E00078EE132E62F38E42FA1BDC9B0CE389643B
:10A1F0000160A9640960D16449601E0560B05ED841
:10A2000098464D60A606E6A176B176DC6654EB5E14
:10A21000B5608C3BBEBE696431608C2B6964316073
:10A220004C87696466660075608C3F4E5C66503D85
:10A23000604C13BE0C60F0E04E6E5E546F94EFD431
:10A2400027544F14679CD09CE0DC90901090509065
:10A2500010505050905CE09094F3631C5D789C50DB
:10A260005C109CE05C5D789C50DCE05C5D785CE0C0
:10A270001C5D781CE00808AE0E2EBAFE43880C1B4D
:10A280008C13485EEE4C457B8C2BAE0ECECE4E5CD6
:10A290001050EE66F62F661B268EEED898EEEEEE88
:10A2A000CEEEF69F8EFB2EEE66DB4EEE98EE4C1B4E
:10A2B0008ECEEE8E5B2EEE98EE4C0BE6F7EEEB8C30
:10A2C00047884C1F48734463840CC38C1B842B88C1
:10A2D0001B8564436E8E00AD743B26F6278EB32E2D
:10A2E0006600B5604C5F98EE66006960696449601D
:10A2F000D8AE0E263B6EEE3BD454B726E36E4EEE40
:10A30000E178EE133E8EF32ED4CEEE549BD88E8E93
:10A310004E5C50D89C90905B8A8ABEEB1ED8AE4EA5
:10A320002ED88E1E62ABAEFAAEFA0B7E661E8E9BE8
:10A33000980C4F8C3B396023B0D898464D60F0D1D3
:10A340006449608C13F08C13BEF00B5ED8AE98AEEF
:10A350000C1F8C1F866EDAC3D8A5600C7B8964D174
:10A36000644960016005600C8739604CA0BEE04E16
:10A370005C6A560E8E0CA02300ED64FA0D63B04C9F
:10A380009F0E1E4E5C66D01D604E5010D0D0D01077
:10A39000501090109C506960F60D62E01CA09C6EFD
:10A3A000138E26F34EAEEEEEEEEEFCA0A2E0CED47F
:10A3B00054AB139C42E60D63B0221FDAEBAEA24E03
:10A3C0002E5C105CEE22270D622EA2F3A637EEEE75
:10A3D000EEFA9BAEB04A1C5090B562B0064E3055B6
:10A3E0007C067C30E04924B83CD88C1F881384D884
:10A3F0007CA8E0302D9C58A051B698DCD0CB06C08C
:10A400001000000000800000000000048080042094
:10A410000020030001080CC41431000D320003CCED
:10A420002B28900210003314900130021028400CA9
:10A430004070A2015039980332900004800000005F
:10A44000C0000580000000005002420AC035003004
:10A45000300000DC000C8A04000068CC39000000E9
:10A460001AA031C1030230B9C040000C00008C00BA
:10A470001303C680088000B32100000850C80032D2
:10A480000800088000080800040001D9200C80C8DA
:10A49000A024933920000000C38D06083068000313
:10A4A0003000F30125000840009013900343A64DAF
:10A4B0008E0C307003190000000003000000000043
:10A4C0003000030000003000C3D0000004C0004290
:10A4D00000380C20153700F7CA89886FC8CB02F303
:10A4E00033840090D00300000240D95555555505DE
:10A4F00095657116695AAAA9EAAA2AAAABEFAE0312
:10A5000054285A3FEFFCE3C38B000BEE2A1E80FC5D
:10A5100000AF02542196A9C091EB95E5286ABB05CE
:10A52000550AC467A25A0A99872352F51188FE4F2B
:10A530008D13EF6E4D0CBA3833CCCC2000002CDAE2
:10A54000555555551500155515005555154055557A
:10A550001515551510001000000000000000100037
:10A5600000401040101560D50CEBD10C448A12123B
:10A57000FFDA8C88221341418B63680C8859206272
:10A58000800C302003C0083E2CC100AFC4C0F8BC12
:10A5900007B3CE204F11138087FC110AA08A8028B0
:10A5A000B820C938808C02FEECC17FFB38FF40C266
:10A5B000BBCFE3684E4C4CBCFF4E5CA80300953902
:10A5C0002292DDDB4B2FF470010F3FFFE12040F2C0
:10A5D00004C631E2C8C8FF310AC88CCCDF8720012D
:10A5E00009C9BFF3EF0B1220131124C40889E01B23
:10A5F000484322C4008F24003E46402C26233C3F83
:10A60000800314D0E76361134F1344343619314D7E
:10A610003B442A400129924FFE51D23C70212838F8
:10A62000CCFC3E400C04506029064CDB60F74E0128
:10A630000C002554D8F36063F7F187AAC1FF8DE3BE
:10A64000224BDC7136EE03C5084A8E288C927410BA
:10A65000CD0420812BCEEF8983040040B74FB00793
:10A660002010224988B04ED24F861258EFA11D0FFC
:10A670003BC0323C3F11CCF21C6F974072FB423D15
:10A68000B51F02300004E3844B12F4760BA2788CE1
:10A69000B30948006262173B0202862D52B8FF11CF
:10A6A000E25E5D50B2C46D0A100C403040866831E5
:10A6B0002658594D241452330029410718240720E5
:10A6C0002900A48002C0C4808CFB0B9522000B786B
:10A6D0008E00AC928400A75423CFF8092044F630B2
:10A6E00043C0B5EE5E298FF0735A2323CEB4001118
:10A6F0008C3CCC0B480C4442BC90393E9320082142
:10A7000000203D460000040040000010000004044A
:10A710000001000001400000410441B915376CFC04
:10A72000D1170304C3CC500C0C330860C4CCD0CC7C
:10A73000800411230A3FC6C80080FFBF78EE8A3F1D
:10A74000034C0322CC3401304C21002330108028EC
:10A75000C33062E2500005C01088C0FCA30438C5B5
:10A760008424B34DCDE02B2F043C123028DE40383A
:10A77000647D1374C6374208403EF6030000C140B2
:10A780002194C83E312220022085006B84CEC8046B
:10A79000599D5316097D7F71D8C532E1463B8038FB
:10A7A000133040C785224E5523DD0E054F4490CC13
:10A7B0001CDDBFB88B44A074125022129130970355
:10A7C00000767FF74C17DF8445CE98F2D949140202
:10A7D000C42012513222C900048C4A3B4BFC800336
:10A7E000050B0051482B0E31EC502DF0DF38C8130B
:10A7F000ECCCD8513D300451FBC73EF37F0CD00C5C
:10A80000441348AD7056390C51844E584488A18089
:10A8100095BCF0B3D5888A3E23E6D7ABAA0A704D23
:10A82000A47E7C81BC8D8CB0AA39887309504E5BA4
:10A830000CDF98EA2DBE0AFC4DA459A4AA0A582997
:10A84000A48A41A4CC57980647662F022762130AB0
:10A85000AEFCCA7004B00A8AB0CA70E5A47CE21FDC
:10A86000F6B362BF62ABF62BF61BF67F0C5B980A61
:10A87000468D8C59A498AA58081304B00A7C060F78
:10A88000662F02EF62DBF5A8B0AA70E5A4EA987023
:10A890001CA18C98622362626E6258B06A775582FE
:10A8A00046FC708A980A29A4BD8C6ADB20B07038F7
:10A8B0009C5898700E388E8E1CB63FB6DCDCDB02DE
:10A8C0007B4AF01C6A101C02BBA666700A4EF09808
:10A8D0007CAA698C70389C98F0467078A6682E66C1
:10A8E0000DBA6670EEF0EEC34670781C10701C0A4C
:10A8F00038E039883E37FEFEFEB183980A7CAA69AB
:10A900008CFC4DA4AA58B00A4DA4AA0A70E5A47CF8
:10A9100022DDAFE078E64E30C058708370383E9349
:10A920001CEA277CEA2371841B5584C606B0666F37
:10A93000E07EEEA0FEDC58B098701CB0FC6A6F7C24
:10A94000705584DE7985AB00000000000000000037
:10A950000000000000B0702E70380E3B55849870D7
:10A960002E58AEF0E07858EE8B1598EE810A4CEF39
:10A970000C27D588671CB1182BCCC3A918AEBC30E6
:10A9800076767627D588437AFA851406DA1A300661
:10A99000098366E64670787066BCFA38D884D8F0C9
:10A9A000BA3A301C62027CA23C0E3A300A7E27EE94
:10A9B000EECBEE3C7066EEAEF0EEBC663FEEAEDC8B
:10A9C000901C3B3C2606467078A6681C02C4BD8CD1
:10A9D00009B81D02B8463C584484B0E06259A66EDE
:10A9E000E0C461A4CAD844D885A43C0AED1ACCA01E
:10A9F000D5886A66A08CE746E000000000000000F1
:10AA0000386B3823380338E338C338A338FCE00008
:10AA100038E038933873385338333893387CE03C17
:10AA2000E07CE07CE03CE086EA667038CAE086E6DE
:10AA3000667038C64B42EAEAEA22E2E61FC61BC647
:10AA4000360A1B261B62620A707C3020FCE0AAC317
:10AA50007CD80CE92F758879A085140CCD071902D4
:10AA60007CD80CD12F758841A4F80C83E6DDA9654C
:10AA7000504C1346261366E8DD8CFBE61F26E8657E
:10AA8000144C1938655026E8E55C75067858EE8751
:10AA9000CC1F41A4A1A48584CDA8884E66480B157F
:10AAA000981CEE1B0C7B810AAE668F840C731B888E
:10AAB0004E704C47CCC98F41A4F8CD84E844B044D3
:10AAC00070198C4C27B066CB95A47CAAFC61A47C41
:10AAD0000A4CA9A76550E62398ADA01D0245BC11FC
:10AAE0000C711C2DA84CAFE0390C0860BC580CA0B0
:10AAF0000498DDD83BA188B030C570CC1F4C1B79C1
:10AB0000A055C42DA87BAA0A584888F5A898AA5829
:10AB1000334E59A48D8C986ACFE0AA8A700A7C3093
:10AB200083FCE0AE1C8A700E7C3080B31DA44BCC3D
:10AB30003F4E70F84666E8467038AA0ACC57E213D2
:10AB400022E21322E2132228E04CC98259A49DA4D8
:10AB5000AA0A29A4AA5839883E5F488C337EFEFE93
:10AB6000FEE3B0E098EE4DA4E5A41C6A4F06E64E65
:10AB70007005BC95BCCE581C0A59A43988FCEE98C7
:10AB80007C1D88EE7CEE6A461746363606277676BA
:10AB900013266A698C980A84F5AA584A174A4A23E8
:10ABA000666262E6E6E6E61322CA101C0A986D8C1D
:10ABB00098E0B9844C1187AE41A444F8E633E5A887
:10ABC0004C3748655026E8DD8E30DADADAEEEEE012
:10ABD000B02BB03A707A258CF3B02BB03A707A254E
:10ABE0008CA3B02BB03A707A258C53B02BB03A704E
:10ABF0007A258C3A3A3A7CEEEEE0B0703C467CE046
:10AC000066BC1C3A3076F6E7E23FEAC3666AAF03F9
:10AC1000222222227B9C229F224F3A3A301C22275A
:10AC20004E4C7F488EA9186EBCCB3A3066AF7A7A0C
:10AC30003C1CE044448641A4CC3FC6BC584C1B4D50
:10AC4000A4E5A47C82E2DFE237E2AFE223DDAC934D
:10AC5000F68384763CAEBC9C98161C66673C0E2935
:10AC6000A48C29A54E70AAE03C0EBB59A4A3E2E730
:10AC700036C736C739883EA74C2FED1848234C3BC2
:10AC800041A44DA4DD8C4E70E0E5A4884B7D9C98DA
:10AC9000CCBF4CAF4C9BCB5C42EE2B0E4E701C4A93
:10ACA00033AA7C8E8ED33C58681598EE9B0C1FC43B
:10ACB000934C7B8CA758B8E683B85898BC30E64BC9
:10ACC000E0C81C0A1DA4A37D9C8411007EFE4B8D50
:10ACD00008063064069B8D901C0AB8E6B38A636A46
:10ACE0008686A644D190EE60810A4670CC2FB85873
:10ACF0004C83B80A38AAFC0EF8FCAAE8AE0930ABBF
:10AD0000EA0130091E04CC7F4C6F06984C8D900CE4
:10AD1000870ABD8CC102CC330A0238BC3A30A6B6D1
:10AD20003A30FCE64738AACA0C4B8A3B384AD3086B
:10AD3000EE41A43DA43DA4AA0A559CEE530C3BEA67
:10AD400049A4E5A4D6E63342EAEAEA22E2E697C657
:10AD5000EAAD3CD86A8C8346425366985846704B9D
:10AD6000C63673A2A2B3AA62620DA48308AD3C8466
:10AD7000D8064891900AD8662702331B061B04AAFE
:10AD8000464223666262E6E6E6E61322CAE641A48C
:10AD9000EDA47CC63CFAFE8D8C59A4CE7C8D8CE54E
:10ADA000A4D8840C1388D88D8C980A7596190856E7
:10ADB000A08A16CCC3468B02A6588C3B84980638D2
:10ADC0004A4B0638AACA237D900A499646BBEAEA4E
:10ADD000868638E2AAE2270DA48B462222421B6611
:10ADE00053A2A23B047D905841A470986627023379
:10ADF0001B061B08AA0DA45697E6567FE68AB0AA42
:10AE00000C1322EAEAEAE63C8D8C9825961C903CCD
:10AE10001E98EE6A21B0001CF61B101CEEEA3CEAFC
:10AE200023BE2F7B3CEAF358845C4E7050FADA9CC8
:10AE300030583A30E6575CDA22A3E5E200D0881CAD
:10AE40003A308C97E63A30C61FE663E60EBC427C89
:10AE5000A67CCA70BCA6F6F6F6A33A3A0E303C1EA3
:10AE600078AE7E3A3A306A677E8E8EFE2F4A2F4445
:10AE7000E34A97BC631C06461F4EE030DF0647C618
:10AE80003C020ABC059AA6FCCA221C70BC0E98AEF5
:10AE90007A30EA8304D88C1B8408D86A3F8E8E0CE3
:10AEA0004F4A777C8C173C019A4ACF48B09C108C53
:10AEB0009F0E3C7A7AFAFAFADAFAFA9C98FAFA9C35
:10AEC000901CAA08E0781C101C0A70383CE6359AE1
:10AED000D5883ED37C62588ACAFCCA0E4DA459A4B8
:10AEE00098EE6E6E1CE5A46E1C6A578E8E986258A2
:10AEF000E24B4A871CCE7C0ABCA34ACF4670CE7C6C
:10AF00000444E0441CCC1F4C3BF80E38AA7CEAEB0E
:10AF1000C8E247C4EAEAEAE66FC628AE4A7CE8F827
:10AF20004666E8890AC6369B4E7048D3C44CA0F8E2
:10AF300046E8CC5795A43C0AED184435BEA918DB69
:10AF400036AF335836C7369903CC1F4CA349A43DBE
:10AF5000A41DB43C3E6B980E4670110C1B19088C56
:10AF600060D91CB8492676C321067858EE319EB8C0
:10AF7000AAA81598EEA19268B806FDBCEE3BB80EE3
:10AF80000801AC1B95BCB806EEEE787CEE0CFF78A1
:10AF9000AE3CEE1C4DA459A4C1A46E1C6AA06E1C4C
:10AFA00058EE8D8C1C98EAA0AE4670855201AC0C10
:10AFB000604ECAFCAA3C7EEE1DA0EE3F706E85502E
:10AFC0000982705838EEF0982606C3E08E85506EE0
:10AFD0000801AE41A4CC2F46CA4602B8AAA8E08C0C
:10AFE0009F061CC3300B0604B898A8A63CB0FC1CF6
:10AFF0001086BC5C221B29CA30E6D3E000000000AA
:10B00000382338F338C3389338633833387CCA3C34
:10B01000B3FCCA7C933CCA7C737CCA3C537CCAFC9C
:10B02000333CCA7C13CAF01CE03CEA7C23D588225E
:10B030003803389338633833380338D338A3730070
:10B04000385B3833381B38EB38BB388B387CEA3CFC
:10B05000EB7CC2D63CF0AA0A6E701C1BFCEA7C7327
:10B060003CEA7C537CEA3C337CEAFC13EACA47F0B6
:10B07000983EAE4670E011A0EED3A5A461A47C1D5D
:10B0800088E6132E698C980A3C1C2376DCDC76E378
:10B090004E70786E682E70E638E66670E6F0E6264A
:10B0A00066A7E6AEF04EAAAE38AEF09870384AF019
:10B0B00098A9A6980A4329A44685A47E58FEC74CA1
:10B0C00013C809824E1C70786E700638EE2F30C09F
:10B0D00006A04EE0CC8795A43C0AB18C41AA2DA8CD
:10B0E000669FE68BE841A4CC2FA1A4D84A2709503B
:10B0F0001B29A4EDA47CC4483BFCCAAED851ACD8F3
:10B100008AAE06B7662F02976A833CC9AABC08308C
:10B110007A76EF3C7E45AAA3583C0A4DA4EDA49C48
:10B12000D08D8C98E041A4AAD8A1803C1BD588D8AA
:10B13000063F6660021F62607C8ACAFCD83E67D800
:10B140003CCA7CD8447EFEFE1348E6170A4ED8E07F
:10B150004E70381CCC17E20AE01CAEE6BD9E5A26A3
:10B160008F263B301D7C44D1026666FC084DA8C585
:10B170000278101C0A703988E62709503BD5883EB2
:10B180006F4DA4E5A47CE21FF6D3B06ADB11A0EEFC
:10B1900009829C101C3020F0B070660A38D88408F0
:10B1A000D8F04E70786668C4B18C0180BD9CC10235
:10B1B000CC53AE0EBC30E04DA459A4AA0A707C302A
:10B1C00021FCE0C6C2A0BB1CCCB76262627186CC17
:10B1D0008F1C23A237A2A22FA2E0A2A2A2A2A2AEFB
:10B1E000E06EE0469C5845A4AE58707C9C98E61CE6
:10B1F0003084FCE0C98C8ECE5C581E99A49EFE5B08
:10B200003E3EBBF5A891A4CDA883FE95AAFEF75CAF
:10B21000224BFC261CE2CF8D8C8B22A70422170820
:10B220008DA4300F0C2391A453F5A82691A48DA4CE
:10B23000CDA841A459A49DA4698C7C698C0C63FCA5
:10B2400061A40A4DA4DD8CF846E8C502FEFE37CEA7
:10B25000DC95A4BB5C62439CE2B790FC5DAA628370
:10B260009CE26FD0BB8DA4FEFE33FC261CE20FD007
:10B270001DA45378EEA091A478CECE68C330F0AE72
:10B2800058782366CECEEEE798AEE0F8261F66E04B
:10B29000044E6EA05CE070CCA795A40C133C52D871
:10B2A0004A431BD5883E33E6DF09503359A4E5A451
:10B2B0007CC4488AD80EB0CA70AED851ACD832AE71
:10B2C000724B06AF662F028F627BAEE3A9184EAABF
:10B2D00058AA0C41A4B0AAD80E442BE5A84C3F7242
:10B2E00098121B0ABFAE707C066550A01C4C60A66D
:10B2F000E8B00ADD8CF8E0C41BC488CC27E5A403C1
:10B30000AABC3A30F6EB3A3076EF7A76E11B488CFD
:10B31000A91A7ABBA24BAA626266700A387CA27C28
:10B3200082E2FB2222A0F62BF61BF64FEACA8DAC76
:10B3300082E25322223BF6ABF69BF68B29A43CCA51
:10B34000E0E2EBE2FF36EF36DF8C258F8DAC8DAC83
:10B350002237484C6029A429A48C173988ED1AE2B9
:10B360008B8DACA253AA101C66700A38FCE0A27C3C
:10B37000E0E22FF66051AE7660EA8DACEA76DB0350
:10B3800004781C10581CFCCAEE30BF26AED8666B81
:10B39000D8AE7070383E437E1E1C6A237C6AE74A32
:10B3A0007F1C8A8AA6B63CCA087C7E137CF03B0CC4
:10B3B000234A3CB33CD84670D8E0B083D813AEFCE7
:10B3C000EE707C1C0A3988E6CBD5883EDBFCAA0EE1
:10B3D000584DA4E5A48A1CDA7C0AFC6AB74A574691
:10B3E0001CDA707C0EB0EE730C33466E8D8C3B987D
:10B3F00008231C980A7C8B3020061CF86AF3B8E0FE
:10B400007F61626364650060060405010C1D7E0DAA
:10B410004EF05C90308C3C0EE5A41CEA5730051CC5
:10B42000426AB7C1B06B3CC1B0E02B6E30051C4224
:10B430006A9F9E301F0C23E8BE3726BE1FE8EBE054
:10B4400020DE6DBA5E270C71B049241CE5A43C8E49
:10B45000D91C7C5675B0AB3080A330C08B0616303B
:10B460003A66AB302C66A3302E66F7304006B8D86B
:10B470004C5F8C4FD8DC101EDE7E3353D8E8302072
:10B48000DE237EBE7E70E8E0163020069730600630
:10B4900073A6D844D806B03070A646A0061B4E5CF2
:10B4A00090101C30663322E3303A5B3C56363B0E3C
:10B4B00041A4C1A41C426A60FC5C021DB48E9C586D
:10B4C00006164670307F66851DCE0E1C7C66DD8FAD
:10B4D000FC0E1DB48E9C58467051B473E0200C6075
:10B4E0004C3FC8CC37486D00CC603080E666FBE04E
:10B4F00030107030FDF09C4ADC909C905C901C9069
:10B50000282828E049246E1CCCE5A66EC9A6381C64
:10B510003CEA6D591C387C0EF87C0AAE28B87C0ACF
:10B52000AEE8787C0AAEA8AE9C9868E0E6251CE6FA
:10B5300056069C58B87CD804D83CA8F6F62F468707
:10B540008CE70C23300BE08C273077E03087E0303D
:10B550001C66273054E09D580CC92289BA84B898DB
:10B56000A82B88B898A80CA78CAB307F069C98E6CF
:10B570008D2666AF652083B83CD808D87CA8D92032
:10B580007924BD2025241D0239B478FE37FED91C4C
:10B59000B81B09B8469875B031B8638C41BB41A45B
:10B5A000198C4E70D92041A41E8EE5A41CEA2B6E86
:10B5B0008DA41E46700C1B29B8E05CA078A0FE7B11
:10B5C0009E60FEDE7E5B8C4BFE301A31B8B37E602F
:10B5D000FEE0D4577822AF145762DC5058D4A099BB
:10B5E000A4130C778CC37EB77EA7C314B794A70CA3
:10B5F000931CA0301B31B878F65329B83BA08DA41A
:10B60000042BA08DA4088D141D02301C9C5899A6F3
:10B61000307F66937846977EFE2F410CBD8AAE8DB3
:10B620008C29A44670AE68633E236520E3AE99A4DE
:10B63000BE008B1E41A459A4BE1EFC1CD08D8C7E66
:10B640000723781E9ED91C5EA0BEB8E3301FE830E9
:10B6500020DE7E6F1E3E5E23E8BEE346F07068E0AB
:10B660005ED3B8580C373CD888D87CA8469C98063E
:10B67000307F667F781CEA3FDC10FED91C1B09B8BE
:10B6800061B6851CDC10FEC1B051B6C98C9C9870A7
:10B6900041A41E30F19C5899A4B09C5899A4AE7E48
:10B6A0006815BA4E705C105CD0100EB8B03C06FA4B
:10B6B000FA7C4638BCA606583C28E0E6174E7009CE
:10B6C000503344A180AA70040A4DA4EDA4D80C27DD
:10B6D00004D8330804D88D8CB00E3988E603D58899
:10B6E0003ED7AA0A704DA40CEB08EDA47CA24BAA8D
:10B6F000626266700A387CA27C82E297E2EFE277AF
:10B70000E263DDAC4BB0E60F700C4B41A44E70E829
:10B7100028DD8CB8584CA0D5885FE27FE217365FF1
:10B72000364F59A4E5A47C22D7E38DAC0BEDA47C65
:10B73000563C8D8CE5A41C4AEECE8D8CCE7C63E508
:10B74000A41C4AEECE8D8CCE7C1BA6FC586E1DB47C
:10B750001C980120C3AEBCD91C0C733A3A3006A623
:10B760003C2EEEB9BC04D5124D140912D91CB9BC3B
:10B77000CE3C061EA114B81CD0E8661EA11463A618
:10B78000EE1C1084101C421F02889C1BDCDCB6EBF4
:10B79000E6161FDCD64E94602213E2B6F30EF88C48
:10B7A00017B858B0E0EE2798022398AE4EF0E0CEDE
:10B7B00070989801207B0C3FB858B0AEBCE06E4D3D
:10B7C0009CCE0592810A4404040C4745A4E5A45983
:10B7D000A42B6E2DB46E66E66ED91C4CD9B0D9126E
:10B7E0000C23EE58EE04D80C23080408D8E0BD1C46
:10B7F00018120F0D20E000000000000000000CB93E
:10B8000062204038238038C4F800C4039D1033D42C
:10B8100010D0CC0C0011802C2E122151C04411717B
:10B820003333809043A21A1F0035802093C1477F95
:10B8300020C4A3612032E2CCA3C838491C524981FC
:10B84000304443C8C64304224B1204F1EB003038A5
:10B850008431000000A00091869B8CE3321070D0F0
:10B860002A8348F420B806B3F836E2C90F0A92805A
:10B870003D86330033E3C94D03DC50C1832303000D
:10B88000440400300C00C07C373B280C0A5359CCD0
:10B890008A6892C4BDCC0431BD4C0C0E04E2A07881
:10B8A00038E00326143003DA203E180470483C4B7D
:10B8B00040E000002920CD9C84FC92EE2E4F87C0F2
:10B8C000804CE14430D00F461263E483E0384E10E0
:10B8D00086E1330334141258D131B2348A104D400A
:10B8E00004C0A0A20894D3206A153E053D0BE132A6
:10B8F0002138FCD7913944E6109943648E7A557209
:10B90000B4EBE27EAA2FAEEF8804E9AB701248C414
:10B91000C87675C4BED2C4D03CC8E4E8E2E1121ACD
:10B920003180CB4E02C258F8F06F8E0808A57D6DAD
:10B9300041C308EA1433A4015FE083F2604382004C
:10B94000C02C50CE0743710E6E4C8FF7C40C0D0601
:10B95000211895C54C4851A37B8DCE8DD7D40C139F
:10B960008A5A851332020C836C3854C8030C2CDEBF
:10B97000D1C404F37FC49C46D74D41334CCC3C0F1B
:10B980006195D01805C2D2A0C47A84C1E3121ECD3D
:10B990004EB838910C51A57DA23EBE8C3DD2704F61
:10B9A00060813B152E2DF67C3C70BC08A456179484
:10B9B000824F240AE00A40330108CF23F240F808FE
:10B9C000BA08D92008553CE038ECA8FA0C5021C43C
:10B9D000722208C7805E0808CFE1608E388E16623A
:10B9E0000B622F880833C20F01E7A0080328232227
:10B9F0006060FE084B0087B8C3913F2759227B0047
:10BA00000400008C00444400C820CB0DC4CC8C281A
:10BA1000C404008C0C4AFA0011110088093E06404B
:10BA200088508FEFB82BA0880F0260824D3180B90B
:10BA300008E01A12CF000522EE0741338C3C00418A
:10BA4000F0F3DFD43ACAD5C843078D40F3F3004979
:10BA5000515BECD038508380486C28C91C1132806F
:10BA60008C2CCE8CC094688C8B3B003040FD0C49F4
:10BA7000520D500D40145D55373324C34902C3188D
:10BA80004A4C50D8821B6449133184331103820419
:10BA9000D0C03C09CC4B0EE0394F8EBBB33EBE0745
:10BAA00049EFF1E22100414403880F230F051024E0
:10BAB000F3F30F015540C544CD03013C13FC0C4882
:10BAC000E4EEAE11E1816ADC861EE11086D2ED2340
:10BAD0008788181116CF704444301ADC878313B856
:10BAE0004C01847421983DCDF02034C9E0868D014D
:10BAF000008580438D30C40C208103604861F4FFD1
:10BB0000000000004C71B204FCE0180143C461BCA9
:10BB100013D30422336110447C7C4CF4217B0C1F32
:10BB200042FCC4C470D7F14CCCE3313821E310306F
:10BB300081F11008040CC2DEF228DFF9611C20300C
:10BB4000D50148E23A7B1D76D411D30434F777351A
:10BB500000B1C4714C2C48F0C74F128D33C2FD0D9B
:10BB60003131A0301310B1108010200B030A302A9D
:10BB70000A3204AC608A38CC3C23C2CC4C800A32F6
:10BB8000C1141333F18E22020C2222327131E443AC
:10BB90006ACCF771203937EBFCD4DF4C312DCE1055
:10BBA00032CE880C41CC30830236DF5B91D1B8C1F4
:10BBB000E4008D3C4D0F140E4A4C2007AA71DB5156
:10BBC0001DA342A0C3FB102632B21ACA083200BC21
:10BBD0000C008F0002D0805EC834233310F30F7343
:10BBE000DB2E0DDFCFF152F7D84B123A30000FC5E4
:10BBF0003043CBC810240C3341B4E43F000E004066
:10BC0000193F0097013B01C60A430AD2057C01D2C5
:10BC100001520A19008809B409AC0D5B0D630C16BA
:10BC2000016907F7037206B20E6205730E3606ACA1
:10BC3000080B0A7B0A85010303AF02B5068600B133
:10BC40000DE403490F530F5B0EC30EBA062D085FB8
:10BC50000E690E2F08050F2C0F350173035703C013
:10BC60000C0400AC009D03B809A300E306A20B2F4F
:10BC70000AFC00F7012001290132023C02CE066CC9
:10BC800000009319050B0C030B8045628432200ED3
:10BC90000306201418052D8D0F0F1213010B80556C
:10BCA0006A8E0306201418052018032D851A09131F
:10BCB0001001C870F868385C581C0E38AA28B044C7
:10BCC0005D5C385CD8284C9B5D1CCC274C09820DF0
:10BCD000FC0E0F20120F0F0DF1FE80BD6A981209A5
:10BCE000040D0581408001620DFC04151020060C36
:10BCF000F1FEBF0705124E78BC067CC6007DC68EDD
:10BD0000130110A9D09868F8F67B0DFC0B051903F8
:10BD10000F0405D9FE009D0E809D66BF0E0E3D18D6
:10BD20000B802D4ABF0E0E4D180B805D4ABF0E0EC4
:10BD30003C180B808D4A870E050C01F9C41379C499
:10BD40000C1B06434E3005EA6DCC66A606E0980F44
:10BD5000140179C40C1B2E53468D8C9C985606F505
:10BD6000C4B94A851A09130C068889E8B08BBF0547
:10BD70001A0913C15C4E70783CC62B0E1B841E3012
:10BD8000107046F0A1144E708C60DE9C7E7E2726DB
:10BD9000D4E30A061E5C422FFAA6E30E8EE0E1C44D
:10BDA0000459A4EDA456E63F3005426AAF089C58FA
:10BDB0001C38FCAA0A7C28E04E703830081C901C05
:10BDC0000A838D150E0179C40C600B801162940FEB
:10BDD00012010B80696660B0307CDADAFC3A307CA4
:10BDE0000B00E00B00E0D05C3066603AC60E300617
:10BDF000A075227E477E59F37E19637E0D4EEDDAE3
:10BE00003CFE4E66A63A5C105C223730C6E3692ED3
:10BE1000D05C30C6D7CC2B71CC66D3550E7C1C3091
:10BE2000060E7A30EA592FA6D3CCDD0E5D1C4CDF0E
:10BE300071CC66BFE92EBF0E0E3D3C180B80714AD7
:10BE4000F80E30E82BF80E3000E6AE6150600E566A
:10BE500037300306E3AE8D080626D3E07E7E895395
:10BE600060065E46FAA056607CA647FCA62FFCA69C
:10BE7000B5A2E10A814081C866BFE6856813A36662
:10BE80003168C66687E61568D34BD05C30E613E0B0
:10BE90007CE046E098E0D91C788C2B84D8842388F9
:10BEA000D888D8F0492660A0D91C783CD888D8FC1E
:10BEB0009B81130F100B80096A0B80F96A0B802598
:10BEC0006A0B00CD9E0286C6E0BF0E0E3E180B80A8
:10BED000C54AD91C30126A5F78D88C1F881384D861
:10BEE000F06330706A63411C30186A9D7E4EF00525
:10BEF0007E78E2D3411C4CC76100D1441BC17E193E
:10BF00007EC676C3A5D00C60C6762330EE13469667
:10BF1000864686AE0E7C0A85D026E61C4E8223A677
:10BF2000A2A2A21F26E386EA02AA0AEAEAEAAACAAB
:10BF30002AE0856813E0A6062658D944E0EB5D1C8C
:10BF4000214687010C060C0312B830FF3CEEB94ABB
:10BF500087010C060F14130B80FD6600203C56066B
:10BF60009CE23BA0005D1C21463087E099050B1444
:10BF700005070B801D6681408488ED64BE58300241
:10BF800089408808AD402570BE981D608CA7FE1FB3
:10BF90000E5B0E300555703BA00EAE00D164EE89ED
:10BFA0004C690208A140257088A393100C03100B64
:10BFB00080696E9807120C030B80C162863E3C18A4
:10BFC00015C845CCB87CAA3CA845CCF5C4CEE871D0
:10BFD0001E5CE6A616E61376A6E6E6E6C6A6D4142A
:10BFE000A3E09828C488C4FD7E3E4E302C5808300B
:10BFF0004070387CE0304070387C063CA6BCF0E0F5
:10C0000059A413A63040562B3001B6166660A5D051
:10C010000CA01C4A2A704E5CAA0A7C9C4AA606F018
:10C020007C70383CA606BCF0FBAE0E7C1CAAFC0E55
:10C030003040562B3001B6167030EF06383C662380
:10C040007666471C4A2A703866F308AE0E7C1630B6
:10C050000156BF0670F038665BA6360670F038668B
:10C060001B062B1C90D0061CE076173670383C66F9
:10C070008B3001763F2BEDA45626E66630075A1327
:10C080003AC6F306E6BCE2667CE62B4E2E1CEA8539
:10C09000D04666064B66861C82A0A2A27BC666A519
:10C0A000D046A063044E70F8EECE71C8700439D04B
:10C0B00006B0BCA6700C1F08B30C60783C06B03C00
:10C0C000063C068C3BB958BC70B95A3C70E06EA077
:10C0D0005627FAA6F330030C1B6608468EAE608D19
:10C0E0000A304056A03001B616E0041308081B04BD
:10C0F000044E7038DC901010102884444E5870386C
:10C100001CFCEADCD0BEEB59A4EDA48A1CEAAB0A05
:10C11000302C6A1F48B3885E5BBE980C23AA3C1B78
:10C120007CAA581C6A3005426AF78A985E630C2B19
:10C130003C58BEC37C1C9010CB2E5F1C38FCCA7CC4
:10C14000288C6F0C0B0CA0CC23D5886A41A47B0CE7
:10C15000A0986815980EEE734C670C771C9DA47C14
:10C160000E7C0AFD1A0DFC0E010D05D9FE83051289
:10C17000140507884B8305120C031201840B80A160
:10C1800052E54C0CA0983C063C4C3B0C17060C139B
:10C19000463CA63C9C4A0EA04E2F8C7B5C628E6671
:10C1A000665C1BFAA642EB8C13BE600D544924F862
:10C1B00028AEE8B5BCFD5A064C2B48B03C06CE7CF8
:10C1C000A6FCEEB0FC061C0201D08408CEFCAA0A34
:10C1D0007CEEEDA456E6C6762697CE7C4C1F261341
:10C1E0006603047CAA0ABCC6BCEE8CC3B07CA6263F
:10C1F0005F0C4FA646BC26BC703A4BA626E6EDD097
:10C2000063FCEEE626E6EDD00C604388983CAA7C01
:10C2100058E0CE7C0698E6B07C463C70B0FC70BC22
:10C22000A63C66063CF0E09301051601130B8099CD
:10C23000568891D04E70F80E300255701BB5A2AEE4
:10C24000BCEE514C4E70783C06F8C4FE1388CEF616
:10C250001348A67C9C4AFE1348A63C583154BCEEB9
:10C260008940A808B156BF0E0E3D3E180B80A14A6A
:10C270004E75F0EE600DFC0E0F200412091605F14C
:10C28000FE8C06130F1049F0F9C40B80E6E956BD89
:10C2900056585D1CCC604C6060B03AE08D0F0F12B8
:10C2A0000D050B809D5A8215131405074433901415
:10C2B0000507480B80594200BCA8E04E0070446856
:10C2C000780605BCEE59DE785E3E683C06660401E1
:10C2D000AC0EC1B01C0C0742271D145BAE012063DD
:10C2E0000C77AEBC4D14DDAC4924E304B1BCC36E85
:10C2F0006EC9A46E085346F059A4E5A459A4046677
:10C300008E060404D91078065830301C622B30B0E9
:10C3100062275613B6D91CB8B81C101C8C3342B80F
:10C32000302DE876B63CA23C3E1E7E7E8518492420
:10C330005DBC99C844785CE291DF3084CC2766EB21
:10C34000B371CC663F785C62683DDE309366FBC8B3
:10C35000CC2FC8CC0D541C101C02784CBB426F76FD
:10C360005B6267A21C10101C021776A268C34E5CA9
:10C370006244D302FDDA3668F6F65BE2E21FF6337A
:10C3800078562268E201DAFE435CE2234830F02B63
:10C39000C1B0BD1C03011420050D101419DDAC083B
:10C3A0000170650E4E9C90CC67601B7A1F7ACB881B
:10C3B00059C8550E1CA020E2F9CFD91C7858492441
:10C3C000300501ECC27012C38700233BB313BB0DD1
:10C3D000549B8CE378068605BC95BC66866608018E
:10C3E000AC4359C85B785C42688859C851DE8CEB15
:10C3F00048C393011405070B80ED520000000000B4
:10C400009805160113883398140507843DF0B0068B
:10C410003C2606F9FBE6C622BC70067CF03DD04EF9
:10C4200070F8AE708C2F38EEB94AAEF0E048F9C41F
:10C4300046C10238467CA65849F0DDD4B0E622FC5D
:10C4400006023DD08A983C0A05CC98420C172E0A69
:10C45000F9FB4EB07C5CD070FCE090051601130B2C
:10C46000803D6A4CE57A040D7CF57A0B80694606BE
:10C470007038F61366663C1EE0D09C30583A1C3A81
:10C4800030E63A30C64FE63F5C50D0D0F19AE60E27
:10C49000BC427CA67CCA70BCA6F6F6F6E33A3A0E1D
:10C4A000303C1E78AE7E3A3A306A677E8E8EFE2F22
:10C4B0004A2F440B4A97BC430E98AE7A30EA830465
:10C4C000D88C1B8408D86A3F8E8E0C374A77BCFD07
:10C4D000E24AE748B19AE6C532308306CE3C56665A
:10C4E00037B85CE2E2E2313238FC9CA262CF1CA297
:10C4F0003C28352EE0DCA0DCF2C156A00EAE1C724A
:10C50000CD564EEB514CD1C8E653D144E0C4F57E34
:10C510007D6813BB664670385C5228A658BDE0BEE5
:10C52000EF983CA6BCBE580948EEEB86983C7038A4
:10C530000EC67066E6386E33EE773A6E5F300406EC
:10C54000983A7EB75826371568A30DFC0E0F2013B6
:10C5500015030820010C0DF1FE266F29E60948EEAF
:10C56000DB33D1C8E62B4670F828B8EE4670CEF023
:10C57000F1688E1C527C706944E86E754CA8987006
:10C5800038F6274E70AB98267038463C05688D709B
:10C59000CE0EDC52BC702626694468454098803D2A
:10C5A0006A84050B800172840C0612038443930194
:10C5B0000C0612038801C8E6B5A2DC908C133E6815
:10C5C000BDD00881F08CA1C34E70780666263DC2AE
:10C5D0005AEEAE3C700698F00DD0A6065870CEF01C
:10C5E00070088C6366700201D030FF8D8CA658985D
:10C5F0000E0DD0A65870B0662F704EF09B0C234ED7
:10C600006EF0C102847E1788B0FC580670BC9C4A4C
:10C610001CBCF004738C060C033EA5E8B07E7E2B98
:10C6200089F63E8C1B78EE55F2BDD07DF20DFC12E2
:10C63000050320140F0F200C0F0E07F1FE920803C4
:10C640001010018408B5E00CAFCEBC06B07C8C2F76
:10C65000A63C707C26E6CEFC0AEDD0AE7C0E980699
:10C66000CEBC4630FF063B3CAA8D8CB03C0698E61B
:10C6700071D8849803920803130E09884349EA830A
:10C680000512130E0904B5E00CA7B03C51D8CE3CFE
:10C690000E889826587C9C0A7C1C0AAE7098E6EDA1
:10C6A000D0B0AA7C0EEDA4AEFCAE8D8CAE7C0E7C20
:10C6B0006A93846262901C622751EC02AE8C2FFC5C
:10C6C0000E888B987C0AFC66588C9BB383051210ED
:10C6D00010014404B9E049D8987C0EFC2BEDA45914
:10C6E000A4AE7CAE8D8C01D098663758AEFCAE738C
:10C6F0004C6030FF8D8E8C061A1305120B807D4A1C
:10C700005ABC1A203C06B0303AE62366DF461AE0EF
:10C71000411CF53E30EFB616666F3001B670387CBE
:10C7200006562306B66666E09819050B1405070B36
:10C730008005427924B5BCC10208D8284E2E687005
:10C7400088C4651C0488ED0600000000000000009D
:10C7500000000000000000000000000000000000D9
:10C7600000000000000000000000000000000000C9
:10C7700000000000000000000000000000000000B9
:10C7800000000000000000000000000000000000A9
:10C790000000000000000000000000000000000099
:10C7A0000000000000000000000000000000000089
:10C7B0000000000000000000000000000000000079
:10C7C0000000000000000000000000000000000069
:10C7D0000000000000000000000000000000000059
:10C7E0000000000000000000000000000000000049
:10C7F0000000000000000000000000000000000039
:10C80000810F1418F8EECE7EFE595A15C89C58397F
:10C81000B69209040D052E009170A56CBDCC06469C
:10C82000BCA63CF0BDCC26BCF0883E4E5859F08CDE
:10C8300053C1B01C4E901A987C5875B0BAD33020B2
:10C84000E8B03000E6E6C67EE3E8B0DCD00EA11426
:10C850004924385E285DBC8001529CC22B387C661E
:10C860003B0D54663002C61306F5C44E708CB551AC
:10C87000EEE8D5CCA6A62FB5BCFD5AC1B0BD1C04B0
:10C88000091220050D101419DDAC080170B902DC85
:10C89000901BDCD0FE84480453DC501BDCD0FE042B
:10C8A00044848404040E30407030BF0638661B0890
:10C8B000634C537C66B5F7EE7CE6FCEEAE0E3CA610
:10C8C0003C263C0E0C7F7038AED86E1788D8AE2E42
:10C8D0006F8C1B6E582DD00CE7A6067038FCA60690
:10C8E0007C7026E63DD00C6F4C278C5F83CE7C6637
:10C8F00037FCEE4B84AE0E3C06704E6EF00C278C6F
:10C900006B8485D0C6A686A6A5D0469330EEA62613
:10C9100086065C424F9B880C2FB0BC16DEBCDEF353
:10C9200076E30DFC060C2014191005D9FE0DFC064B
:10C930000C200E0F1420060F150E04F1FE1C3040C3
:10C94000704C57AE0EBC06387CA6BCF00CA04E2E28
:10C95000BC30BFF0E09208030C0504884383051245
:10C960000C05048449F08808E9D48CF9FB8C7B4ED3
:10C970007001C898A658CEBC06B07CC6E698A6063C
:10C9800027C6DB0686A6467098C60658CEBCA6C645
:10C990003CAA8D8C98E63C0AEDD0987C83B07C460E
:10C9A000707C707CF0CEFC0AD9D0CE7CAA0E84EDCF
:10C9B000A4F0664BB0561C2A13886A1CF0AE7CAEFD
:10C9C0008D8C8C60A293A63040562B3001B6166633
:10C9D0002F70383C06A2A2A28CAFAEFCAE88338C7E
:10C9E00006121510A068A5E88EB05A580881F09874
:10C9F0006E46262642EA4E7078063DC3BDCC46BC44
:10CA0000F0AE0E3C0A3DD0BA3CE6A670A638EE70F9
:10CA1000EEF0DA3C66A084A63040562B3001B61604
:10CA2000661FA5D0668C27887B981205160113888F
:10CA30003B9812140507843DF0B0588891D0B00699
:10CA40003CC61306BCA606BCD870E63C4626832628
:10CA5000E698A658B0FCA61C223DD098EEDB9214B6
:10CA60000507843B920516011388DC90FE95E8C10A
:10CA70005C4E70783CC6A660E6B006978C730DFCE1
:10CA8000050E04200F0620060CF1FE66A6C686BC25
:10CA9000A6BCFAB0FC060DD07AB0FC70BCC626BCB1
:10CAA000F0AE7084448C57A67CA63CA6700488B374
:10CAB00008849B90011713070512484B85160F0D2C
:10CAC000070512448491D0E6136670063C063C06C6
:10CAD000B958BCB958063C0627883C70B00E3CA635
:10CAE000BCA670840404B07C7038EEB07038EEF0F0
:10CAF0004C33B07C70CEF0B03C66603C048C7F8CD4
:10CB00001B661326700C600CEF3C080C9B700E2DFE
:10CB1000D0B0A68BAE7C0EB0E622FC06023DD08AD9
:10CB2000AE0E3C0A05CE94100B050513844B811400
:10CB3000100B0505138889E84E7001C8FCFA1E7EAB
:10CB40007EB0FC70BCA6063C463C7080C15A941076
:10CB50000C031284438114100C03128889E8B03C42
:10CB6000A6F5C4CEF07C06F5C46EA05A233003C6E9
:10CB7000B01D60EEB94ABD1C20051212DDAC0801E3
:10CB800070ED8AA188C1B0BD1E492404CDB4734E96
:10CB90005C90D0D010309C6262BDC06B49A43DA4B3
:10CBA0008A3DA4E5A4581C22071CAA588CDF6AED14
:10CBB0001898EA6DCC3010701EA114D91C7E9EBE50
:10CBC000B8BEF37EBAFC8518F90E46F070B85CE288
:10CBD000E2E24660E21BAE4BAEBC067CA63CA63C45
:10CBE0005EE0000000000000000000000000000007
:10CBF000000000000000000000000004320605E80C
:10CC00000000000000000000000000000000000024
:10CC10000000000000000000000000000000000014
:10CC2000000054000000009001000000042AD08899
:10CC300022282280008051018045028001C05504D5
:10CC4000C02422006024110054005001400500243B
:10CC50000204100D2002C05000000C0C00E0344F04
:10CC6000C8834F8A4F3C372C8E20C13B08E16810A7
:10CC70000D204E064065F3B8144DBFF48308922290
:10CC80000159C91D744FCC78E4452FC2F1020054FC
:10CC9000D450C1D8C430FD3A06FE876130164E41EB
:10CCA0008660434BC43D898BBBD1D3BB031011516C
:10CCB000D100034035312DE212133131D5C172500C
:10CCC00031E04C0005D10444151E50455D4C762FD3
:10CCD00003005C000000194207C9C4004066021648
:10CCE000F6460522501012B4CD460A001900740011
:10CCF000318F4F40384454F37F2B4147888714E0ED
:10CD00004331410F3C4A349009941140314166301F
:10CD1000CD2823514ECA60CAC01F8FC2E72F080119
:10CD2000B60501C2C8105D07FC2210301100FB04DB
:10CD30002244448C738748E0C4073D03A3064AA4F9
:10CD400080C1084B31C1142013044B03D60F1B02C2
:10CD5000023D0CC1E724E20051086000800000524F
:10CD6000D147842000923374CDFD6405C1111104B4
:10CD70000004F04020800661761402C404640012AE
:10CD80000012EE450D0511A0803900102148410028
:10CD90005238B18C40225015F70500549C0B0060AE
:10CDA0000020409A25CE660040050002205D3EA985
:10CDB0002686E8B534D00C004033C14149C223A3D4
:10CDC0007463C71333CDEFD27188521027BAD2E300
:10CDD000C4B84EF9F3B5A78448F623C2BAA24521D8
:10CDE000A28D6CF63300004E32C884B83260301D1C
:10CDF0000100104CE98608B7203B2AE10E0019001B
:10CE00000008804278001A0A820280078F442200BC
:10CE1000215410E1417004001D65155D2275F3B8C1
:10CE2000E322C140244354689FA88F2F638F854B12
:10CE30008B3D1F4FBCA244C05C357A9F2B0896D413
:10CE4000C515724F45A1214505910921A130E24444
:10CE500029BD290000603C981F8E04884668819196
:10CE6000089282470BA9C55401110002008620A236
:10CE7000833C683D40964089240204500189800724
:10CE80003A8A500A640200E8C0A48C0800006000DE
:10CE900080C1612444020555582C00146001800EA5
:10CEA00000040F80996110440009001073CD003C0C
:10CEB0007D840900500011C8000049C01D000074A5
:10CEC00094D4CA63114113480DD4000051DC70980A
:10CED0001913000000000000000000000000000026
:10CEE0000000000000000000000000000000000042
:10CEF0000000000000000000000000000000000032
:10CF000000804A0C00404613912302090D54171D5E
:10CF100053B58F34215E94A01611043630C5D10C60
:10CF20000080938C20000802F01246CC800200148E
:10CF3000482734878189904020227082815389025A
:10CF400031057041D43D5124230060080000601079
:10CF50000215828F8403800080427218468451C477
:10CF60004820514800511110204241B420B02C00FB
:10CF7000F0514CD008550B3C00094048A4803E03BA
:10CF800052098180487F314103FC038000A0104298
:10CF90000451019D4400480420002800E0D43022C0
:10CFA00000008640040480620208117C1F0000001B
:10CFB0000088488851C41004C14B02824022380CBA
:10CFC0008838C693C014400854000003000C184071
:10CFD00081124404C000C0000454E0440030809337
:10CFE000CCCC4406F5BF5A318CBC41400484CC40C3
:10CFF0003708C25EF501D4080C00000000000040B4
:10D000001A24005D0B6E08060F380B670B5F02D702
:10D0100002E202EA02F306340407010002C102C878
:10D0200001790089016E0122011701350B010423EA
:10D03000040F0B440CE5056009FB00EE09410054A8
:10D04000006902D0007A007100610000850D0914AA
:10D050002018032D83322020050D09142D9410175C
:10D0600013C5DA810D0C010C0341E68D0C010C0394
:10D070001289E6930D0C01120C03C9CE00000000CA
:10D08000000000000000970F0404A140F944694823
:10D0900063C1B0981E7E3570DDAC6564983102586E
:10D0A000300370C158CE6152814084D54CF88C1346
:10D0B000B86ED330200C3330188C1326E6A18804C8
:10D0C000B17022D91CB8C6E86564ED8A389C4AE084
:10D0D0003E3E3E8A1E4E62EFCECAD47EC31E4EAA8C
:10D0E000E05830107030FBF0E8E0850D0914D96885
:10D0F0008E7C5E61446948BB6ED9708B85140104D7
:10D10000D968754C694843C1B008F548656498EE24
:10D11000B94A97130C0312514C04E5449B86010C49
:10D12000031295445B514CF8BC6944FEA0DC50E00E
:10D1300097130E1512514C68E08940A838A0FE1BC9
:10D140005C8A0E9E1EB1644E46D95C5C19688D7077
:10D15000CE0E5C7CEACED95C5C4AFA1F4E5BA00E18
:10D16000665C1BFAA642EBAE0E60E099040DB8BCFB
:10D17000D844D87CA8E0990D04B8BCD848AB0E8E32
:10D180008EA04E5C504E4E9C3E3ED05C4140603C7A
:10D19000E00408E0DCA046F098067038F6136666F6
:10D1A0003C7E60BCA6BCDC100EC1B0AE5C900E46EE
:10D1B000F03C70380C435C04F2277CA2E370D91C6D
:10D1C0008EB07C7075B06E8E5E4B5CA2A39CA2AFDD
:10D1D0007AD30CE361009CD2BB9CD2A0C1B0DC101E
:10D1E000FE04041B300B3C0E1CF86A1FBEE3B8495A
:10D1F000243E616A856869547008A968E60670383B
:10D200001CFC6A6A1E6A337E7E98A658B08148ED7F
:10D210004E6954BE3E0165DB000045DA00000000A7
:10D2200000006954F693E0DCA01CEE982670380EDE
:10D23000A0F2A65EEBA6728940387C323200003242
:10D240001F12EF662792B2939260981D68A6049809
:10D2500070CE1C42F0861E81487E98C6BE6066EB8A
:10D26000F613263C5E9E9870380C134E7098532629
:10D270007038A670A6F066A60626AFC670B0F0BEDF
:10D2800033E0300870A6DCD09C1E387C4A3CEE604F
:10D29000A6BE60A6067038BB8940387C4666E6A606
:10D2A000260E4B361CE2172AA6496870383E607E6F
:10D2B0001C128B1C42F0935C0A6029FEAB05140122
:10D2C00004D9CE93190104048DCE980D0C010C03E2
:10D2D00011E6B2310B0C03DD48449828E0B4320B60
:10D2E0000C03DD4848AB940B0C03DD48846B8414BD
:10D2F0000B0C03DD488823514CAD72754C46178EDC
:10D3000030020C6BE01CA01C50509C30057217665C
:10D31000884884DD6C0C0BDDAC4E30200EB8B8B8FC
:10D32000662F7EB86623D888D8E8492438D91C9C53
:10D330004A9EF9447E3570492659CA85683389402A
:10D340004EA8E0454A93000099CA08C1B04944007C
:10D35000B9620058894068F858A8B80E4EA07A60A3
:10D360006E1F8CA0A84E2828A82828E8E828E8A83E
:10D370002828E8A8E04970136BDD48A00E3CAA7C81
:10D38000C6A670663004062B301246BA9A4EA6BC6A
:10D3900001700EB01A9A70DAA5709A7C2B816CA07D
:10D3A0000E0E4924389C0AAE284A7C0E4E5C50D0A2
:10D3B00010101090504E5CD0905090DC4140AEBCAC
:10D3C0000E389C4ABC70BAA57070BC0E4E1CD010B2
:10D3D000903A5C49404E5C100E2BCE7A1A23AE7CFC
:10D3E00006B0A6705A0170BC30120EB0BA5A7A66F6
:10D3F00006237AA646FCDA3C5CAA7C0EDD48694628
:10D4000094030512120F034843850D0914051344B4
:10D410004E7D4070CD6C49503C2EFCBB8514010400
:10D420001405134E7E708140EEB5A258CD6C448435
:10D430004950704570380EB0284CD3492478AECE90
:10D440003010956078AE68CEF0AE5C4E138A0A302C
:10D450001095607858B075604E3004583A3024BC4E
:10D460004960709544A0EE1FA01B2D60B02560EEB2
:10D470003961216CC4F57C856813E061481CCAF9E8
:10D4800072E0AEBC0EA01C30120A334A2356134A77
:10D4900016E004E0DCA005688EB03E777E4970138C
:10D4A000730950EA0A4BAE3C0E1C12D1501B84ABE0
:10D4B000D8EE271CD2D3D54CB540EE4D704E1C5043
:10D4C000501C0A1BCD4290901C0AD36E816C4E0EEC
:10D4D0008D70CE4EFD50A0980EE09ED95C4D70131D
:10D4E00063D95C8A8A4B30030455701B616A8A8A4F
:10D4F0008A1ED95CA04E9C909C0A931C3C0A73A087
:10D500005C99704E5CA5700E0E60E00E695013EBD6
:10D51000D95CDE7098067C6627B00E2B6670C15809
:10D52000CED95CFE23A03E2B6E6D50234C670BD9E9
:10D530005CDEA05CFE138A0EB0FE138AAECE5E6F78
:10D540009E2146307A66FB61020404981D5C5AE114
:10D55000080698467CA6BC58E01C987038E09713E3
:10D56000783CE64EC67CC63CEE514CC4780ED1E207
:10D57000B1640E681CE260CE3C58B96C6100CCED21
:10D5800057080C7F44E544CCCFE05CB5708C171C89
:10D59000D85346F0987CB95844CECC37FE2BA03EE9
:10D5A0007E538C2B2D548B234970630460B1702201
:10D5B00008D91C495C638ECC4FE01C214CCCF55C37
:10D5C000A0CCCF6089406C9BF89CE27B4970CC1D5D
:10D5D00070CC4F89403031E8F9561CF8EA23A8385E
:10D5E0000E98BC62EBCCAFA2023C580CAF0844AE24
:10D5F000F544CC47214CE05C115C3B6046F03013B5
:10D60000716487138474348575358676363718824D
:10D61000C21283C37300230B36363636363636369F
:10D6200036134B237BFBFB6B53306E66FBF1568B43
:10D63000030F0C039170E5EE995ABB05D40D5449C4
:10D64000248142115AB95A855A0DD49170A56CA003
:10D65000F9CE73AB8C374C73195C061C62131C42F9
:10D6600062315D33D38940F81C0CFFEABF4EA82815
:10D670009B4C8FB570A88C1B281368580C2555F34C
:10D680008C178C1F883B842B4CD73032155CA08CB8
:10D690002FA6FB415E66134660315C315488E54C31
:10D6A000AB8C9F4C8F0C1F0813042D5404434C3734
:10D6B0008C370CCF08A55A044C1F481344989C4241
:10D6C0001C4258C3155C044C374666B64893367600
:10D6D000DF1C862233A24C47C62B629C86A24431B3
:10D6E0005C4CCF3154BB4C778940A838700C255521
:10D6F000987CB958B004F544987C70AEF0C8CC7BE7
:10D7000008488C2D55C8CC3BE01CF55C46F0983C95
:10D71000A02660F61348315C7C26BC588CE54D6130
:10D7200000987C26167616577038AE98F038AEF012
:10D73000986E4971F9560CA04C43C8CC60A060208B
:10D74000E0CCED57E006983C0CA03CE03C0C173CCC
:10D7500058E0302E0C1B303DE830128C1B3004E8B2
:10D76000195CD95C065E3E4C1B3E234C17E63030FC
:10D770007CB6163C761B301FE8E67EABE0A0C1B05D
:10D78000600C495CD95C6EE00C2B5E4BD43B5E13A5
:10D790001C4C135C2BE01CA05E0EC1B03E04885CE8
:10D7A000421B3EC3EAE0DCA07EBB830491704C4F79
:10D7B000D8C9705C422F3E33D8885E3EFED91C78B3
:10D7C00068786860E0EAA09C9A5E339A509C029068
:10D7D000DEDE1790D95C13D07EF3D0D0D0D0D0D07D
:10D7E000D0E0DCD08C7F0A9417904C276210135045
:10D7F00050DC0210CA683828380AAE28A046F0E08B
:10D800009401030D0C017D681B796666A65E3E5887
:10D81000C4440D54E0C170843D6404CDB47B758C68
:10D82000E06564E04871682B65644164E04544EB61
:10D83000B068CDB42BE5AC88138478703D64E065A6
:10D84000443B8CE5AD3D6413208C758DE020843322
:10D85000985E580D54214C492498FE2BCC6F1568C6
:10D860004330FFCC3766EB235162203C560630181C
:10D87000662D5A308766D3309366FBC8CC6100FBB7
:10D880004E9C90CCA7601B7A1F7ACBF55A894858DA
:10D89000C17085641385644B1C20E2B78C73E54C22
:10D8A000300671643470C28412C300133383533B57
:10D8B000DBBBD14413037966E168E09C83016442D9
:10D8C00049621B985E3E4962E54C2B3008716480CA
:10D8D0003482C2848712C300CB033B3B6333538B38
:10D8E00073EB1568E365203BF168E05CE17084410F
:10D8F00062F168C1B008ED48B3447168008B294EED
:10D900008568668698663315C84D68CBC658E02092
:10D9100030F1CC256366E3E0E008017201EE884156
:10D92000DE9870C4F57CB058E0000000A09C4ED09A
:10D9300090CEFBE0B87CD88C6089028D0C011A195E
:10D9400018300289407D4070514CE83888084D50AD
:10D950007C46EE173A70842689400EEE6B8899500B
:10D960002B301AF1424E360ECFAE7C466860094825
:10D97000B0300446068C1B66367066A658851406C1
:10D980009806678826260613848568238C97A188C5
:10D99000C1B0BD1C0E0F20120F0F0D38F8214286AA
:10D9A000C626704E7EF0C6704EDC90901090F0044B
:10D9B000A96858B0C6260E2568869806B05568989E
:10D9C000A658A670660638D87066D8F026ABC67022
:10D9D0002658B0F65BF04670780E98702658AEF078
:10D9E000B09C629F0948EE173AD87026D8F0BE3F27
:10D9F000A6667006388BD152982B148140CD6C2EC0
:10DA00005899501BB5A2A0DE1B8E0E70984E5E3347
:10DA10000ED164AE734E9C501090D05010D090AE8A
:10DA20000E874570380EB00E286B8606B05568C656
:10DA30007038FC1CAA0C2F0A3967134A7CF026A602
:10DA400004A568A6A6E0A6496870381C3E607E1250
:10DA5000B3E0067038F61366663C46FC0606E051F5
:10DA60004C4EF0E0DCA030C0085C905C0E13664EBB
:10DA70007078067BA60670383EAF7E62A0FC5646E4
:10DA8000EE770CA0A398496870383E6F98A658E0CE
:10DA9000894833D144E07EA060B03AE06954F69BF7
:10DAA000982670383C05688D70CE0EBC555CD91C2C
:10DAB000B83B4C604EBB514C894038339870384667
:10DAC0003C0E0430059C5A109010DCDCDCDCA0FA23
:10DAD0005A13229AF33A0C534C2BC8CCA023CCED0A
:10DAE000576627D4BA73945BFA5A5CD0905CFA46B6
:10DAF00026139423FA10C3FCAA0E60E086011405D5
:10DB000013514CE838288140EE8349701B4E5BDC92
:10DB100050AEFC1E1B261FE6EBBC89403CA8E8E08B
:10DB20004EDC5050501090E084E80444D828E8308F
:10DB300029E8E0EE514CE8380E4E70AE68A0E09750
:10DB400013140513417013339E048D501BB5A24D61
:10DB50004C98DE1BA08E28E0B432050D0914018418
:10DB6000887B850D091401843B8514010401888498
:10DB700044417013CBB87C1C50600691704C23D884
:10DB80008813D8492430260213A222D888D88C7B47
:10DB90008662271CEAEA0604E948E2B308A3068C79
:10DBA0004FC9705C4267DC906B095060AE3C0E134D
:10DBB000FA4C47DCD0A25D6C6E4BD91C9C10D0A2F5
:10DBC0007CE89CA2BB8C608C603020616C30414C46
:10DBD0001B3050616C304D6E5851B6B6A31C8C7F13
:10DBE000A25390909C5D6C6E167693D090BBA2CFA2
:10DBF000302F0C4B664C73B8D848D81B4C3BE84BC5
:10DC00000EEE0E0EEECEEE0EE0CE30046944A0E035
:10DC100081400E3001A0A65C4636616B7606138A01
:10DC200066F3E0A0A01CE0DCA04EB2CEEE4EEEE02B
:10DC3000F16804E09C23E09C08A0C1B0AE707C5E5B
:10DC40000EAD5C0C60D91CF8F8B00EED4A7E7C1A63
:10DC5000FA5AA57013150E0D0F0E141505170504AD
:10DC6000140815061209130114B01A30E83ABEE37D
:10DC7000E09806C44924B8BCF6F6F6A088E004C5CE
:10DC8000703059D866F31BC570301E0C1BCC8766EC
:10DC9000DB2308C570302DD80C1BCC1F66D3C458AD
:10DCA000A60658E030107030FBF0A838238940F801
:10DCB000D8E0AE8444BC0E30121C0A776A53A0CA66
:10DCC0000A374A881B563348234ADF0660AE3C0EAB
:10DCD000E00E4E7078EE894078A0AE8E0E68E09728
:10DCE00013100F1413514C28E060FCB07CA0EE0E12
:10DCF0001CD09050A636369C133AA2F38E76E3AE33
:10DD0000BC0EDA3CDAB0BA5A707A9A4E5C109C417A
:10DD100040AE3C0E3C5A4E1C50D010509010AEDA23
:10DD2000CEFC70B01AE05D1C0C13C88498A8150CCA
:10DD3000711EE1688CD972E0C97020E0894038A07A
:10DD40002E2E60E000000000000000000000000037
:10DD5000000000000000000000080B6CBB8CAB0E44
:10DD60004E70B89CA2A8B5708C1B585B4C43C1B0D8
:10DD700048042BA16C044484617604588940594CB2
:10DD800038580CC76C2F4C517EDBE8F8D84C4D76D8
:10DD9000D80C1F4CC34670B83CD80C738C674C57DA
:10DDA000D80C7BC97491704898A828E8381CEA57A9
:10DDB0008CA30568EA274E907BF83CFECFFEBF603F
:10DDC0003D5BCC4B3B4E36682B854044E804D8A8DD
:10DDD000288940BD6C88044408844484608940F8E4
:10DDE000D88C3BD83038E8FD7E0C27D8D57E5848F3
:10DDF0003031E8757A980670389C62CFF613666603
:10DE00003C1EA6067038AE7E1B4E23267038AEE050
:10DE1000DCA05CEE5D7AF237B2EEEE7CD37C0630AD
:10DE20005EA61C6A873C5CB27C0E4EB2EEEE521BC4
:10DE30003CD31CEE25510E917004E6C61CEA4BE063
:10DE400008F174A8E8557E3C305E6A478E8E8CBF20
:10DE5000CC87A3FE97C68C7F4C6FD844CCD3655437
:10DE6000D0F0F9700D7EC6A16C49240C37B8D844A7
:10DE7000D8A8AE6841683B8DE2F174A8E8CC9974EB
:10DE80005D1C0C330498A809B8BC5884983CA87849
:10DE900058EE091E44D5420C676554D0F09888BCF2
:10DEA000983C589974E020F97098BC584C93C1B0D4
:10DEB000BD1C14090D051220010C01120D20534543
:10DEC000441333C17098BC5846F06666FB610098F5
:10DED000DC1044E05830F1CCFF66EB2030264C2BB0
:10DEE00008FD7046CC9F66EB987E4B4C1F482B4834
:10DEF0008C979170A56C6B2020441C583C1C0A49DF
:10DF0000CA30C36A8B2E4C4544000D54654400460C
:10DF100066CC3766EB0D54411C4C5F9C985606301E
:10DF200072665F4CFBD57E8C6B480D7CCB4168BB29
:10DF300098E3970F0E0D0C01514C88C4084860857A
:10DF4000684B2315684389400EDB6631687038E6FC
:10DF5000463C0E8940F9740E630C474C3F8C271CDD
:10DF6000C217D5764C43F8D88C1B58E058AEA8E8B9
:10DF70003038E84C60E00C132049244CA7CC091F32
:10DF80008C8B91704C37D88C53C502603D5BC97443
:10DF9000F90C9170048498A82860A05D1C98CD9E0F
:10DFA00058B8EE514C6C9B385888989CC2285D1C20
:10DFB000089842A84B4D4C38580484D91C783C89A9
:10DFC00040A8FE63084E2B00E080E02E6889CE4C0E
:10DFD000EBA56C33587D6813DBDC90F091708CA757
:10DFE0006148D6F970736576817ED968C97071BA57
:10DFF000D57EE976008B93CBD3DB0003320D14CEB4
:10E000000000000000000000000000000000000010
:10E0100000000000000000000000000004000000FC
:10E0200000006C454C54434D613076314C4C8C4C67
:10E03000C1CC34CAAAF4BD031FC60F60481110003A
:10E0400066C4781400404503401794EB00D4DF28E1
:10E050001B505047BB402060CD3D3930B30FCCDC66
:10E060004B45DA6707C225523BE40D172330723364
:10E07000300173171992E4E3C4793F7D6055402461
:10E08000A348451455922000508E404ADEC7B14245
:10E090007CF45845324211EDE291008482183D62D1
:10E0A0001F2246E435C9C708060B94B8FC3838006F
:10E0B0000400020000C07503700D700EC07999CD88
:10E0C0002144688C43D910FDD3B31F8E505448713E
:10E0D000300DD21847374FA8C3E0129BC4139A489B
:10E0E00043315140140AA790161A425812250507C9
:10E0F00029C05104E961838D01501188137A71564A
:10E100000080008018642B00006242E4C615594864
:10E110001122B05884214406012921804253B16D57
:10E120004D79CC4C3C7220125843C53149500611F0
:10E1300036063D6474670E11D01311F643423C3E1F
:10E140005190798704E5501A90281C3EE16288F4CA
:10E1500054B848C554429F0C0388D434242344F255
:10E1600025D28109C71972A2320444064DC1405D0F
:10E170009C371CB6DD05353DD50E91263405A61C11
:10E18000040000000050AAAA5645851700069754BF
:10E19000CC998911501ED521961D5B33B72DF316EE
:10E1A0003E7719A53409564948885810C210C00452
:10E1B000914520A1BF00E353659537581944293E86
:10E1C000393D501CAA504A92A43442826DD5F227A0
:10E1D0007F17CE091D12C7C44521481C9311EF3388
:10E1E00052043033002134C623334E16DB03830C34
:10E1F0008040CF1708042E12308010011F0004F059
:10E20000005050605B1294719219441A681820E40F
:10E210008111732E51556463F4782414576CF98B73
:10E22000C8843851445398464100C080724C06D18E
:10E2300054587410000004BC600A0664D978675C06
:10E2400015CDD4F479B92790C444030AF5B70B006F
:10E250008419356F23B2967C84E1336A844D124968
:10E26000CD3A57333300601F288AA82014585154E0
:10E2700084469A8F868896862C26A619685C8051DB
:10E280001DA01835109015047F850914C2808618CA
:10E29000554C09EE9F488D763112ED113E24EE4328
:10E2A000DE5422D1C4DD6625291E6D36DF5C0709E8
:10E2B0005684F52F6017F2F3C92F10050EB0E40055
:10E2C000D4644280818877CE08D907773035213AE7
:10E2D0000004744025CA00C000C0003010CE99C5AB
:10E2E00070D4E03F4F1F1610D8239810837030036E
:10E2F0007F3CC745C405403EC11F34DE01F237FCF8
:10E3000065BD1FE556C86AC2BE84C0D5260232204C
:10E31000990FD365550000000000E4DBDF31D55FC5
:10E32000A54E458C539531BEF4617C1C0F553C6362
:10E33000134C7C428772483200D44B0852E8D43BDD
:10E34000858100E561462545102EA32F6192F48753
:10E35000EA0000000000D44C786C333009D95757DC
:10E360009D83357303E17F541319DF2C724270488B
:10E37000F5601CF11D6D0B1ECF01C13581952C522E
:10E3800047828002B226FC5FF03B073FBE930987BD
:10E3900012DA311F4E3030565B05853C8F46104AED
:10E3A00002FCF4B3398AD6461379D53003000088CD
:10E3B00001D5AC4BA6C5F82D15E3B97866D406DCBB
:10E3C000C4805107BE57C0500C94531B0100D56246
:10E3D00081719009D8D108CB7EC0F383013B4738C7
:10E3E00063304C4561FE89344D7D7F24CE57FBE47C
:10E3F0001D40B70D9315ABF6665D665456FC0B8851
:10E4000000F8615044FE1348260E7676B5A3D91C59
:10E4100078D88484D88C1326F046F009C886E64B59
:10E42000309EA62BA058F142CC2766EBA3D91C78CE
:10E4300058203C56069CE21B4EAB3012664761C822
:10E440006686A568E330C4064FC64ED0A646263C75
:10E45000A3E6761C4E906AC6FB303162276A13A68B
:10E4600062AA3C26048C2B08A07E60585D1C98BCD8
:10E470009CE22B0602A2E6C602A23003622F1C42D7
:10E48000136230088C270C237B0C134630555EFC3E
:10E4900006BC30E61BF61B2E03068C2FC16813C387
:10E4A000A60EA05A7C1AFAFAFAFA56233C3AFCEE67
:10E4B0001A46BC26260E55C4604C61008859C8789F
:10E4C00028B86898A859C4EA005ABC1AB0303AE68D
:10E4D0002366DF461AE0BDD065F04C2FA18002DB39
:10E4E000CC3F4E70B8584C7BCC6795A43C0A59A4DD
:10E4F000E5A4D88C1744A180FD188A8514064E70B7
:10E50000CA685878A6C6026A6DCCB05E3C062B5D20
:10E51000C4C830DA7004B07C0E01D0EDA4AE3C6605
:10E520007F7098AE59A48D8CAE7C6606FC5843046F
:10E53000987C1666C3084E70980E78061BA66878FD
:10E540000E59A430C08D8C4DA4468D8C4E587078D9
:10E550000E4C23C4BD8C783C667BEDA4D884D88D4A
:10E560008C29A429A4AE0E584E70780EB8BC5884DD
:10E57000E0DCA0DC1050121C8AE5A43C5CF2CB7EEF
:10E580000F02FF1C8A4DA4EDA47C6A22D398AA69CD
:10E590008C0A588C574DA459A4468D8C980A29A4EE
:10E5A0001B1C6AF5A89B623C5888821B59A4468DA7
:10E5B0008C42D762101C021F023BA666700A4EF006
:10E5C00098AA698C7038989C50F09806467078A686
:10E5D000682E063B6670EEF0EECB4924F85A5EE8F2
:10E5E00030BF2684A80E78AE66CB70380E4670AE6B
:10E5F0003E8B1C8C137CEA330EFDBC95BCB88C1F83
:10E60000884B781C0A29A429A4B8AAA8A1801C397F
:10E6100088E68F0C2F59C4F0000DFC03080B13156E
:10E620000DD9FED5883E434670AA680A4DA4E5A4DC
:10E63000AA704670785816468386FDBCEE4B66B8C5
:10E64000FCEE0825AC1B95BC780EE3D1486E2B5927
:10E65000C42E1659C41916D1486ECFA3D1489D486F
:10E66000FE738BD1486E4BBBD1486E439D48FE2351
:10E67000FBD148CB4E3E304C0EB87E5B81C806784D
:10E680003C06B9586E63AE6E7F3A3A3A3A3C7038FF
:10E690000E8E844E70F8E030546E9B305A6E736666
:10E6A0006E53666E33B5A20EA04E3E7EC37E7EA034
:10E6B0007ECE7E574E43EEA0663346F6A0BEE04EB9
:10E6C0005EE76EE0CE7E1B5EE0E0DCA0DC5EEE1F6F
:10E6D000237CF2F3AE5EEE1F237CF2F30E03E0A583
:10E6E000CCBC0E4670AE6881F04E70789A66AE680B
:10E6F000304070AEF03E55F04E7084B07E7E7E2F7E
:10E700007E89F68801C8E6B5A286B0668DC61C066D
:10E71000A54FC678A6063DC358B0FC06707C26E619
:10E72000F002223DD0AED8E63C7006023DD0B0E605
:10E730000CC38604304006A5D00C49D1C676431CD4
:10E740000A6AA5D049D066B0E6C67038A670A6F0B1
:10E75000986666776651ECA606704EF09866BF8D97
:10E76000C68451EC8C276688D326E67022FC06020C
:10E770003DD0A658B026E6FC063DD098BCA6588CE5
:10E78000A3BA44DDD47AFA9A983C0698767FA60616
:10E79000BF0DFC060C2013091A05D9FEA5D00C9755
:10E7A00098762BA5D00C5F98E63CA6B0FC707CF068
:10E7B0005DC40A3EE6B006A63CA60667BC704E7075
:10E7C000F8FE2F66A6067038EE472DD0983C66AF4F
:10E7D000BB0000000000000000000000000000007E
:10E7E0000000000000000000000000000000000029
:10E7F0000000000000000000000000000000000019
:10E800009CC2FFCC574626FBCC2F5DC4243C71CC68
:10E810006653309066FBC8CC6100839C4262E2A5DF
:10E82000684E9C90CC5F601B7A1F7ACB5DC4E01071
:10E8300071CC664FA5689C228859C87BA568D91CF5
:10E8400078583012662761C8CB30C266AF46F08C6C
:10E850005B59C8BDCC66E627652073BCF05DC42952
:10E860003C26662F8865C82B49F08804E9D48C2B98
:10E870005DC47E3E4E70088C2B4540061BF9C430AB
:10E8800018A6C6B07CEEBCA686A6061F04A666988F
:10E890003CC658B03C0671D84E70B87CD8040C13F6
:10E8A00008D8BCA898668DC77C0EEDA4E601D0AE52
:10E8B0003C58C69C584E7051B41C53BDD0C1D85E54
:10E8C0003E2DE0DDFCB1C0BDD04C1BE9D071F0B0F5
:10E8D000FC700602385AF051FCAAAE3C58C9C099E7
:10E8E000C0980A01D098AA0A5841C480E68741C45A
:10E8F0004C5780E6AB708D8C987C0EB004D88C138E
:10E9000008D826CABFAE3C580AB066577001D0413D
:10E91000C4808D8CAB0C2341C4804B081304980A2F
:10E9200030FF8D8CA156C1D8BDD04CD9C85E7E7E3B
:10E93000FE39E098EEB5F604DCD01EB07E7E2F08DE
:10E940007E29E331F40C533E85E0B05E3E7095F0D5
:10E9500059C0B0CE46CE6E6E68BDD071F04E7078A4
:10E9600058B0FC060201D0EDA48A0456705C0A0679
:10E9700076265766D88C1B086AD86A6A98AACAE7AE
:10E98000AA581C4699C4B0A1C46AB0664F7001D0A1
:10E99000EDA4A1C4B30C7B46A1C45B0830FF99C4AD
:10E9A000640530FFA1C469D095DC0C554AF9FA38EA
:10E9B000BCA6BC288804E9D48C434E30913CEEE9D7
:10E9C0005ACEBC06B07CC698BC1ABCEE4E70385C01
:10E9D000AA581C06BC065F3C0EEDA459A4E6AEBCCA
:10E9E0000EEDA4AE5884C61C6A17881C987C66E697
:10E9F0001F8CAF8CFBFC580A01D098AABCDBE156F7
:10EA00003BB03C263C463C7098E63C0AEDD02E8458
:10EA100049D463BC6658CEFC0A01D0B07C263C7059
:10EA2000983CAA7C5806D3B0FC707CF05DC45E3F75
:10EA30007E2F06ABF0837E7E89F788480DD4CE58B2
:10EA40004E70F80E8C2BEEC3F9FA3DD00698BC063A
:10EA50007F0DFC050E04200F0620120503F1FE6653
:10EA6000B03C065DD8554AA5CC06BCA63CF081F06A
:10EA7000D5CC663002C61306F5C459C42E12000068
:10EA80000000000000000000000000000000000086
:10EA90000000000000000000000000000000000076
:10EAA0000000000000000000000000000000000066
:10EAB0000000000000000000000000000000000056
:10EAC0000000000000000000000000000000000046
:10EAD0000000000000000000000000000000000036
:10EAE0000000000000000000000000000000000026
:10EAF0000000000000000000000000000000000016
:10EB00000000000000000000000000000000000005
:10EB100000000000000000000000000000000000F5
:10EB200000000000000000000000000000000000E5
:10EB300000000000000000000000000000000000D5
:10EB400000000000000000000000000000000000C5
:10EB500000000000000000000000000000000000B5
:10EB600000000000000000000000000000000000A5
:10EB70000000000000000000000000000000000095
:10EB80000000000000000000000000000000000085
:10EB90000000000000000000000000000000000075
:10EBA0000000000000000000000000000000000065
:10EBB0000000000000000000000000000000000055
:10EBC0000000000000000000000000000000000045
:10EBD0000000000000000000000000000000000035
:10EBE0000000000000000000000000000000000025
:10EBF0000000000000000000000000000000000015
:10EC000081C8E6B5A2064540B9CCA6BCA63CF048F2
:10EC100085F08C5BB0FC2670381CEE77709BD5CCF1
:10EC2000A04E70EE59C4EA003CEAF30E4E70AE6896
:10EC3000B01E4E3E1CBEBE33501050903B10BE2B3B
:10EC400010105003BE2B5050D0D3B046FC06F5C474
:10EC5000A3F85E5AE8A878E630C0062663A60670D8
:10EC6000383E334E7EF066A3A1803CD5883E7B7053
:10EC7000AE0E584DA459A4468D8C980EB0E66F7018
:10EC80005DC414218A4E6E56DC90688DB8BC08981D
:10EC90003C28441C6A8AEDA45606303A067B303084
:10ECA00006AF3020469C58DD201C6A4E30056A5B5A
:10ECB00059A46A4C8FEB48783A87783A8DC7B83CAC
:10ECC000D808D87CA88CB5515DC4333B3045663F2D
:10ECD000783A27301B83302B66832666378C7F304B
:10ECE0001A23266627301CD32666678C9F4C435315
:10ECF000F8EECE71C8700439D006B0BCA6700839E1
:10ED0000D0E6172606B0BCA670783C06B03C063CA0
:10ED100006B958BCB95826703C063CE64EA670A60B
:10ED2000F0B02606C78DC60E66176629C6BC069CBF
:10ED3000E2D330901C02AB30316A8B30460217664A
:10ED40009C024B501C62276A136AA6A606C6E6A25E
:10ED5000065E233008465DC46A27F9C40C2F70157F
:10ED6000C8E68DC606F8FEB0C6FB46DE1BA6C6A6E4
:10ED70007079C4AA58B0665F701C980AEDA49C58BC
:10ED8000461C8D8C51B47B4E1C10CC2F6EEB4E4B21
:10ED9000203C56069CE21B4E5330C4064FC64ED054
:10EDA000A646263CA3E6761C4E906AC6FB3031622E
:10EDB000276A13A662AA3C26EE61005DC42E1230BB
:10EDC000FF06F8BC66470EB8A6AEA88DC6B8BC66EE
:10EDD000B5A3840895D0302B06B006273C061B81CE
:10EDE0000A06B8BC13EEA6F30EB03CE630A8AEEEB1
:10EDF000176668A69C583508B0063C260677BC7096
:10EE0000783BF87EFE5F5C10EEAB1C7CEAF33C3393
:10EE100015C83C9C4A7079C40C2F8AB058EDA4AE3A
:10EE2000D87C1C846A1788D8AE987CEA1F8CBF4EA9
:10EE300030051C6A538C2F6A59A40359A4034E70E1
:10EE400030913CEE3B79C46DCCF5C459C4EA00BDA9
:10EE5000E0DC101E46FCBE77E6A670066638EE7053
:10EE600066EEF0BEAB5DC4EE00307A66FB61027800
:10EE7000E8380E38D81CAA28E09CA01C380EF8AA46
:10EE80007CE8AE7C280EE0D4948DC7A0EA73E267DC
:10EE90009846AE283B48084EDDE04E300BAAA0FA5B
:10EEA00060E6133AA6CB3C30030E51C45DC42E126B
:10EEB000B87CD83C30300693302E66370C60A6A65E
:10EEC000E0300D664F302D06E0303A066061DAB171
:10EED000D0AE0E3CEECEFCEA6DCC666686664E3059
:10EEE00007A63AC6F346703CEEBCC66804044CE183
:10EEF000C4E9D00881F08C4BB07EFEA1C3A1F4839D
:10EF00004E70780666263DC2EE4E9CCA1C3E70AE20
:10EF10003C06027098F00DD0A60670B0F07A4670EC
:10EF2000CEAA7C0EE5A4E6AEBC0E01D0C68D8CB098
:10EF3000A626A67A2770AE5B7001D0B08D8C0DD05E
:10EF4000A6704E6EF05DC4F000492438FC7006389F
:10EF5000FCA67C70E04670387CAA0A3C28E00404D9
:10EF600084E9D4983C1C0A0451FC4A2A2AE0306007
:10EF70000698467004261C7C4A300AFC58B8A6A89D
:10EF8000E0D91C78D8E0EDA40616D91C303A6643C7
:10EF9000302C6623302E6661DAE0B1D08E0441A4B5
:10EFA00044CE0637662FA20217484ECA686A054645
:10EFB0000000000000000000000000000000000051
:10EFC0000000000000000000000000000000000041
:10EFD0000000000000000000000000000000000031
:10EFE0000000000000000000000000000000000021
:10EFF0000000000000000000000000000000000011
:10F0000088DCD0FE95E84E705C380AB0AA2845D856
:10F010001388D91C78468C1326F0256C88080404C4
:10F02000E9D40C5B44DDD4CE7C06463BA6265DD8F5
:10F03000705B7C0A556CB03C46BC70C57E256C0488
:10F040004670387C1C0AEDA4563CAA7CEE3BCEFCF4
:10F050001C0A556CDABC06B07C063B86BC065DD843
:10F0600070DA7CE6917AAE4670CE68C1B0E0B07CD2
:10F0700006300B0697300D46DA7C06333017C63E55
:10F080009306301806BBB03C061EA114F87E7E9E87
:10F09000066646F098A6581CB07C26E6CE7C0A048C
:10F0A000EDD098E67CAAFC58CE7C0AEDD098AA5800
:10F0B000CE7C0AD9D0DC101E9E9E1C98AA5804084B
:10F0C00093EDA48A06D91C79B01CCCE746F06A01FE
:10F0D000D0987C6A6F98DE586A8744D91C987E2F36
:10F0E000581EA9763020E805768A48196C4479B014
:10F0F00098DE1EFCDC901E1F5E1BBE5E3C5883ED3E
:10F10000A48A06D91CCC33D9B008357679B01C6AEC
:10F1100046F001D0986A63DE3FFCFE9B0C8BFEDE5E
:10F1200004F3D91C0CE37E9EBEC7F8BEF3A3D91C22
:10F13000B8F8568A063040C64B46F06A196C1B79FF
:10F14000B0980C37FC1E9E3C1E3C9CE2042030F024
:10F15000E6E09CA0443020CC697766E3C666797708
:10F16000E699C8D91C9C6282B8A2F34C1B98F3069E
:10F17000E094339C98A60658A0D88444D84C77C60F
:10F18000A69C58301F6617260698069CE8D09C025D
:10F1900082B8A2F34C5177485576203CF64BA568CF
:10F1A000711C5DC4E01078581A7A7A4E203C5A1CC3
:10F1B0005D001AE000105B504B903BF3D023000041
:10F1C000103C56063044668F788C1B84138884D894
:10F1D000F0A5680C6973517626669FB07C06668C34
:10F1E00023300B4686BC0646F05DD8C97A26667782
:10F1F000B07C0646268C1B300CC653064349247847
:10F20000FC5CEAEE9C300842A17CF6DD7B30088C89
:10F210001F4200957C068C47C1681BC17A7C5898B8
:10F22000A6588CBB796C4A57C1B0BD1C0E0F20127A
:10F230000F0F0DDDAC78D884D8F049246D586100EB
:10F2400030FF66675ACCE3203C0630C366DD7A693E
:10F250007288489806C96C25E8E3CEBC06B07C6687
:10F260002326E6CEFC1C0A04EDD0988D8C0666861B
:10F27000B03C0671D8C97A3008957CE6EFDABC0656
:10F280001C3001667FE6CEFC0AEDD030608D8CB07C
:10F290003C9D7EB07C667766C6E6A658BC065DD807
:10F2A0007C26E633C626E6A658CEFC0A04EDD098A6
:10F2B0003CAA7C58066611F4D3F6278C557B1C06B5
:10F2C000300825400E7E9B9A0507088700D36B3BCC
:10F2D000E3FBEBD323DBB17E75F44670387C0AED9B
:10F2E000A4567626A3617E056C8C1B8413883D761C
:10F2F0006520056C8498F0A568F572796C0AA17B8D
:10F30000B96CB0684829E84670787083BB843BFBD1
:10F31000796C0A5788CEFC0AD9D0B03C26BC70ED77
:10F32000A456768CEBE6556CC6263FAA7C5CCAEEEA
:10F3300083B96CB0FC5CEAC41C59E8056C8498F095
:10F3400046F01B056C8C1B84138898F0C97AB03C7E
:10F35000E6C17A6606265DD8056C8498F0A56869D2
:10F3600072267F556CB03C06265DD80B4666E68853
:10F3700059C804C1B0BD1C07140F201E7E7EC63CB8
:10F3800030033E1B30017EFCE8BEB3DDAC0C3B46D7
:10F39000F0C6E10803A5684E5C10901ACC4F26EB2E
:10F3A00099C8BACB7976300B01ECC3847434857577
:10F3B00035867636370023363636363636363636A6
:10F3C0005B65209300000000E080E006C61C224739
:10F3D0001C8622279C860882CD7EC61C222B1C22DE
:10F3E000DD7B02A29F8C174230555EFC06BC30E0EC
:10F3F000000005CAF3EBE3DBD3CBC303180D14679E
:10F40000308AA630BD8B72201165E34F0B1D10238F
:10F4100050C604A89C60C74C81496A521BF515F37D
:10F4200014124485B60825C6205B15EBA2262A0ACD
:10F43000400C50AD3C362203820F003532388184B7
:10F44000D80400CCC040819010038074D184F5B002
:10F450004DC000A409302333CC5068BB881F88FB03
:10F460000D8C8C84D4CC0035C0A803033C3181863C
:10F4700021F25B38338A1CC3A1362321B22485E8EC
:10F480002ECD8843480C08000638622380C71082BE
:10F49000B02066CDC040FD657EFDF5E6D61831D1C1
:10F4A00018C0A82221727CBCEF43E2F030E363BBBA
:10F4B000EF0C2320EC20ECFF10A2A0802122282AB0
:10F4C0008221C0C3953C412282101102821108CCD6
:10F4D00004002088310089FD0CCF0B1042084991AF
:10F4E0009D3055C3080018E00D7800880350F08166
:10F4F00034242AF102000000000000000000000097
:10F50000C9E0331053FE72482113E20331158A35E6
:10F510001D23C6B0CB28320EF88A423203980C4025
:10F52000102131411204B81BCE392500C520F0044A
:10F5300052D9C408182044D915449146A603153D54
:10F540006D50210009076954011693A150421A4ACF
:10F550001B050452C7AC8EA0418010409A4F5D112C
:10F56000040481004227644114441785A2244348BF
:10F5700061542468441EC98009CD33A1DC50106A4F
:10F58000821041C1B30601194525880333D6404393
:10F59000482331E50800000610D014294304310047
:10F5A000000000000000000000000000000000005B
:10F5B000000000000000000000000000000000004B
:10F5C000000000000000000000000000000000003B
:10F5D000000000000000000000000000000000002B
:10F5E000000000000000000000000000000000001B
:10F5F000000000000000000000000000000000000B
:10F600002134432432A02C3222037A488414111767
:10F61000C54108160E3BD19008DA2308D40C50B827
:10F620000320AAC428201417170E003183AAAE7332
:10F630007F3703F17A18EB40E8C42EE340E044E062
:10F6400088114C2046211420D24F22D41E7F7C8C5E
:10F650003FCF143D4D34004238019D1008E1503237
:10F660000030344E4207C404A89C60C74C81C84097
:10F6700045D3F0D0801231CC44D401412433841BD3
:10F680008E32F62E61200609FD73B40CC10CF38C8A
:10F690002108C44098186081620F848B9EC008279F
:10F6A00008C70FEEC5174060865D2403B731315C93
:10F6B000C744C7CB50005044642384930C32E88C79
:10F6C000683D00088509240A6002040084C0000027
:10F6D000880E841800A3512E4891801E8508048945
:10F6E0004F2F313131B13C1432C3085200000000B9
:10F6F000000000000000000000000000000000000A
:10F700000B801A2838215A84720934015C0504954B
:10F710006824000054180D059034E248C5443411A3
:10F72000140F3113C411249811405844587841C41F
:10F73000084D700CC447E3244571A11991368087A8
:10F74000D0CC54010C8D2B033B0371330F45304655
:10F7500034D6061D20F4E668C8003744C8516C4B07
:10F760004C8C214BDD14E55131D0141E6300C000D8
:10F770004931CDEC56540E954414C339144A34879C
:10F78000064767C5C435C67D44753300E0B41B2306
:10F790002DBC141F595580D10A901110105C9C612A
:10F7A000C4004500148D4105090941465124C9444E
:10F7B0007155591055508296A0968978626E514DB8
:10F7C00085094A4DF5430186E051080816C68CB1FB
:10F7D0009C01B0079E01E6167941C088F20C200515
:10F7E00021A1F70C331654E3D21600000090AAAA08
:10F7F000884077282F3FC5A2474B85F630FF3F88CA
:10F8000000000000010000000200000003000100F1
:10F8100005000100050101000800020109000201C4
:10F82000090102010A0000020B0000030C000004A1
:10F830000D0000050E0000090E00000A0F00000B6D
:10F840000E00000C0F00000C584E5554302000588C
:10F850004E5554312000584E5554322000435846DE
:10F86000554E300054494D45522000435846554EA0
:10F8700031004164764C31200041647655312000DE
:10F88000416476553220004D6174683144005374F0
:10F89000617431420046696E616E63005A656E7232
:10F8A0006F6D0047616D657331004372645264721D
:10F8B00000486F6D653141005050434C205200505C
:10F8C00050435520520020502058203420312043EE
:10F8D00020582020202020202020202020202020F0
:10F8E00020202020200020687474702F2F706178F1
:10F8F00065722E6E65742F70783431637820202005
:10F90000202020202000204D616E75616C206F6EDC
:10F91000203A2020202020202020202020202020CD
:10F9200020202020200020202020687474703A2F8E
:10F930002F636C6F6E65732E70687765622E6D65D0
:06F9400020202020200021
:020000040001F9
:100000001640008F00A60299009E026600950247E6
:1000100003370309031E032602EC02F90451052FDE
:100020000557056A0577050C059104800485048A47
:10003000048F05B104630456045C046A047705A5C3
:10004000059A05D205A005C204E70504051204BE01
:1000500004C904A904DF04D004D7051604B0049E23
:10006000049704B704EF05CA054605290522054F84
:10007000056405710583058A05BA05360608066319
:1000800003B400008220160E0F03201604012DE099
:100090008E091805084830088B8E0914030F300F9D
:1000A000438E090E0902300244E6B83C5804CC1FC6
:1000B0008C2BC4840C5F04C1B0301F682668C668EE
:1000C0001E2B6520610049244E00309D3CFA7EB80D
:1000D0003C98FC6D1C3C587EFA7A6F605B0C2F08D4
:1000E0006B0B133C7A17FCCC8B0C67793C2E3812C7
:1000F000C6C3837711C08070301084743485753521
:100100008676363700E3E323DB53B300C3666666C7
:100110006666666666666666666666661B693CACAB
:100120004CE733FB300A06B34CA7DB5E23793CDE99
:100130002146A3B87CD84C1B441348D83CA8A34CF8
:10014000EF8B4C1B446B485B5E2F6100410EE0D986
:100150001CB8E6F8302006A8B8B856A66617B8A6A8
:10016000E826E8C6E8BE5E2B6D8CDF005D1C3C58BF
:10017000200BE066D91CB8569C5806E223E2E20642
:10018000A2263B66F8693C2403DC904C1B7E7E066D
:100190007E9BFEB806B8300A664623302F0626E856
:1001A0007E3E23C666E8E6E89C98E8EB5E6BD91CC9
:1001B000B8E63020E86606B8B8B8566613F866A602
:1001C000E8E6E84924793CC8B01A5A300CBC1A70E9
:1001D0008DBCF10E8498A8793CDE5D1C1106E0D937
:1001E0001C0EB89CE2337E7E4C137E7E302FE81CC2
:1001F00022A6F8B0E21B62DFA0FCCAF61F226656F8
:100200005ABCBADEFA7EF35AF8B0E2736263601E3B
:100210003009065C422FFAA6E30E6EC1B04924B83D
:100220003CD808D87CA8208CB55188EEE8E04E2058
:100230003C063018BC1AB0303AE62366DF061AE0F6
:1002400097050916180508F8AE6D8CDF8C3008008C
:10025000E66D8CDF3A5C005AD070088DBCF10E97C9
:1002600005091614030FF8AE6D8CDF8CAE0E9C00E2
:10027000E21B8902DCE2E7E2D7E05CA01C4EA202AE
:10028000E2EEEEEE3CBAF2BAA2DCD493300FE669AD
:100290003C51970509160E0902F8AE6D8CDF8C4EA5
:1002A00000BA1A3CFA1B8902E6EFE6DFE05CA01C0C
:1002B000BAF2F2F2BA42421322A2DCD4A33002E62E
:1002C000693C51B8AE6D8CDF8CAE00F06D8CDFE711
:1002D000A600F0EE3004EE465BCE1C58DC9886C3D8
:1002E000EE66F3BC463CE09918140F12793CC370DB
:1002F000793C43B0CBBF140902793CC33CD88C276E
:10030000D8B95AD8655A840E01793C43B0BC463CF2
:10031000BA6D8CDF6C6E008C9102A902920F793C51
:1003200043705B920F18793C4358AEB0D8AEAEB074
:10033000AED870D3940F0EF888AE6D8CDF8CBA00F7
:10034000BA005BF88458B8AE6D8CDF8CAE00D8AEC6
:100350006D8CDF8CD800E00B00A188C1B080B0307C
:10036000063000E6465D003CA6BC300656A87A562C
:10037000D3492408000170ED8A0B00C1020B00B9BB
:100380004A0B0089520B00B5A20B0089020B001921
:100390005A0B00810A0B0009828814010D201604F3
:1003A000012DE08D1614201604012DE00B00A1880C
:1003B00080E00440CC00F3004D50A631F27F3A6952
:1003C000111B1342A631F27F3D85C2032F0270C676
:1003D00000F600534952544EA605C8012F0470C6BA
:1003E00000F400535A3FF653495A453E3DA631A802
:1003F0001997738B9BF37585C8032F0000000000CD
:10040000050E04200F062001121201190E0F1420F0
:10041000011212011920060C0E010D052005121201
:100420000F120E0F20120F0F0D04090D20051212CE
:100430000F120E0F20182D0D050D0F1219150E0499
:1004400005062001121201199812140D201604013C
:100450002DE0AB14010D4EABAD14010D308073AA2D
:1004600014010D30203BAF14010D30A0D8793CD9D8
:10047000038D090414010DF86150753CD6CFAB090A
:100480003016F3AD093056CBAB0A3036A3AD0A3087
:10049000767B810A09130D30053B8A09130D301153
:1004A00058F86150EB8A09120D3013ABAB03130DF2
:1004B000301273AB12130D30323BAB03120D30927E
:1004C00058753CD606AD03120D30D2ABAB12120DEF
:1004D00030B273AD12120D30F23B810A09120D30A9
:1004E00007FB85160F0D0DC4483B900117130DC473
:1004F0008808F86150B80E785150753CD697BF0502
:100500000D010E0D793CDF22BF0D0904793CD62286
:10051000920DC433930DC4608848793CDFD0BF127C
:100520003E12C448C3923E3C12C493833E3C03C473
:10053000085B832B0319B86150C40888F8615075B3
:100540003CE5CE96091008048B820118010D1204B7
:1005500043820118010D030808844884F86150EBB8
:100560008D120E1204338D120E0308846B8D151339
:100570001204338D1513030888448404753CDFF19D
:100580008D1513883B82010D151384843B8D120E4B
:1005900006888844A3820118010D84845B8E090DAE
:1005A000882B98010D8488480804793CDF428D2A05
:1005B0000D793CE56793100E1214793CDF49960ED5
:1005C000090D793CE5259319130D793CE5EA94056D
:1005D000040D793CE58EB030CBB030F6F6366BB01A
:1005E00030F636F63BB030F636F636F61336F613FE
:1005F000363A70DADADA3ABC80E000000000000037
:100600000000000000000D50CA00F6004D454449AE
:1006100054A81B10A5AFCF66A90AA819A5AEAB199F
:10062000B6B2018BA5A8AC0AB6AA87A5BFA5A59BA3
:1006300073AC08B997F27F3FA9178EA5A57179A56C
:10064000AC9A73AC17A5AC0AA596B12A09A8157E79
:10065000BA0BCF6F06AC071DF34D5452A5A4C40CC2
:100660002F1F10C401F700434D45444954A81B07F0
:10067000A906A59283F74E4F542043505868124B59
:10068000638E75691A10101245A806AC06B1874B27
:1006900067B1838EB72701A90A73CF661242111A78
:1006A00010101141A819A5AEAB19D07D8F02AC0A6C
:1006B000D0778FE06683F352452EA5BFA5A59B7327
:1006C000AC08B994F27F3F8EA5ACAC06B98AA5966A
:1006D000A594A5ACA597A59509A815AC087EE03B07
:1006E00083F3494D2EA5BFA594A5A59B73AC08BA6D
:1006F00091F27F3F8EA5B0AC06BB8FA59554A5ADFA
:10070000BB880A7EA596AC06B25D0BAC0AD01A8FE8
:10071000AD06A596AD09A595B26D04A5A8111A1050
:10072000101140124385CF6FCF0FAC071DF34D540E
:1007300052A5A4CA1D2F2150CA00F6004D415452A3
:100740005801A902A81BF5524C2043588ECF68CF00
:1007500069CF6AB114CF67A802CF66F74F524445FC
:10076000523D3F8E616883AC024030511140A6215A
:10077000AB198E2083F152111B1C134240A59DC260
:100780000AF4004D5452CF6F02A908A907A815A872
:100790001BFC2041204920445420422053458EB266
:1007A0001904F152A5A0F44445543D9B737EB22830
:1007B000CF7BA808CF66F152BFB9CF67F152A5A28F
:1007C000B23ACF68AD02B4279F00B244CF6AE02DA1
:1007D000829A73F2522C9B73A5B2B254CF7CF15221
:1007E000AC029F00AD02A5BBB262CF7EA808CF6964
:1007F000E00B820FA807AC02A5BEA5BD03F152A570
:10080000926883511140A63175A819A59DAA198532
:1008100074401140A6218ED0926FC2162F3D30C079
:1008200001F4005A5E4E8030754F205371204271A2
:10083000054E01AC0485A815F2553D9B737EF2561A
:100840003D9B727E85C605F5004D41475A4FA81560
:10085000F2523D9B73AD047E85CC02F400655E5A76
:1008600081554E80B134CC01F4004C4E5A814F502A
:1008700080B141CC01F6005A5E312F4E8030131604
:1008800010714331754F20686053712068437104C3
:10089000E061049700B28185024F71214071B4116B
:1008A000C606F50053494E5A81325A7133E04C8ADC
:1008B00042225923E0518B4280B100CC03F5004322
:1008C0004F535A8132597133E0318A4254225A23AC
:1008D000E0358B4280B100C004F50054414E5A818E
:1008E0001242325A71124233E01D8B4023E00C8ACF
:1008F0007143762259714380B1000B83835871553F
:1009000043715840BD850C558360400D124385C02E
:1009100008F400615E5A7532717450427622421DAD
:10092000F3655E5AC003F5004C4F475A5034758149
:100930004F5024957195727580B100C403F6005A2A
:100940005E312F57327533753151713051402071FE
:100950004354762171432322C204F4005A5E578126
:100960004F504F75754F7175427540744E554E809E
:10097000B100CA03F300432B71067540754074B192
:1009800000C202F300432D547154B613C801F500A0
:1009900043494E56E00482B100034F607154714EDA
:1009A00085C003F300432A4F75754F757571754205
:1009B0007540744EB100C003F300432FE024021DC4
:1009C000F2432ACC012F5B70C600F400504C591240
:1009D00013A621AB198ECF6AF84445475245453DD1
:1009E0003F8E1245D00F6A71121146D0166A71A857
:1009F00000A903A905A9069116911506E04B8C974D
:100A000015B608E0448CCF6FA815A81BFC465820EB
:100A10005254202020204E45578ED0156FCF66A906
:100A200006901691157183838397159096AC059562
:100A30007342E1E18E9073909642AD0571F4463CAD
:100A4000583EE18B8FD0406F0DF1619015A631F3C8
:100A50007F3D3F778E919585CF67A619D0576FC898
:100A600015F40052545312141A11AC069117AC0528
:100A7000BB9390161141911590960C95959715BCC6
:100A8000079500A8050B2036213722382339243A50
:100A90009016121040A819AE73F34E3E358E85CFD6
:100AA0001911101A10101691149115E12E902DE0C5
:100AB000DC842A11E17191E16E91E16B91E1689121
:100AC000CF18289112543827911129911342269159
:100AD0001014424137901214429013514190104229
:100AE0009011514136A900E06397AA038503AA0239
:100AF000B1882D29453D2D2A453D0190133C129585
:100B00000C950D2D51901041661000111B1C1845BD
:100B1000E0358675523F2C2D4290111243416711EA
:100B20008361433E2C519012412D12424052940E4B
:100B3000A800E00287082C2E543E40372D2F543F4A
:100B40004036E02796850771777185CF17181A1000
:100B5000101691149115E08390AC03852DAC00E044
:100B60002C842811E0C191E0BE91CF162754124386
:100B7000838351264166B1A2524039AC00E00E8415
:100B80007476413AAC00E00584A9028505F4524F21
:100B90004F54E03B8F77E02C8D850154523B742BF2
:100BA00054AC00E00586A802850774F155E0208F5B
:100BB00074F156E01A8F74F155E0148F74F156E019
:100BC0000E8F850EAD068591979617917385CF0F81
:100BD000E00E0DF27F3D9B737E85CF10103D268386
:100BE0006167B4D0433E7690956140566811405796
:100BF0001146713C0A1110950C2E543E092D2D2CD6
:100C00002E42403D78858383E00B8E67852E4266B9
:100C1000B916BA200F909540429715BF099095409C
:100C2000901491157585CF119715012D424090951F
:100C30007191958504A803103D27362837E0D41616
:100C4000B300C0452F2320C201F600444946455158
:100C500019A621AB198EA815F54E414D453F8C8E36
:100C60009A07F74F524445523D3F8B8EA901977327
:100C7000A801FB535445502053495A453D3F8E121D
:100C80004331F458303D3F8E32F459303D3F8E337E
:100C9000AC01E02D800A2322E0958135E06B84369B
:100CA000E06784920683402340222183403440E061
:100CB0007E81254026834040134324E05482BA2B92
:100CC00001F559302E3D3F8E340B242322E0608104
:100CD000353021E0498636302120244025E0448506
:100CE0009206834030218340E034862683404025AD
:100CF000401343244034762625401343402183404B
:100D0000354276E00C82BB3F052340222140B29E53
:100D10000392027192038F980298037F8507202423
:100D2000402006124324407442234022744002AE05
:100D300087082142CC212F3A50CA00F3005643A91C
:100D400004CF6FA815A81BFC4450204350200D2051
:100D50004D2055568EA627D0176FCF7EA62DF16455
:100D6000CF14F27F3D9B737ED0286FCF7DA62FCF0F
:100D700068A62CF10DD01614CF6BA62AD03C6FCFED
:100D80007BA629D0068FCF7CA628CF0FAC04D04EEF
:100D90006FCF7FF2583D9B737EF2593D9B727EF27E
:100DA0005A3D9B717ED0656FCC0FF60043524F5376
:100DB0005383CE023042CE022342CE01947171940D
:100DC0000342742042234121744190712241CE712B
:100DD000A62785CF67A623D04E0FCF6DA624D09E21
:100DE0006FC208F300565361686877139474967461
:100DF0000F7591F496740F7591F496740F7591F4C4
:100E0000757585CF6EA625D07E0FCC05F3005652A2
:100E1000686175A627741342134090F3977290F29D
:100E2000977190F185CF66A626F3444F54D0CE1427
:100E3000C605F400444F54214271224240712342BE
:100E40004085CF6AA62BD0BD0FCF69A62B74F14D7C
:100E5000D0F114C005F30056453175327533757500
:100E600085C002F300562D1C11A62EC601F30056B4
:100E70002B920175920275920323222185C802F4F8
:100E800000565859CE0175CE0275CE03757585C8CA
:100E900002F30055564F90714F917077114ECE70FE
:100EA000754E85CC02F300560DA62BA62AA62BA6BE
:100EB000265D85C402F3005644A628A62B7485CA75
:100EC00001F300562A9470947142C8012F2030C05B
:100ED00001F30054521117A621AB198ECF6AA91B3A
:100EE000FA5A302C59302C5830203F8E13A62477D4
:100EF000F5524F540D3F8EA90567B198A805911082
:100F00007311CE71F7632C622C61203F8EA62B12D9
:100F1000A624CF6F01A81BA815A901FC5E4E205E78
:100F20004F202020204E45578EB117CF7DA622CFCF
:100F300066A801A630D008FFCF67A901A630CF7FF1
:100F4000F2583D9B737EF2593D9B727EF25A3D9B57
:100F5000717EB140C013F3004354AD01B38813A6B2
:100F600025A628AD058503AD05B2B611A62412A6A7
:100F700025A6239010AD015459A62E1130A6259018
:100F8000105A9300A62EA62914A62412A62511A64F
:100F900025A6269400A62A20A62E14E00783AC01DD
:100FA00085021304A625A629C00C2F00000000000E
:100FB0000000000000000000000000000000000031
:100FC0000000000000000000000000000000000021
:100FD0000000000000000000000000000000000011
:100FE0000000000000000000000000000000000001
:100FF0000B00D19E000000CBC30000311604011885
:1010000000000000000000000000000000000000E0
:1010100000000000000000000000000000000022AE
:10102000020000C0001800100010F223E3F3C4CE49
:10103000201214C16F3C5888FFE6EF080000000042
:10104000006804545555554D1CF1EC4CE30DC03D62
:1010500006CC23E2CCD14F333B3713F22B3353541E
:101060000D4FAB28CF1D48E80DCEB33713DBCF1C97
:10107000734C456417FC24E2F05112F1F2F2BA28E5
:101080000479EF2FD173C3C4FD7D138C14D5CA63CB
:1010900000004C444C10D705000013542274334018
:1010A0005513ECC10800C0041122DD0C5430B20706
:1010B000234C101304C12CD07530002333008C3C1A
:1010C000C300CC074CD033303F30E7E1B4003341AC
:1010D000220713141335CDD4650D74EC47C9D01015
:1010E000D0109010D01000003000C0348D0110419D
:1010F00041111462000011620010004444512100AB
:1011000001000001000001001000040010000004B4
:10111000000000000C0000014000104F02003301ED
:10112000114410410440001033000400014000103D
:101130004F00C40031400C4008C001C0CB1033093F
:10114000009300D330B0330D70000CC002C02CCC23
:10115000246000800080910C00022000088064134D
:101160000000800060008000024839054C0330090F
:101170003005300530D9744967746618DA6F050098
:101180000080010044111111511151444404515483
:1011900044441145114500116200004411050054FA
:1011A00055014544455114154011111441101011B9
:1011B00011411111111145140444444404454414CF
:1011C00051115104111151045015110144880100AD
:1011D00014110045444444004055541551454045C0
:1011E0000010454404000050141140141111111155
:1011F0001111111144101111111111114111114549
:10120000541545445551106200505555551441141C
:1012100044050014414405005511005445000015D3
:101220005455555541445515010055055541450046
:10123000405541554145004055554105555551557D
:101240005551555500505555000100555544450020
:101250000055555555550140555555551100555595
:1012600004401501004154550540555555110041A4
:1012700040880140441401005441515044444441C9
:10128000441011010000144444544544144414050E
:1012900010044544404511410010101111155144EE
:1012A00044545555114504540440445050411004D1
:1012B00051545154544545455145101551555554B7
:1012C00044454540415545555515551511545555FD
:1012D00015545504101144455041105555155504E9
:1012E00055114405101454554510550445500445F6
:1012F00050514414411015551555545555455455E4
:10130000555541551145454411155115454555054E
:1013100011620000451401501100501111000050DD
:1013200015400550115441414154555550555510E3
:10133000054055055550550551554155555555557F
:101340005510551545514455555555555421064090
:10135000444400000045101111444144440411412B
:1013600044101111441005511005010014151551B8
:1013700054551515514410110440551115511115AE
:10138000554410005554151111450404014055559C
:10139000151144144100545505404400445154056E
:1013A000005114550014451555004444540044544C
:1013B00000441462004444110100404501501411DE
:1013C0001501004511454400000045444404111135
:1013D000411444411401105144544451444445457E
:1013E00014114551444451105511210000000000D2
:1013F00000000000000000000000000034C003E016
:101400001839F738F77FF3A2007B00BC00CAF3CF8E
:10141000F81FF845F859F866F873F8A0F8BBF8D744
:10142000F90FF924F93BF958F972F981F98CF9A10E
:10143000F9B6F9C8FA5FFC470DDE0E280E3F0EB470
:101440000ECF0F5CF3DFFD39FDA8FDE1FE0AFE3093
:10145000FE53FE61FE6BFE7DFE8FFEA3FEB3FEBF5C
:10146000FECFFF540FB7F3AB0B900C350CA40CC19F
:101470000CE40D21000085160C0F1308793C2C6834
:101480004670F87030C070381CD0F0A04E68A8B01C
:10149000E80E4924B8AE4EEED74E9F30C7704E5C72
:1014A000229CD08628E806706048658C015C621B2F
:1014B000A2A230C770AE738705140E0904793C2CC4
:1014C000A8898C00900F0F0C0913CC37793C92C47B
:1014D000E0793C3BEEA038588C4F0C27693C924C8D
:1014E000E733784C270CB3B846FC064924F81E7E37
:1014F0007E37793C92895270A6A687A647A6B7A6E2
:10150000BF898C5DEE3B0E658C32EE2F58658C21C9
:1015100070658C3A898CC5898C50793C92793C1ADB
:10152000120503151213090F0E898C881E7EF87E92
:1015300023B87E37793C92895244793C3BEEA338FC
:10154000580C270C63AB8C9F884844CC13488843C5
:10155000084404CC13080898F04670B87C588C876F
:1015600088983CA86D8C9F580C1F04138498F04CED
:10157000471348300B0C1F301E06793C65E6534C70
:10158000C36D8C9F580C174B793C92793C1A0E0F07
:1015900020120F0F0D898C884E58793CD36AF3DCEA
:1015A000901E1C793CE5E698E6D63C58BEB31C98E4
:1015B000EA1F3CEB58681598EE1B4C33793C92813E
:1015C0000A5C420A0C23AA62231C29A430C3704E71
:1015D0005CAAF04D9CCC67B8584C474EE8380E0AD0
:1015E000AE28B80A30C370387CAABCF04E705C10CC
:1015F0009050105090105050D058681598EE1B4CD9
:1016000023693CBCC80C17C40E1C1DA4BD8C4D9C8A
:101610000E30C37038BCAA7CF0E0A18888C1B0BD90
:101620001EBA60A67066A638E67066E6F0A3BA60D9
:10163000A67026A638E67026E6F0A3E0DCA0467089
:1016400078E630C0067026CB38EEB33E8F7E5C1253
:10165000DC90905C726B5E725BFC560643A6262B98
:101660004EE0E026E046704EA668793C3BEE43A68D
:101670000670264338EE2BFC5606B3668646707815
:101680003CC6BC68860630C070383C1CCA60164632
:10169000A0A6262746E02B66E6C60A3C0A7CF03662
:1016A0006630C1464670783CA6C6A65ABC1A783C3D
:1016B000066626A666A6793C21A6E066866D8C9F06
:1016C0003E13664670783CC6BC682626C61B46E0BC
:1016D00030C00670383E23A626CB30C01E7EC646DC
:1016E0001F661E46707826467CA63C66683C06A6A9
:1016F0008630BF46BC265E1726463C5ABC1A667921
:101700003C21467078E67C0630C0704EDC9090FC40
:10171000A6B606167CE6F67CF04E68A830C00666D3
:1017200070383E274E7EF04626E0044460793C3B0C
:10173000EEA038588C13488CE30C8B084C3F0448BF
:1017400098F0B833844498F07858FB7858C44C1318
:10175000C88CBF6B0C1F4EE0B858C40C13C80C5794
:101760004670B87C5884983CA84670987C1CEAA0C7
:101770000E6D8CBAB858259E4924B0E888793C2A69
:101780000C27793C954C534924B87C588C1F450252
:10179000C502793C2A793C3BEEA0A6067026433868
:1017A000EE2BFC5606B38630C00670383C56062633
:1017B0000670385CEA273E1366A6066686A65ABC03
:1017C0001A6630C0E6793C2E662643A67026064E81
:1017D000F0C3E04E1C909C101C0AE5A456E6603055
:1017E00005426ABFE01CEDA43C3005426A1F1E1B87
:1017F00059A47CE000000000000000000000000090
:101800004408918C6B30C170385CEA1CBC0A46708D
:10181000793CBA5C6AC44213C81CBD8C4C091FC118
:1018200002793C95F858793CAB6BB058793C9558A7
:10183000793CAB793CA2F0418C78793CA8EE2769E1
:101840003CA10EB05EFE23693CAF1EA0BE1D6160D0
:10185000FE1FEE27693CF3793CA5EE63793C9F1CA3
:1018600002D0761613B6F0793CA86838E8F828B0AC
:10187000A8B80E793CB53A356060793C1D793CF2E8
:10188000EE9B793C6A0E793C1A793CB52626BE253A
:101890006160FE574E5C2226260E793C1A793C99EF
:1018A0000E38AEA0BE1D6160793C1D793C79793C53
:1018B000A2A0256060793C1D793C56D85EFE6B790C
:1018C0003C52A04E3E6EA03D60A5500E60793CFD9E
:1018D000EE9F793C56793CA2A02560A550600E7918
:1018E0003CFDEEFBF8700648693C00793C524E5CCA
:1018F000223AA3793CA5EE37B068693C71793C9FE8
:10190000F627693C6A76F0793CE7793C1DB00E79A0
:101910003CA8A0BE1D6160793C52A04D6060793C3E
:101920001D793CF2793C1D793CEC793C06A0BE1E49
:1019300060793CE3793C81793C990EF8AEA0BE1DFC
:101940006160793C063ECE63793C0EA0BE1E607994
:101950003CDF23793C5A793C87EE67793C5A793CE5
:1019600087EE27F8E82BF84EEED7793CA858793C5B
:101970009558793CAB793CA2F04670B0E8498C2A86
:101980000C27498C95B95AA04E5C66503D6030C812
:1019900070382560A5500E30C770AEE80E384E6026
:1019A000E0B0A84E68793C99E8064870693C00B8F8
:1019B00068380E793C99AEE884B0A8F8280E793CD6
:1019C00099A0BE1D6160793C1D793CA50EB8A0614F
:1019D000604E5C223ABE256160793C060E793CA2DD
:1019E000A01D60A5500E60793CFDEE87793CEC7936
:1019F0003CA2A05CFA37BEB626228B5E37FE373A91
:101A00005BBBFEE762FA1B2213667A00A5500E60EC
:101A1000793C99AEE84EEE27693C2A7870F80E7949
:101A20003C994EEE27B08C53AE0E06664870693C6A
:101A3000000E793CA85EFE23693CAFA0B8AE6160A1
:101A4000096060793C1D793C990EF8A0BE1D61606B
:101A5000793C52A0496060793C1D793CE7793C6A49
:101A60000E793CB5BE1D610E60793C99AE680E7969
:101A70003CD3BE1D6160FE9B793CA55E680E793C3F
:101A8000D31D6060793C1D793CA50E793CB51D6085
:101A900060793C06793C1D793CD386BE2561FE7396
:101AA00060793C52B0A0BE3D61BB793CA50E793C4B
:101AB000D386BE1D61FEBB30C970380EB0BE356125
:101AC000A5500E60793C99AE6888693CB9B026266D
:101AD00026BE77793CB5666666E0A0316060E07945
:101AE0003C5AC3793C56A3793C99F823793C990E2A
:101AF0003833793CA50EB8A0BE1D6160E0793C99F1
:101B0000AE0EE8384EE0793C52A0756060E0793C5A
:101B100056C3793C352B793C52E32E7A0B30C0709A
:101B20003868F828CEBE1EE8B8BA9CEAEAEABAA835
:101B3000AA8A8A8AE330C070EED8B81A9ABABABABA
:101B40001CEAE6A8F8EE38E87828BA463CFED8EE5B
:101B50005CE030C39C4330C41C2330C59C7038EE1D
:101B6000D8B8D4CE14EBFEAED83B793C52A0756009
:101B7000A55060E0AE0E58CE23793C56A049606077
:101B8000E030C070B83CA6BCA830C37038BE5CEA78
:101B9000F0E07038E0793CAB0E30C7BB30D0A330FA
:101BA000C08B30C87330C95B30CA434E707828B8D8
:101BB0006898A85CE04E5C22A0E01C38AAFC0EF8F5
:101BC000FCAAE8AE28E0B0A0FA274626765C5A5E6A
:101BD00050EE4670B87C0E9CA2467C60E6E6A0AE55
:101BE0001C2666E21B4213A6B67FB66F58860646D1
:101BF000B6504626561B26986E466030D070E000E0
:101C00004924F870B80E30D0704EF0F0586D8CAB9F
:101C1000AE5830C07098E8A0BE1D616030D0704EE4
:101C200028E8DA2F58693C3E793C5B30C070F825D3
:101C300060706006481344666630D07038F0EE5825
:101C40004670B028EE7004793C6B30C270658C0829
:101C50006D8CC6AE68F8F0E80666693C506D8CC6BF
:101C600078A01D6068B80EB86160AE0E58CE4960AD
:101C700009604EBE50503D60606D8C1D30D0707854
:101C8000A03D6030C070B82560A830D070F80E302C
:101C9000C07038F01D6060793C55B0FED830DE7001
:101CA00038FED83160606D8C1D30DE7038A6F07E55
:101CB00030C070CE284E900E30D070B8A01D60A8F5
:101CC0000E60693C0A30D0704EE86D8CC6B068304A
:101CD000C070AE6830D0705C4E90A830DE70385E58
:101CE00046F030C0704E28A830D070F80E78A01D95
:101CF000602830C070F80E30D07038AEBE1D61382C
:101D00003D60A550F05C4E22A80EA0B8AEBE1D618D
:101D1000FE2B60693C55B86960AE0E58CE4960E84C
:101D2000B80E1D60B82560F83D60B869604E6690D9
:101D3000503D607030C070F80E60793C62B03D601C
:101D4000700E30C070F81D60F00E60793C62E806DD
:101D50006660693C36B80EA0BE35612830C070B8E8
:101D60000E30D070B86160F030C070780E30D07036
:101D700038616030C07078BE2561B0256060793C04
:101D80005B78256068606D8C5230D070F870B8A0B8
:101D9000696078BE2561B02560606D8C1D30D070A3
:101DA000780EF0A01D60386960606D8C35A03160E0
:101DB00060793C5BF02560606D8C1D30C070787080
:101DC00030D070B8A0FA23DA50260EA8356009602A
:101DD00058606D8C95B0AEA06160B0256068EE462D
:101DE00070B80E78A846703868EE2E7A606D8C0652
:101DF0006D8C52A03160709E30C070CE2830DE7085
:101E000038A606F0B0BE256158380E30C070AEA8B6
:101E100030D07098E8780EB0AEBE1D6128B06888EA
:101E2000084E6830C070B84AFC0E4E1C50A8901C7A
:101E3000029C48021BAE44F08C1F04138430D07007
:101E4000780E4E5C10A035604ED0256068F80E30DC
:101E500007E66030C070B8AE26AE7038A0BE1D6117
:101E6000382560A830C070780EE0DCA01CF2525E0D
:101E70001B669230D070B85EBE1D61FE7384083060
:101E800007E66030C070B80EB09C02EB26AE70AEB4
:101E900038A0BEAE60267038A01D60783D60B8697D
:101EA000604E90BE2561FE1B88083007E66030D08A
:101EB00070F80E30C070B8A626A670AEF0B80E78D6
:101EC000A06160F82560E83007E6C66030C070B8F1
:101ED0000E0C33B0AE9C22A80227693C38B80E4CD9
:101EE0005730D070F826AE70AEF030DE7038A03EBD
:101EF000137E46F060693CE2F858606D8C9530D0F6
:101F00007038586D8CABAEA0BE1D6130D07078704B
:101F1000F858606D8C81980EB0A01D6060793C55BA
:101F200070606D8C521E30C07078A03D60B0FA4376
:101F30005A5E5066D414EB2560A550F05C58606D75
:101F40008CABB0A0A550F060D44B30C07038D888AE
:101F5000D8F0418C786D8C52A049624EA05C6650DE
:101F60003D6230D07038AEA0BE1D636630C10C1724
:101F7000267038FC9CA2023CF0A0B0A550584670D8
:101F800098F068A8E87060E0DDAC0170ED8A5470EC
:101F9000C600F40054564D1110A621AB198EA900AD
:101FA000CF7F773132333435D00BEF0FA815F27F66
:101FB0003D9B737ECF6FA81BA916FF204E2C204996
:101FC0002C2050562C504D542C46F27F568ED01B50
:101FD0006FCF7B111242CF66F14E31AB16A634BFE4
:101FE00036CF7C111243CF67F14932AB16A638BF0A
:101FF00046CF68F2505633AB16A635BF52CF69F3C1
:10200000504D5434AB16A636BF5FCF6AF2465635F4
:10201000AB16A637BF6BCF7EA815F3454E44AB0079
:10202000A800AC00F5424547494EF67F204D4F448D
:10203000457ED07F6FC817F2004E2267B49B111BFC
:10204000124336E02F8864BBA32864B29705F624B8
:102050004552524F528ED0A36F042325402467B5BA
:102060001443B18402E0068A015431850B6526656C
:1020700043318509E0118938E00D8939850CAC00C0
:1020800011AD001042850A2383CE05334026543615
:1020900061E0150B114024422623424067B55243AC
:1020A00026425485CC0FF30050562267B189E05484
:1020B0008727254226B2830125210224424054333A
:1020C00085C204F400504D542267B18BE036872757
:1020D0002542234026B28501232540210267B50011
:1020E00043543485C005F30046562267B18BE01493
:1020F00087244223402743B2860124214223400201
:102100005435850822111B124365214254553776F8
:10211000585422111B12434376E09D0B1140423666
:1021200085CA08F3002A492124422340254067320A
:102130006785A9052324E0BA0B403676244154254F
:1021400040374264B500211178B1842463B2900114
:1021500026274267B50027264354216053B3BB02AC
:10216000216011403226244266E065850D2250210F
:10217000425822114167B18343B2820121023811D2
:102180004124422221532642403921284122114133
:1021900067B18D4322422442B28E0311714D3285C4
:1021A0000121112141421243022921424029714358
:1021B0002754294371532242767132714D61111BAC
:1021C0001C1646BD59AC05E00785A90522B33506A6
:1021D000A80522603227CE0637C41A2F4270C600E7
:1021E000F50043464954A815A81B1118A621AB19A0
:1021F0008ED016E8CF6F2BFC207E2B2020434C7E08
:10220000204649548ED0126FCF689900709906709D
:10221000990C70D0206FCF66A61CCF67CF69D02BEA
:102220006FCF7BA61DD0326FC80AF300417E719933
:1022300006917447E021804774920574920485C426
:1022400003F300447E719906917448E00A80487453
:10225000930574930485017576507176715071768B
:1022600094705071947150990C85CF6A2B11415024
:102270000C2BA901A902A903A904A807FC4C20451D
:1022800058204C4F47205020428ED0976FCF6AA6DF
:102290001ED0E7E2CF6611A61FD0DFE2CF6712A6FD
:1022A0001FD0D7E2CF6813A61FD0CFE2CF6914A604
:1022B0001FD0C7E2CA10F500424649547733A980BF
:1022C000A907E01A81E02882E03683E0448420CC2C
:1022D00003F40046495430A880A807AE0002273214
:1022E000292A2628E0408511F34C494EBFB2032D20
:1022F0003229252C28E02F8512F3455850BFA10420
:1023000027322F24262EE01E8513F34C4F47BF9013
:10231000052D322F90102C2EE00C8514F3504F57C2
:102320000FAA0630850631719111422B434171216C
:10233000512B4341434276CE029011512B434143EE
:10234000AC07B78623714685A80607339011212272
:1023500042412B43AC0255AC04553185C214F40004
:10236000593F5821229071AE00045002424085032B
:10237000425542850571534285CF62307EF2613D00
:102380009B017EF2623D9B027EF4525E323D9B03D6
:102390007ECF0FF3583D3FA9168EAD16BC00A62088
:1023A000F2593D9B737ED0160FC00B2F000000002A
:1023B00000000000900901F86150F6134E88ED64AA
:1023C000DC86D058143B2B00E080E0DC58E051B4B0
:1023D000A09866A66BE000CCC75878AE30C070AE4F
:1023E0000663387C0630EE1C6A27498C955D1C9884
:1023F000CD9E0B800000E313FBCB0032160401B826
:1024000020020020222222222222222222222222F2
:1024100022222222222222222200222222004013D1
:102420000821A22815A04CC89E0A3A141532004D66
:102430000C0020B38FCE023303305840330F454495
:102440000CD2280D0CC3308F0000CEC430F3381AE4
:1024500007A89204A0F8E22DDEF331AC6144348A7F
:10246000CCA7F30800CE348FC54C607DE23922F34F
:1024700040523021E0C8034E6C2182685764E488E2
:102480004C08313085803ECD340A28DE28A03882C1
:1024900013398878FEC380E33C23381A390838A101
:1024A0009014D2CD375CA02244280425513432CD7B
:1024B000120AA9C191081ED4046A9152843906C532
:1024C0008852213E104302A122289E8ECEA34000B6
:1024D0000BB2041902C0A438787B63E2CD0F01CDA2
:1024E000314BDC32338F4E0E024E24A1C9221141F2
:1024F000118C0C1A3EB42478F0230603F30000007C
:1025000036870084333000CECC364373F3CC3CCBDB
:1025100014CA848222C32CB3D1E0AC29DA6C388F80
:102520003237CF2A28AC36CF8982F33C0BCE73DA10
:102530002C6A408E32CF02D82802C3CCEA2C38CC89
:1025400032E938D3ACE0AC388FF3386B8EF39C288B
:102550003823B3E6C83CC93C89A1363737CF20CCF5
:1025600031836C11025048A923CE0283DA4CA03685
:102570002B38CFA9B00ACECD02E468E3EC82CA883A
:10258000EC8A2890332A83D8AC004430342B932231
:10259000E03CA782B3E13CCECD42CED828683336AA
:1025A00082F3DC0CCEF3A860CE6830372A48481896
:1025B000903332A1FAAC2EF8FCFC2C7332A782CFF8
:1025C000A43E2B3E3F3B0F844510D14FFC8454FC6E
:1025D000411005101F101109F50E3D2BE014CC869B
:1025E000874185302ECFC5711CC73102C4B3CE9050
:1025F000208F820E81C3B025AB8011195A436438F5
:10260000011482CD14B6822121CD73382062854118
:1026100048D01C0E330034CD081442118014CE2152
:1026200046381C5238E00C8510388720214361421F
:1026300039853453C8E1400818F22125145E084258
:10264000018E2508E28450040401812005E139133C
:10265000140EE40C399046E18508E18549B800384C
:102660000F3B8781920038878590380BCE80733876
:1026700021C618013983020C122000CEB300218735
:10268000900851C8611408914138C6DFDD101286E8
:10269000C41900506038210A41E121D474188259CC
:1026A00060783C21282A0291802016185238211681
:1026B0000A4080E115EC335E848418A2880EE71C82
:1026C000D28C4218E45C08CE38136E20903F80E72D
:1026D0008C8010F23BCF066E118242118AD30A849D
:1026E00009E0238301404414515541114411110064
:1026F00000001014441451444414514444504444C0
:102700004011114111111110110110001404501148
:102710005450541400145455140555555541411541
:102720004555455505555545550150115445555587
:102730000500154155455515550150115455545531
:1027400055055555555005550540555515155455C4
:102750005551454555515545555505555515455501
:10276000555555554555515555555555555555156D
:1027700050441045511585180010111105510000E5
:1027800000051145511011114404015044414551B7
:1027900000145150515455555151145515111101F2
:1027A0000000144404510451045104510401001563
:1027B0001104415000504454554101515505054400
:1027C0005515141055514101455551555555445510
:1027D00011555151555154014045545555554505D4
:1027E00051100510454014114114840000002300CD
:1027F0000242F701448F3421C3C5334B43F00EA886
:102800000000918CFB954C576D8CAFEE2F918C098D
:10281000216D8C8D688CBB0C33918C1EEE2B0C774C
:10282000918CC078703CAE06A71297AEA346707824
:1028300070FC7038580E3CAE8CDF0637918C090B5B
:10284000A30C97666D8C687038EE8C4F793CF4F869
:10285000AE70AEF04ED80EE09CA01C12727F123CFF
:10286000F227693C3666D2F352728C53793CB88EAB
:10287000918CFB7DE3B03C04448C43A63CA63CB267
:102880003CA64C7BA646B748B252270866C3066BE7
:102890003BFB664708487223047206668C43A63CDD
